:100000000C9439220C946A220C946A220C946A2271
:100010000C946A220C946A220C946A220C946A2230
:100020000C946A220C946A220C946A220C946A2220
:100030000C946A220C9489740C946A220C946A229F
:100040000C946A220C946A220C946A220C946A2200
:100050000C946A220C946A220C946A220C943F74C9
:100060000C946A220C9409740C94DF730C946A2229
:100070000C946A220C946A220C946A220C946A22D0
:100080000C946A220C946A220C946A220C946A22C0
:100090000C946A220C946A220C946A220C942C759B
:1000A0000C946A220C946A220C946A220C946A22A0
:1000B0000C946A220C946A220C946A220C946A2290
:1000C0000C946A220C946A220C946A220C946A2280
:1000D0000C946A220C946A220C946A220C946A2270
:1000E0000C946A22FFFFFFFFFFFFFFFFFFFFFFFFF0
:1000F000FFFFFFFF0300000000000000FEFFFFFF06
:10010000FFFFFFFF838FB582DE030000FEDD63F794
:10011000F8FCFEFF034285C642040000FEED6D7749
:100120007BFDFEFF0322C5AA42040000FEF56D77A9
:100130007BFDFEFF0312A5924E040000FEF96EB097
:10014000BBFDFEFF03F29582C2030000FEF560379F
:10015000B8FDFEFF03128D8242000000FEED6EB777
:10016000DBFDFEFF031285825E000000FEDD6EB740
:10017000DBFDF0FF0300000000000000FEFFFFFFBA
:10018000FFFFFFFFFFFFFFFFFFFFFFFFFFFFFFFF7F
:10019000FFFFFFFF01000000000000000000000062
:1001A00000000080017C003C00380022003E001C62
:1001B0000F3C00800144004400440022002200A2C1
:1001C00000440080014411441F0407221F221F82A3
:1001D00007440E800144113C0404092204220482D5
:1001E000083C118001441F440404093C0422048299
:1001F000084401800144114404440720042204A25D
:10020000084411800144113C043801200422041CDC
:10021000073E0E800100000000000000000000000A
:10022000000000800100000000000000000000004D
:10023000000000800100000000000000000000003D
:10024000000000800100000000000000000000002D
:10025000000000800100000000000000000000001D
:1002600000000080210000000000000000000000ED
:1002700000000080390000000000000000000000C5
:100280000000008021600000000000000C0300005E
:100290000000008021100000000000008A0400001F
:1002A0000000008021100000000000008A0400000F
:1002B0000000008021100000000000009F040000EA
:1002C00000000080F9600000000000001103000041
:1002D000000000800100000000000000000000009D
:1002E000000000800100000000000000000000008D
:1002F000000000810100000000000000000000007C
:1003000000000081A58AFFFFFF07002011FEFFFF0C
:100310001F000080A5840000000400903802000047
:1003200010002C8DA5840000000400401002000085
:1003300010005495ED8A00000004002031020000F6
:10034000100054950180FFFFFF07009000FEFFFFA3
:100350001F00549501000000000000000000000094
:10036000000000800100000000000000000000000C
:10037000000000807100000000000000000000008C
:100380000000008089000000000000000000000064
:100390000000008041600000000000000C0300002D
:1003A0000000008021100000000000008A0400000E
:1003B0000000008011100000000000008A0400000E
:1003C0000000008089100000000000009F04000071
:1003D00000000080F9600000000000001103000030
:1003E000000000800100000000000000000000008C
:1003F000000000800100000000000000000000007C
:10040000000000800100000000000000000000006B
:1004100000000081A58AFFFFFF07002011FEFFFFFB
:100420001F000080A5840000000400903802000036
:1004300010002C8DA5840000000400401002000074
:1004400010005495ED8A00000004002031020000E5
:10045000100054950180FFFFFF07009000FEFFFF92
:100460001F00549501000000000000000000000083
:1004700000000080017044971218490700C7A5BB0F
:1004800001EC0E8001F86CB112244902804F2C89D6
:100490000222048001F854D39225490280CF349976
:1004A0006164048001F8449112244902804F248938
:1004B00002280480017044970C58460200C725B9F1
:1004C00002E60480010000000000000000000000BF
:1004D00000000080FFFFFFFFFFFFFFFFFFFFFFFFA8
:1004E000FFFFFFFFFFFFFFFFFFFFFFFFFFFFFFFF1C
:1004F000FFFFFFFF0100000000000000F8FFFFFF0A
:10050000FFFFFFFFE179495110224E14F8FFCF2E73
:100510007CBAFFFF210A2AD118225114F8FFB7B67E
:10052000BBBAFFFF210A1C5115225174F8FFBFBA54
:10053000BBBAFFFF213A0859123E9197F8FF8FBCD2
:10054000DB82FFFFE1091C5510221194F8FFBF3A2E
:100550001CBAFFFF21082A5310221194F8FFB7B6E6
:10056000EFBAFFFF2178495110220E74F8FFCFAE89
:10057000EFBAFFFF0100000000000000F8FFFFFFDE
:10058000FFFFFFFFFFFFFFFFFFFFFFFFFFFFFFFF7B
:10059000FFFFFFFF0100000000000000000000005E
:1005A00000000080010000000000000000000000CA
:1005B00000000080010000000000000000000000BA
:1005C00000000080010000000000000000000000AA
:1005D0000000008001600000000000000C0300002B
:1005E0000000008001100000000000008A040000EC
:1005F0000000008001100000000000008A040000DC
:100600000000008001100000000000009F040000B6
:1006100000000080016000000000000011030000E5
:100620000000008001000000000000000000000049
:100630000000008001000000000000000000000039
:100640000000008001000000000000000000000029
:10065000000000809554F8FFFF7F0000CC55F8FFA4
:10066000FF7F008055550800004000004A540800F4
:10067000004000805DD9080000400000CADC08008E
:100680000040008055510900004000005F540900FF
:100690000040008095D0F8FFFF7F0000D1D5F8FF23
:1006A000FF7F00800100000000000000000000004B
:1006B00000000080010000000000000000000000B9
:1006C00000000080010000000000000000000000A9
:1006D00000000080FFFFFFFFFFFFFFFFFFFFFFFFA6
:1006E000FFFFFFFF0100000000000000000000000D
:1006F00000000080E179495110E004C1B024CC8BA6
:1007000022070080210A2AD1181089A028154A88BA
:10071000A2040080210A1C51151051A0280E4A88FD
:10072000A2040080213A0859121021902404C9F92A
:1007300032070080E1091C55101051903C0E498889
:100740002A06008021082A531010898822955F8884
:10075000260500802178495110E00489A2A4D08B9D
:10076000A204008001000000000000000000000062
:1007700000000080FFFFFFFFFFFFFFFFFFFFFFFF05
:10078000FFFFFFFF0100000000000000000000006C
:1007900000000080010000000000000000000000D8
:1007A00000000080090000000000000002000000BE
:1007B00000000080090000000000000002000000AE
:1007C0000000008039000000000000000E00000062
:1007D000000000800900000000000000020000008E
:1007E00000000080091900000000000042360000EF
:1007F00000000080892A000000000000A212000012
:1008000000000080892A000000000000A2360000DD
:100810000000008039290000000000004E12000096
:100820000000008001000000000000000000000047
:100830000000008001000000000000000000000037
:100840000000008001000000000000000000000027
:1008500000000080FFFFFFFFFFFFFFFFFFFFFFFF24
:10086000FFFFFFFF0100000000000000000000008B
:1008700000000080017044971218490700C7A5BB0B
:1008800001EC0E8001F86CB112244902804F2C89D2
:100890000222048001F854D39225490280CF349972
:1008A0006164048001F8449112244902804F248934
:1008B00002280480017044970C58460200C725B9ED
:1008C00002E60480010000000000000000000000BB
:1008D00000000080FFFFFFFFFFFFFFFFFFFFFFFFA4
:1008E000FFFFFFFFFFFFFFFFFFFFFFFFFFFFFFFF18
:1008F000FFFFFFFF030000000000C0FFFFFFFFFF3E
:10090000FFFFFFFF030000000000C0FFFFFFFFFF2D
:10091000FFFFFFFF03EC3E8FFB1CC0FFFFFFFFFF4D
:10092000FFFFFFFF032208512212C0FFFFFFFFFF5E
:10093000FFFFFFFF036608512212C0FFFFFFFFFF0A
:10094000FFFFFFFF032808D1231EC0FFFFFFFFFFAB
:10095000FFFFFFFF032808512212C0FFFFFFFFFF28
:10096000FFFFFFFF03E6084F2212C0FFFFFFFFFF5C
:10097000FFFFFFFF030000000000C0FFFFFFFFFFBD
:10098000FFFFFFFFFFFFFFFFFFFFFFFFFFFFFFFF77
:10099000FFFFFFFFFFFFFFFFFFFFFFFFFFFFFFFF67
:1009A000FFFFFFFF0100000000000000000000400A
:1009B000000000C001000000000000000000004036
:1009C000000000C001000000000000000000004026
:1009D000000000C001000000000000000000004016
:1009E000000000C001000000000000000000004006
:1009F000000080C301000000000000000000004073
:100A00000000C0C70100000000000000000000401E
:100A10000000C0C70100000000000000000000400E
:100A20000040C0C7010000000000000000000040BE
:100A300000E080C301000000000000000000004052
:100A400000F001C0010000000000000000000040B4
:100A500000F803C00100000000000000000000409A
:100A600000F803C00100000000000000000000408A
:100A700000B803C0010000000000000000000040BA
:100A8000000802C00100000000000000000000405B
:100A9000000000C001000000000000000000004055
:100AA000000000C001000000000000000000004045
:100AB000000000C001000000000000000000004035
:100AC000F000E0C101000000000000000000004054
:100AD00078E0C0C3010000000000000000000040FA
:100AE0007CF0C1C7010000000000000000000040D1
:100AF0003EF081CF01000000000000000000004037
:100B00007CF0C1C7010000000000000000000040B0
:100B100078E0C0C3010000000000000000000040B9
:100B2000F000E0C1010000000000000000000040F3
:100B3000000000C0010000000000000000000040B4
:100B4000000000C0010000000000000000000040A4
:100B5000000802C00100000000000000000000408A
:100B600000B803C0010000000000000000000040C9
:100B700000F803C001000000000000000000004079
:100B800000F803C001000000000000000000004069
:100B900000F001C001000000000000000000004063
:100BA00000E000C001000000000000000000004064
:100BB000004000C0010000000000000000000040F4
:100BC000000000C001000000000000000000004024
:100BD000000000C001000000000000000000004014
:100BE00000773AC001000000000000000000004053
:100BF000009112C001000000000000000000004051
:100C0000009312C00100000000000000000000403E
:100C1000009112C001000000000000000000004030
:100C2000007712C00100000000000000000000403A
:100C3000000000C0010000000000000000000040B3
:100C4000000000C0FFFFFFFFFFFFFFFFFFFFFFFFF0
:100C5000FFFFFFFF01000000000000000000000097
:100C6000000000C0018EE8520223E900E0B87437AA
:100C700080DD01C0019F2D5682244900F089255155
:100C8000408400C0019F6A5AB2244900F09926337B
:100C90008C8C00C0019F285282244900F089245185
:100CA000008500C0018EE89201CB4800E0B82457CF
:100CB000C09C00C001000000000000000000000017
:100CC000000000C001000000000000000000000063
:100CD000000000C0FFFFFFFFFFFFFFFFFFFFFFFF60
:100CE000FFFFFFFF0000F03F502510201831881152
:100CF00008110C1904090408FC0F00000000F03F63
:100D00005025F03F783CF81DF81EFC1EFC0EFC0F31
:100D1000FC0F0000000820127014F824F828FC4989
:100D2000FC51FE13FE037000200000000000841040
:100D3000C8093006700790047005380EF80FC4110A
:100D400082200000FFFFFFFFFFFFFFFFFFFFFFFF0D
:100D5000FFFFFFFF4300000000000000FEFFFFFF59
:100D6000FFFFFFFF7B00000000000000FEFFFFFF11
:100D7000FFFFFFFF0B00000000000000FEFFFFFF71
:100D8000FFFFFFFF6B6CBEB3DF7117DDFEFFFFFFE0
:100D9000FFFFFFFF9B441419892092A9FEFFFFFF6C
:100DA000FFFFFFFF8B28141589E75339FEFFFFFF74
:100DB000FFFFFFFF8B28141389243249FEFFFFFF3A
:100DC000FFFFFFFF7310BFB9DC7797DDFEFFFFFF6A
:100DD000FFFFFFFF0314210000000000FEFFFFFFE4
:100DE000FFFFFFFFFFFFFFFFFFFFFFFFFFFFFFFF13
:100DF000FFFFFFFFFFFFFFFFFFFFFFFFFFFFFFFF03
:100E0000FFFFFFFF010000000000000000000040A5
:100E1000000000C0010000000000000000000040D1
:100E2000000000C0010000000000000000000040C1
:100E3000000000C0010000000000000000000040B1
:100E4000000000C0010000000000000000000040A1
:100E5000000080C30100000000000000000000400E
:100E60000000C0C7010000000000000000000040BA
:100E70000000C0C7010000000000000000000040AA
:100E80000040C0C70100000000000000000000405A
:100E900000E080C3010000000000000000000040EE
:100EA00000F001C001000000000000000000004050
:100EB00000F803C001000000000000000000004036
:100EC00000F803C001000000000000000000004026
:100ED00000B803C001000000000000000000004056
:100EE000000802C0FFFFFFFFFFFFFFFFFFFFFF7FC4
:100EF000000000C0010000000000000000000040F1
:100F0000000000C0010000000000000000000040E0
:100F1000000000C0C10778800388C0071CCF0340D1
:100F2000F000E0C14104884004884004A24004402D
:100F300078E0C0C34114894EF0884E748247E44083
:100F40007CF0C1C7411479441089442482C81341FC
:100F50003EF081CF41F4894410F14424824814408A
:100F60007CF0C1C74114894414814424A24814412F
:100F700078E0C0C341147984F38044241CC7E34063
:100F8000F000E0C10100000010000000000000407F
:100F9000000000C001000000100000000000004040
:100FA000000000C001000000000000000000004040
:100FB000000802C001000000000000000000004026
:100FC00000B803C001000000000000000000004065
:100FD00000F803C001000000000000000000004015
:100FE00000F803C0FFFFFFFFFFFFFFFFFFFFFF7FD2
:100FF00000F001C0010000000000000000000040FF
:1010000000E000C0010000000000000000000040FF
:10101000004000C00100000000000000000000408F
:10102000000000C0DDE344C9712E00000000004054
:10103000000000C045146D258A2400000000004017
:1010400000773AC045146D230AE401000000004017
:10105000009112C0451455258A240200000000406A
:10106000009312C0C5E354C971E4010000000040C0
:10107000009112C04100000000000000000000408C
:10108000007712C041000000000000000000004096
:10109000000000C00100000000000000000000404F
:1010A000000000C0FFFFFFFFFFFFFFFFFFFFFFFF8C
:1010B000FFFFFFFF01000000000000000000000033
:1010C000000000C0018EE8520223E900E0B8743746
:1010D00080DD01C0019F2D5682244900F0892551F1
:1010E000408400C0019F6A5AB2244900F099263317
:1010F0008C8C00C0019F285282244900F089245121
:10110000008500C0018EE89201CB4800E0B824576A
:10111000C09C00C0010000000000000000000000B2
:10112000000000C0010000000000000000000000FE
:10113000000000C0FFFFFFFFFFFFFFFFFFFFFFFFFB
:10114000FFFFFFFFFFFFFFFFFFFFFFFFFFFFFFFFAF
:10115000FFFFFFFF0300000000000000FEFFFFFF95
:10116000FFFFFFFF838FB582DE030000FEDD63F724
:10117000F8FCFFFF034285C642040000FEED6D77D8
:101180007BFDFFFF0322C5AA42040000FEF56D7738
:101190007BFDFFFF0312A5924E040000FEF96EB026
:1011A000BBFDFFFF03F29582C2030000FEF560372E
:1011B000B8FDFFFF03128D8242000000FEED6EB706
:1011C000DBFDFFFF031285825E000000FEDD6EB7CF
:1011D000DBFDFFFF0300000000000000FEFFFFFF3B
:1011E000FFFFFFFFFFFFFFFFFFFFFFFFFFFFFFFF0F
:1011F000FFFFFFFF010000000000000000000000F2
:10120000000000C0017C003C00380022003E001CB1
:101210000F3C00C00144004400440022002200A210
:10122000004400C0014411441F0407221F221F82F2
:1012300007440EC00144113C040409220422048224
:10124000083C11C001441F440404093C04220482E8
:10125000084401C00144114404440720042204A2AC
:10126000084411C00144113C043801200422041C2C
:10127000073E0EC00100000000000000000000005A
:10128000000000C00100000000000000000000009D
:10129000000000C00100000000000000000000008D
:1012A000000000C00100000000000000000000007D
:1012B000000000C00100000000000000000000006D
:1012C000000000C02100000000000000000000003D
:1012D000000000C039000000000000000000000015
:1012E000000000C02100000000000000000000001D
:1012F000000000C021600000000000000C0300009E
:10130000000000C021100000000000009204000056
:10131000000000C021100000000000009204000046
:10132000000000C021100000000000009E0400002A
:10133000000000C0F9600000000000001103000080
:10134000000000C0010000000000000000000000DC
:10135000000000C0010000000000000000000000CC
:10136000000000C0010000000000000000000000BC
:10137000000000C07100000000000000000000003C
:10138000000000C089000000000000000000000014
:10139000000000C08100000000000000000000000C
:1013A000000000C041600000000000000C030000CD
:1013B000000000C0211000000000000092040000A6
:1013C000000000C0111000000000000092040000A6
:1013D000000000C089100000000000009E04000012
:1013E000000000C0F96000000000000011030000D0
:1013F000000000C00100000000000000000000002C
:10140000000000C00100000000000000000000001B
:10141000000000C00100000000000000000000000B
:10142000000000C07100000000000000000000008B
:10143000000000C089000000000000000000000063
:10144000000000C08100000000000000000000005B
:10145000000000C061600000000000000C030000FC
:10146000000000C081100000000000009204000095
:10147000000000C081100000000000009204000085
:10148000000000C089100000000000009E04000061
:10149000000000C0716000000000000011030000A7
:1014A000000000C00100000000000000000000007B
:1014B000000000C00100000000000000000000006B
:1014C000000000C00100000000000000000000005B
:1014D000000000C0017044971218490700C7A5BB5F
:1014E00001EC0EC001F86CB112244902804F2C8926
:1014F000022204C001F854D39225490280CF3499C6
:10150000616404C001F8449112244902804F248987
:10151000022804C0017044970C58460200C725B940
:1015200002E604C00100000000000000000000000E
:10153000000000C0FFFFFFFFFFFFFFFFFFFFFFFFF7
:10154000FFFFFFFFFFFFFFFFFFFFFFFFFFFFFFFFAB
:10155000FFFFFFFF0300000000000000FEFFFFFF91
:10156000FFFFFFFF838FB582DE030000FEDD63F720
:10157000F8FCFFFF034285C642040000FEED6D77D4
:101580007BFDFFFF0322C5AA42040000FEF56D7734
:101590007BFDFFFF0312A5924E040000FEF96EB022
:1015A000BBFDFFFF03F29582C2030000FEF560372A
:1015B000B8FDFFFF03128D8242000000FEED6EB702
:1015C000DBFDFFFF031285825E000000FEDD6EB7CB
:1015D000DBFDFFFF0300000000000000FEFFFFFF37
:1015E000FFFFFFFFFFFFFFFFFFFFFFFFFFFFFFFF0B
:1015F000FFFFFFFF010000000000000000000000EE
:10160000000000C001FFFFFFFFFFFFFFFFFFFFFF24
:10161000FFFF00C001FFFFFFFFFFFFFFFFFFFFFF16
:10162000FFFF00C001FFFFFFFFFFFFFFFFFFFFFF06
:10163000FFFF00C001FFFFFFFFFFFFFFFFFFFFFFF6
:10164000FFFF00C001FFFFFFFFFFFFFFFFFFFFFFE6
:10165000FFFF00C001FFFFFFFFFFFFFFFFFFFFFFD6
:10166000FFFF00C001FFFFFFFFFFFFFFFFFFFFFFC6
:10167000FFFF00C001FFFFFFFFFFFFFFFFFFFFFFB6
:10168000FFFF00C001FFFFFFFFFFFFFFFFFFFFFFA6
:10169000FFFF00C001FFFFFFFFFFFFFFFFFFFFFF96
:1016A000FFFF00C00101000000000000000000007A
:1016B000008000C0010100000000000000000000E8
:1016C000008000C02101E00100000000000000E0F7
:1016D000008000C03901100100000000000000106F
:1016E000018000C0210108F098D9F0B83BFB3B0015
:1016F000018000C0210108089130091191491200B0
:10170000018000C0210108086110F1F15149F28007
:10171000008000C0210108086110091151411041E9
:10172000008000C021011009911089113141100180
:10173000008000C0F901E0F098F170BB9BE3F86015
:10174000008000C001010000001000000000000047
:10175000008000C00101000000380000000000000F
:10176000008000C001010000000000000000000037
:10177000008000C0710100000000000000000000B7
:10178000008000C08901FCFFFFFF0300FEFFFFFF98
:10179000018000C08101040000000200020000007E
:1017A000018000C0410104E04000020002A4FB00EF
:1017B000018000C0210104B06000020002A42000EA
:1017C000018000C0110104905000020002BC210001
:1017D000018000C0890104907800020002A420006A
:1017E000018000C0F90104F84900020002A42300AE
:1017F000018000C001010408010002000200000095
:10180000018000C00101FCFFFFFF0300FEFFFFFF9E
:10181000018000C001010000000000000000000085
:10182000008000C071010000000000000000000006
:10183000008000C0890100000000000000000000DE
:10184000008000C0810100000000000000000000D6
:10185000008000C0610100000000000000000000E6
:10186000008000C081FFFFFFFFFFFFFFFFFFFFFFC2
:10187000FFFF00C081FFFFFFFFFFFFFFFFFFFFFF34
:10188000FFFF00C089FFFFFFFFFFFFFFFFFFFFFF1C
:10189000FFFF00C071FFFFFFFFFFFFFFFFFFFFFF24
:1018A000FFFF00C001FFFFFFFFFFFFFFFFFFFFFF84
:1018B000FFFF00C001000000000000000000000069
:1018C000000000C001000000000000000000000057
:1018D000000000C0017044971218490700C7A5BB5B
:1018E00001EC0EC001F86CB112244902804F2C8922
:1018F000022204C001F854D39225490280CF3499C2
:10190000616404C001F8449112244902804F248983
:10191000022804C0017044970C58460200C725B93C
:1019200002E604C00100000000000000000000000A
:10193000000000C0FFFFFFFFFFFFFFFFFFFFFFFFF3
:10194000FFFFFFFFFFD0FFE0FFCFFF64FFD1FF32BB
:10195000380C060201FF64FFD0FFFE1F1C1F1E1F74
:101960001E1F1F1E1F1E1F00002200250028002B07
:10197000002E003100340002010000050108010BB7
:1019800001000020002300260029002C002F003237
:10199000000001000003010601090100000A0B021A
:1019A000090C0D0E080703040100000000000000F0
:1019B0000000000000000000000000000000000027
:1019C00000000000000000121110000000000000E4
:1019D0000000000000000000000000000000000007
:1019E0000000002100240027002A002D00300033D1
:1019F0000001010000040107010A0101021020207A
:101A00000808102040102040800201020108040252
:101A100001010204081020408080402010080402C8
:101A20000180040201804020100804020108040221
:101A30000101020408102040800102040810204027
:101A40008005050505070508080808020202020AC4
:101A50000A08080404040401010101010101010351
:101A600003030303030303040707070C0C0C0C0C0C
:101A70000C0C0C0202020206060606060606060BFF
:101A80000B0B0B0B0B0B0B00000080FFFFFFFFFF8E
:101A9000FFFFFF07000000000000C0FFFFFFFFFF87
:101AA000FFFFFF03000700F0FF0FC0FFFFFFFFFF76
:101AB000FFFFFF03C01F00000000E0FFFFFFFFFF6C
:101AC000FFFFFF01C01A00000000E0FFFFFFFFFF63
:101AD000FFFFFF01603700C0FF03F0FFFFFFFFFFC4
:101AE000FFFFFF00E03D00000000F0FFFFFFFFFFF1
:101AF000FFFFFF00603700000000F8FFFFFFFFFF5F
:101B0000FFFF7F00C01A00F0FF0FF8FFFFFFFFFF8D
:101B1000FFFF7F00C01F00000000FCFFFFFFFFFF72
:101B2000FFFF3F00000700000000FCFFFFFFFFFF7A
:101B3000FFFF3F00000000FFFFFFFFFFFFFFFFFF71
:101B4000FFFFFFFFFFFFFF0100000000000000009B
:101B50000000000000008001000000000000000004
:101B6000000000000000800100000080DD3174C42E
:101B7000151D0000000080010000004084502686F2
:101B8000B005000000008001000000808C50258519
:101B9000540D0000000080010000000085502787E0
:101BA0001405000000008001000000C09C30258565
:101BB000141D000000008001000000000000000073
:101BC0000000000000008001000000000000000094
:101BD0000000000000008001000000000000000084
:101BE0000000000000008001000000000000000074
:101BF00000000000000080011C000000FF1F00002A
:101C000000100000F0FF81017700000001100000CB
:101C100000100000F0FF8181F70000004513000074
:101C20000014000090138181F700000025150000CA
:101C30000014000050B581C1F70100002515000017
:101C40000014000050B18141760100004D130000E6
:101C50000015000090B581C1EF01000001100000E7
:101C600000150000F0FF8181DF000000FF1F000071
:101C700040150000B0AA8181F7000000240900008F
:101C800050150000B0AA810177000000240900006F
:101C900054150000A0AA81011C00000024090000C6
:101CA000FC1F0000C0FF81010000000000000000D8
:101CB00000000000000080010000000000000000A3
:101CC0000000000000008001000000000000000093
:101CD0000000000000008001000000000000000083
:101CE0000000000000008001000000000000000073
:101CF0000000000000008001000000000000000063
:101D00000000000000008001000000000000000052
:101D10000000000000008001000038000000800387
:101D200000000003000080010000440000004004A7
:101D300000008004000080010000BA00000040059F
:101D40000000400800008001000092000000C00771
:101D500000004008000080010000920000004005E3
:101D60000000800400008001000092000000400597
:101D70000000E01F00008001000044000000400758
:101D8000000090270000800100003800000040049F
:101D900000000843000080010000380000008003BC
:101DA00000000843000080010000380000008003AC
:101DB00000009024000080010000100000000001DD
:101DC000000060180000800100000000000000001A
:101DD0000000000000008001000000000000000082
:101DE0000000000000008001000000000000000072
:101DF00000000000000080FFFFFFFFFFFFFFFFFF6C
:101E0000FFFFFFFFFFFFFF010000000000000000D8
:101E10000000000000008021E0882E2530920E0096
:101E2000C7A5BB01EC0E8431F0D96225489204802D
:101E30004F2C890222048C39B0A9A6254B9204802C
:101E4000CD34996164049C31F08922254892048044
:101E50004F24890228048C21E0882E19B08C0400BC
:101E6000C725B902E604840100000000000000005C
:101E700000000000000080FFFFFFFFFFFFFFFFFFEB
:101E8000FFFFFFFFFFFFFF00000080FFFFFFFFFFDE
:101E9000FFFFFF07000000000000C0FFFFFFFFFF83
:101EA000FFFFFF03000000000000C0FFFFFFFFFF77
:101EB000FFFFFF03000000000000E0FFFFFFFFFF47
:101EC000FFFFFF01000000000000E0FFFFFFFFFF39
:101ED000FFFFFF01000000000000F0FFFFFFFFFF19
:101EE000FFFFFF00000000000000F0FFFFFFFFFF0A
:101EF000FFFFFF00000000000000F8FFFFFFFFFFF2
:101F0000FFFF7F00000000000000F8FFFFFFFFFF61
:101F1000FFFF7F00000000000000FCFFFFFFFFFF4D
:101F2000FFFF3F00000000000000FCFFFFFFFFFF7D
:101F3000FFFF3F00000000FFFFFFFFFFFFFFFFFF6D
:101F4000FFFFFFFFFFFFFF01000000000000000196
:101F50000020000000008001017000070800070158
:101F600000200000000080810140000428000101E1
:101F7000002000000000800101200002380007015D
:101F80000020000000008001011000042000040176
:101F90000020000000008001017000072000070100
:101FA000002000000000800100000000000000018F
:101FB00000200000000080810778800778800701FA
:101FC000002000000000804108844008844008018F
:101FD000002000000000802110022110022110FFCB
:101FE000FFFFFFFFFFFFFF21100221100221100160
:101FF00000200000000080211002211002211001A9
:102000000020000000008021100221100221100198
:10201000002000000000804108844008844008013E
:102020000020000000008081077880077880070189
:1020300000200000000080010000000000000001FE
:1020400000200000000080010000000000000001EE
:1020500000200000000080010000000000000001DE
:1020600000200000000080010000000000000001CE
:102070000020000000008009F2FFFF7F000048FF01
:10208000FFFFFFFFFFFFFF091300004000002401D6
:102090000020000000008009120000400000100134
:1020A00000200000000080091200004000004801EC
:1020B0000020000000008039F2FFFF7F00002401B3
:1020C000002000000000800100000000000000016E
:1020D000002000000000800100000000000000015E
:1020E000002000000000800100000000000000014E
:1020F0000020000000008009F7FFFF7F000048017A
:1021000000200000000080091400004000002401AD
:1021100000200000000080091200004000001001B3
:10212000002000000000800911000040000048FF6E
:10213000FFFFFFFFFFFFFF39F7FFFF7F00002401D4
:1021400000200000000080010000000000000001ED
:1021500000200000000080010000000000000001DD
:1021600000200000000080010000000000000001CD
:102170000020000000008009F7FFFF7F00004801F9
:10218000002000000000800914000040000024012D
:102190000020000000008009120000400000100133
:1021A00000200000000080091400004000004801E9
:1021B0000020000000008039F7FFFF7F00002401AD
:1021C000002000000000800100000000000000016D
:1021D000002000000000800100000000000000FF5F
:1021E000FFFFFFFFFFFFFF010000000000000001F4
:1021F00000200000000080FFFFFFFFFFFFFFFF0146
:102200000020000000008001010101010101010125
:1022100000200000000080113939393939391101A5
:1022200000200000000080797D45454545453D0181
:10223000002000000000807D6D45454545457D013D
:1022400000200000000080797D45454545453D0161
:102250000020000000008011393939393939110165
:1022600000200000000080010101010101010101C5
:1022700000200000000080FFFFFFFFFFFFFFFFFFC7
:10228000FFFFFFFFFFFFFF01050600FF0500FA014A
:10229000F0207FFF05FF05FF02003002152580803A
:1022A000800080053242A0A002556550F850F850D9
:1022B00002455570A0F050E0025565C8D0205898EE
:1022C000025565E080F890F00512228080022535E5
:1022D0004080808040022535804040408004334368
:1022E000A040A003334340E040012232408004314B
:1022F00041E002112180025565081020408002450E
:1023000055F0909090F0022535C040404040024585
:1023100055F010F080F0024555F010F010F0024535
:1023200055909090F010024555F080F010F0024565
:1023300055E080F090F0024555F0102040400245F5
:1023400055F090F090F0024555F090F010700313A6
:1023500023800080021424800080800235452040C4
:10236000804020033343E000E002354580402040B8
:1023700080024555F010700040025565F888B8A8F5
:10238000F0024555F090F09090024555E0A0F09095
:10239000F0024555F0808080F0024555E090909025
:1023A000E0024555F080F080F0024555F080F08065
:1023B00080024555F080B090F00245559090F09025
:1023C00090023545E0404040E00245553010109005
:1023D000F00245559090E0909002455580808080B5
:1023E000F0025565F8A8A8A8A802455590D0B0906D
:1023F00090024555F0909090F0024555F09090F085
:1024000080024555F09090B0F0024555F090F0A054
:10241000B0024555F080F010F0023545E0404040F4
:102420004002455590909090F00245559090A0A0A4
:1024300040025565A8A8A8A8F8024555909060905C
:10244000900245559090F010F0024555F0106080D4
:10245000F0022535C0808080C00255658040201084
:1024600008022535C0404040C005324240A002412C
:1024700051F005223280400243537090F0024454E0
:1024800080F090F0023343E080E002445410F0907A
:10249000F0024353F0A0700244547040F0400144F5
:1024A00054F090F02002445480F090900214248064
:1024B0000080800115258000808080024454809037
:1024C000E09002142480808080025363F8A8A80260
:1024D0004353F09090024353F090F0014454F09035
:1024E000F080014454F090F010023343E080800209
:1024F0004353F040F002344440E0406002435390C4
:1025000090F0024353909060025363A8A8F80233FE
:1025100043A040A00144549090F010024353F02097
:10252000F002354560408040600215258080808043
:1025300080023545C0402040C005425250A0FF00F7
:10254000101000FE0A06A7089500FFFE0EFE0BFE07
:102550001010201000FEAAAA0001800000018000D7
:102560004A51EA505A51C99E000180000001800082
:102570000001800055551010201000FEAAAA00018D
:102580008000000180003993C252325F8A527193F9
:1025900080000001800000018000555510102010BF
:1025A00000FEAAAA00018000000180003BA5C12412
:1025B000311989247125800000018000000180000C
:1025C00055551010201000FEAAAA0001800000013D
:1025D00080007BA5C1247919C124792580000001E0
:1025E00080000001800055551010201000FEAAAA9E
:1025F000000180000001800079BFC2487A49C248CA
:10260000798980000001800000018000555510107C
:10261000201000FEAAAA00018000000180007A4D6F
:10262000C2527B53C2D67A4F800000018000000165
:10263000800055551010201000FEAAAA000180004D
:102640000001800031A5CA287A31CA2849A5800036
:10265000000180000001800055551010201000FE80
:10266000AAAA000180000001800073D1CA1073D1B2
:10267000CA1073DF80000001800000018000555502
:102680001010201000FEAAAA0001800000018000A6
:102690001E3991401E3191081E718000000180009A
:1026A0000001800055551010201000FEAAAA00015C
:1026B00080000001800022F9A2203E21A2202221D8
:1026C000800000018000000180005555101020108E
:1026D00000FEAAAA000180000001800020F9A0806D
:1026E00020F9A0803E818000000180000001800070
:1026F00055551010201000FEAAAA0001800000010C
:10270000800022F9A22022219420082180000001CB
:1027100080000001800055551010201000FEAAAA6C
:1027200000018000000180003EF9A0803EF9A080F9
:1027300020818000000180000001800055551010AC
:10274000201000FEAAAA00018000000180001EF1F6
:10275000A08820F1A0901E89800000018000000167
:10276000800055551010201000FEAAAA000180001C
:10277000000180001E71A0881C8982883C71800045
:10278000000180000001800055551010201000FE4F
:10279000AAAA00018000000180001EF9A0201C21CF
:1027A00082203CF980000001800000018000555526
:1027B0001010201000FEAAAA000180000001800075
:1027C000391DA510251DA51039DD800000018000F0
:1027D0000001800055551010201000FEAAAA00012B
:1027E0008000000180007189CA184A09CA08719DD9
:1027F000800000018000000180005555101020105D
:1028000000FEAAAA00018000000180007199CA049C
:102810004A09CA10719D80000001800000018000FB
:1028200055551010201000FEAAAA000180000001DA
:1028300080007199CA044A19CA0471998000000184
:1028400080000001800055551010201000FEAAAA3B
:1028500000018000000180007185CA0C4A15CA1C65
:102860007185800000018000000180005555101026
:10287000201000FEAAAA00018000000180004993F8
:10288000EA546A59DBD44A538000000180000001F9
:10289000800055551010201000FEAAAA00018000EB
:1028A000000180003453C29A3117891271138000DD
:1028B000000180000001800055551010201000FE1E
:1028C000AAAA00018000000180007BB9C1247939E7
:1028D000C124793980000001800000018000555535
:1028E0001010201000FEAAAA000180000001800044
:1028F0003325C4B447ADC4A434A5800000018000D2
:102900000001800055551010201000FEAAAA0001F9
:102910008000000180003E89A0D83EA9A0883E89A1
:10292000800000018000000180005555101020102B
:1029300000FEAAAA00018000000180003A5DC25298
:10294000325D8A52719D800000018000000180008C
:1029500055551010201000FEAAAA000180000001A9
:10296000800079CFC2107991C0507B8F8000000128
:1029700080000001800055551010201000FEAAAA0A
:1029800000018000000180001E7190801E61901087
:1029900010E18000000180000001800055551010FA
:1029A000201000FEAAAA00018000000180000E7124
:1029B0009080166192100EE18000000180000001FD
:1029C000800055551010201000FEAAAA00018000BA
:1029D000000180001C7192801C61941012E1800043
:1029E000000180000001800055551010201000FEED
:1029F000AAAA000180000001800012719280126179
:102A000092100CE18000000180000001800055550B
:102A100000000008000E010A0A080400808080807F
:102A200080808000808005040408020888888888E7
:102A3000060A0A080100242424FC4848FC909090CF
:102A4000070A0A080100107C9290701C12927C10F8
:102A5000070A0A0801006294946810102C52528CE4
:102A6000070A0A0801003844442830528A848C72CC
:102A700001040408040880808080030C0C0803FF14
:102A8000204040808080808080404020030C0C08E3
:102A900002FF804040202020202020404080070767
:102AA00007080101109254385492100707070801D3
:102AB00001101010FE1010100204040803FEC040A4
:102AC0004080040101080204F0020202080300C071
:102AD000C0060A0A080100040408101020204080E3
:102AE00080060A0A0801003048848484848484486B
:102AF00030050A0A0802002060A0202020202020A3
:102B0000F8060A0A080100788484041820408080AE
:102B1000FC060A0A080100788484043804048484CA
:102B200078060A0A080100081828488888FC08085E
:102B300008060A0A080100FC808080F80404048466
:102B400078060A0A08010038408080F8848484846A
:102B500078060A0A080100FC04040808081010108E
:102B600010060A0A080100788484847884848484A6
:102B700078060A0A080100788484847C0404040826
:102B800070020707080301C0C0000000C0C00209AE
:102B9000090803FFC0C0000000C0404080050909CB
:102BA0000802000810204080402010080605050893
:102BB0000102FC000000FC0509090801008040201A
:102BC000100810204080060A0A0801007884840456
:102BD000081010001010060A0A080100384494ACCE
:102BE000A4A4A49C403C060A0A080100304848847A
:102BF00084FC84848484060A0A080100F88484849E
:102C0000F884848484F8060A0A08010078848480A1
:102C1000808080848478060A0A080100F088848411
:102C20008484848488F0060A0A080100FC8080807D
:102C3000F880808080FC060A0A080100FC80808001
:102C4000F88080808080060A0A08010078848480E9
:102C5000809C84848C74060A0A080100848484841D
:102C6000FC8484848484050A0A080200F820202059
:102C70002020202020F8070A0A0801003E08080842
:102C8000080808888870060A0A080100848890A04D
:102C9000C0C0A0908884060A0A0801008080808055
:102CA0008080808080FC060A0A0801008484CCCCE5
:102CB000B4B484848484060A0A08010084C4C4A4C9
:102CC000A494948C8C84060A0A0801007884848475
:102CD000848484848478060A0A080100F884848441
:102CE000F88080808080070B0B0801FF7884848443
:102CF000848484B4CC7806060A0A080100F8848427
:102D000084F89088888484060A0A080100788484FC
:102D100080601804848478070A0A080100FE1010F5
:102D200010101010101010060A0A08010084848484
:102D300084848484848478070A0A08010082828259
:102D400044444428281010060A0A08010084848498
:102D500084B4B4CCCC8484060A0A08010084844874
:102D600048303048488484070A0A080100828244B7
:102D700044281010101010060A0A080100FC040470
:102D8000081020408080FC030C0C0804FFE08080C9
:102D90008080808080808080E0060A0A08010080B0
:102DA000804020201010080404030C0C0801FFE0F0
:102DB00020202020202020202020E00603030801DE
:102DC000093048840701010801FFFE0303030802DC
:102DD0000A8040200608080801007884047C848466
:102DE0008C74060B0B080100808080B8C484848436
:102DF00084C4B80608080801007884808080808434
:102E000078060B0B080100040404748C8484848409
:102E10008C74060808080100788484FC808084781B
:102E2000050B0B08010018202020F820202020206E
:102E300020060B0B0801FE04748888887040788493
:102E40008478060B0B080100808080B8C4848484D9
:102E5000848484050B0B08020020200060202020C1
:102E6000202020F8050D0D0801FE080800180808AC
:102E700008080808089060060B0B08010080808095
:102E80008890A0C0A0908884050B0B0802006020E9
:102E90002020202020202020F8070808080100EC2E
:102EA00092929292929292060808080100B8C48405
:102EB00084848484840608080801007884848484D7
:102EC000848478060A0A0801FEB8C484848484C411
:102ED000B88080060A0A0801FE748C848484848C7D
:102EE000740404060808080100B8C4848080808047
:102EF000800608080801007884806018048478053A
:102F00000A0A080100202020F8202020202018068E
:102F100008080801008484848484848C740608086A
:102F200008010084848448484830300708080801B4
:102F300000829292929292926C0608080801008494
:102F400084483030488484060A0A0801FE84848458
:102F500084844C34040478060808080100FC040842
:102F600010204080FC030C0C0803FF608080404070
:102F700080804040808060010E0E0804FE808080CA
:102F80008080808080808080808080030C0C08029C
:102F9000FFC020204040202040402020C0070303E5
:102FA00008010862928C1010201000FEAAAA0001ED
:102FB00080000001800073D1CA104BD1CA1073DFAA
:102FC0008000000180000001800055551010201085
:102FD00000FEAAAA0001800000018000719DCA5273
:102FE00073D3C252425D8000000180000001800066
:102FF00055551010201000FEAAAA00018000000103
:103000008000499DCA527A5DCA50499180000001F2
:1030100080000001800055551010201000FEAAAA63
:1030200000018000000180007393CA52739FCA128E
:1030300072138000000180000001800055551010BF
:10304000201000FEAAAA00018000000180004B931E
:10305000EA525B9FCA524B9380000001800000013E
:10306000800055551010201000FEAAAA0001800013
:103070000001800074B9A6A425A5A4A474B9800099
:10308000000180000001800055551010201000FE46
:10309000AAAA00018000000180004BD1EA105BD198
:1030A000CA104BDF800000018000000180005555F0
:1030B0001010201000FEAAAA00018000000180006C
:1030C00039CDC212319F8852739380000001800075
:1030D0000001800055551010201000FEAAAA000122
:1030E00080000001800079CDC212799FC0527B938D
:1030F0008000000180000001800055551010201054
:1031000000FEAAAA00018000000180004B9DC9209A
:103110007919C9044939800000018000000180004C
:1031200055551010201000FEAAAA000180000001D1
:10313000800025DDA4843C85A484249980000001BE
:1031400080000001800055551010201000FEAAAA32
:10315000000180000001800045CDC4904489A8840E
:10316000109980000001800000018000555510106A
:10317000201000FEAAAA0001800000018000721D3C
:10318000CA127213C21243DD8000000180000001E8
:10319000800055551010201000FEAAAA00018000E2
:1031A000000180007213CA127213C21243CD800054
:1031B000000180000001800055551010201000FE15
:1031C000AAAA00018000000180000E2189200E21A2
:1031D0008A200921800000018000000180005555EF
:1031E0001010201000FEAAAA00018000000180003B
:1031F00039DDC202318D8850739F8000000180004C
:103200000001800055551010201000FEAAAA0001F0
:1032100080000001800039DDC202318D8842739D3B
:103220008000000180000001800055551010201022
:1032300000FEAAAA000180000001800071CFCA1020
:103240004A0DCA0271DD800000018000000180008B
:1032500055551010201000FEAAAA000180000001A0
:1032600080007245CA4C7245C244418F8000000103
:1032700080000001800055551010201000FEAAAA01
:103280000001800000018000725DCA42724DC25090
:10329000419F800000018000000180005555101002
:1032A000201000FEAAAA00018000000180003B9DC2
:1032B000C1203119890471398000000180000001AA
:1032C000800055551010201000FEAAAA00018000B1
:1032D0000001800039D3C212421FC21239D38000CC
:1032E000000180000001800055551010201000FEE4
:1032F000AAAA00018000000180002289B6882AA9BC
:10330000A2D822898000000180000001800055556C
:103310001010201000FEAAAA000180000001800009
:103320003B8DC252339F8A127213800000018000CD
:103330000001800055551010201000FEAAAA0001BF
:103340008000000180007B8DC2527B9FC2127A13E5
:1033500080000001800000018000555510102010F1
:1033600000FEAAAA0001800000018000398FC2502F
:10337000324D8A42719D8000000180000001800072
:1033800055551010201000FEAAAA0001800000016F
:103390008000339BC42225A394A2639B800000017C
:1033A00080000001800055551010201000FEAAAAD0
:1033B000000180000001800039DDC20832098A085E
:1033C00071DD800000018000000180005555101063
:1033D000201000FEAAAA000180000001800039DD53
:1033E000C2084189C0483B9D800000018000000167
:1033F000800055551010201000FEAAAA0001800080
:10340000000180000EF990200C2182201C218000F8
:10341000000180000001800055551010201000FEB2
:10342000AAAA000180000001800031CFCA10499192
:10343000C850338F80000001800000018000555586
:103440001010201000FEAAAA0001800000018000D8
:103450001C8992D81CA990881089800000018000E6
:103460000001800055551010201000FEAAAA00018E
:10347000800000018000338FCA507B91CA104A0F30
:103480008000000180000001800055550000000808
:10349000000E010A0A08040080800080808080807D
:1034A0008080070A0A08010010107C929090927C9C
:1034B0001010070A0A0801001C202020F8202020F4
:1034C0007CC2060808080101844878484878488486
:1034D000070A0A08010082442810FE10FE1010108E
:1034E000010A0A08040080808080000080808080BB
:1034F000060A0A0801007884807884847804847835
:1035000004020208020C9090080A0A0800003C42DB
:1035100099A5A1A1A599423C0507070802057008D5
:1035200078887800F80609090801002424484890A2
:1035300048482424060404080100FC040404101074
:10354000201000FEAAAA000180003A63C25433C9C9
:103550008A48724980000001800003C18000000198
:1035600080005555080A0A0800003C42B9A5A5B9D3
:10357000A9A5423C06010108010BFC030404080252
:103580000A40A0A040070909080101101010FE1010
:10359000101000FE0507070802057088087080807B
:1035A000F80507070802057088087008887003038B
:1035B0000308030A204080080A0A0800FE4242422B
:1035C00042424266594080060C0C0801FF7CF4F42C
:1035D000F4F47414141414141C020202080304C03A
:1035E000C00302020802FE20C003070708020520EC
:1035F00060A0202020200507070802057088888821
:103600007000F806090908010090904848244848CD
:103610009090060A0A08010044C4485050242C54D3
:103620009C84060A0A08010044C4485050283444C7
:10363000889C060A0A080100C4244830D0242C546F
:103640009C84060A0A08010010100010106084848F
:103650008478060E0E080100601800003048488487
:1036600084FC84848484060E0E0801001860000027
:103670003048488484FC84848484060E0E0801004B
:10368000304800003048488484FC84848484060EDA
:103690000E080100649800003048488484FC84844B
:1036A0008484060E0E080100484800003048488413
:1036B00084FC84848484060E0E08010030483000A7
:1036C0003048488484FC84848484070A0A08010002
:1036D0003E509090FE909090909E060C0C0801FE3B
:1036E000788484808080808484781060060E0E0840
:1036F000010060180000FC808080F880808080FCE1
:10370000060E0E08010018600000FC808080F88022
:10371000808080FC060E0E08010030480000FC800E
:103720008080F880808080FC060E0E0801004848EA
:103730000000FC808080F880808080FC050E0E08F0
:10374000020060180000F82020202020202020F80F
:10375000050E0E08020030C00000F82020202020B6
:10376000202020F8050E0E08020060900000F820CE
:1037700020202020202020F8050E0E080200909026
:103780000000F82020202020202020F8070A0A0826
:10379000000078444242F24242424478060E0E084B
:1037A00001006498000084C4C4A4A494948C8C8404
:1037B000060E0E080100601800007884848484845A
:1037C00084848478060E0E08010018600000788456
:1037D0008484848484848478060E0E080100304832
:1037E000000078848484848484848478060E0E089F
:1037F00001006498000078848484848484848478BC
:10380000060E0E08010048480000788484848484F1
:1038100084848478060505080102844830488406BB
:103820000C0C0801FF0474888C9494A4A4C444B8BC
:1038300080060E0E080100601800008484848484D1
:103840008484848478060E0E0801001860000084C9
:10385000848484848484848478060E0E0801003075
:1038600048000084848484848484848478060E0ED2
:10387000080100484800008484848484848484840B
:1038800078070E0E08010018600000828244442868
:103890001010101010060B0B0801008080F08884B7
:1038A0008488F0808080060A0A0801007088889069
:1038B000B0888484A498060C0C08010060180000ED
:1038C0007884047C84848C74060C0C0801001860D5
:1038D00000007884047C84848C74060C0C0801003D
:1038E000304800007884047C84848C74060C0C08B6
:1038F0000100649800007884047C84848C74060C35
:103900000C080100484800007884047C84848C748E
:10391000060D0D08010030483000007884047C84D6
:10392000848C740708080801007C92127E909092A3
:103930007C060A0A0801FE788480808080847810E2
:1039400060060C0C08010060180000788484FC807C
:10395000808478060C0C08010018600000788484CC
:10396000FC80808478060C0C080100304800007848
:103970008484FC80808478060C0C08010048480090
:1039800000788484FC80808478050C0C080200C0D8
:1039900030000060202020202020F8050C0C0802B8
:1039A0000030C0000060202020202020F8050C0CF2
:1039B0000802006090000060202020202020F805F0
:1039C0000C0C080200909000006020202020202095
:1039D000F8060C0C08010064182844047C848484D4
:1039E000848478060C0C08010064980000B8C48434
:1039F0008484848484060C0C08010060180000781C
:103A000084848484848478060C0C08010018600087
:103A1000007884848484848478060C0C0801003047
:103A20004800007884848484848478060C0C08011F
:103A300000649800007884848484848478060C0C64
:103A400008010048480000788484848484847806CF
:103A50000707080101300000FC000030060A0A08D0
:103A600001FF04788C9494A4A4C47880060C0C08FC
:103A70000100601800008484848484848C74060CA3
:103A80000C080100186000008484848484848C7491
:103A9000060C0C080100304800008484848484846F
:103AA0008C74060C0C08010048480000848484844F
:103AB00084848C74060E0E0801FE18600000848455
:103AC0008484844C34040478050C0C0802FE808045
:103AD000F088888890A0C0808080060E0E0801FEC5
:103AE0004848000084848484844C34040478000AA8
:103AF00010FEFC060197031520FFFE09FE07FE00DD
:103B00000000060001010707060200808080808017
:103B10000080030303060104A0A0A0050808060115
:103B2000FF5050F85050F850500408080601FF208C
:103B300070806010906020060707060000E0A4C8AF
:103B4000305C9418060606060000304060948874C5
:103B50000103030602048080800309090602FE2097
:103B600040408080804040200309090601FE8040DB
:103B70004020202040408005040406000320D82077
:103B8000500505050600012020F820200203030649
:103B900001FE404080040101060103F0010202061B
:103BA000020080800609090600FF0408101020208A
:103BB000404080040707060100609090909090605C
:103BC00004070706010020E020202020F00407075A
:103BD000060100609010204080F0040707060100F5
:103BE00060901060109060050707060000103050CC
:103BF00090F81010040707060100F08080E0101014
:103C0000E0040707060100708080E09090600407E0
:103C100007060100F090102020404004070706012D
:103C2000006090906090906004070706010060902B
:103C300090701010E0010505060200808000808071
:103C40000206060601FE40400040408003050506CE
:103C500001012040804020040303060102F000F02F
:103C60000305050602018040204080040606060187
:103C7000006090204000400608080600FF38449C81
:103C8000A8A89C4038060606060000702848784818
:103C9000CC050606060000F048704848F004060609
:103CA000060100609080809060050606060000F026
:103CB00048484848F0050606060000F848704048A5
:103CC000F8050606060000F848705040E0040606B5
:103CD000060100609080B09060060606060000CCE9
:103CE00048784848CC050606060100F82020202028
:103CF000F80506060601007810109090600606068A
:103D0000060000D850605048E4050606060100E0B1
:103D100040404048F805060606010088D8A8A88853
:103D2000D8060606060000DC48685848C80406069F
:103D3000060100609090909060050606060100F074
:103D400048487040E00407070601FF60909090909B
:103D50006070060606060000F048487048E4040655
:103D6000060601007080601090E00506060600005F
:103D7000F8A820202070060606060000CC48484817
:103D80004830060606060000DC8850505020060623
:103D900006060000DC88A8A85050050606060100AB
:103DA000D850202050D8050606060100D88850209B
:103DB0002070040606060100F090204090F00209F1
:103DC000090602FEC080808080808080C0050909CD
:103DD0000601FF80804040202010100802090906DB
:103DE00002FEC040404040404040C0050303060181
:103DF000042050880601010600FEFC0202020601B2
:103E000006804005050506000060107090680507F3
:103E100007060000C04070484848F0040505060148
:103E200000609080906005070706010030107090D8
:103E30009090680405050601006090E0906004071A
:103E4000070601003040F0404040F005070706013A
:103E5000FE689090907010E0060707060000C040D2
:103E600070484848EC050707060100200060202044
:103E700020F80309090601FE2000E0202020202070
:103E8000C0050707060000C04058506050D805071D
:103E900007060100602020202020F8060505060006
:103EA00000D0A8A8A8AC060505060000B048484800
:103EB000EC04050506010060909090600507070678
:103EC00000FEB04848487040F00507070601FE684C
:103ED000909090701038050505060100B8404040EC
:103EE000F004050506010070806010E00507070674
:103EF00001004040F040404830060505060000D86B
:103F000048484834060505060000CC442828100619
:103F10000505060000ACA8A85050050505060000E0
:103F2000D8502050D80507070600FED8484848302A
:103F300020C0040505060100F0204090F0030909A7
:103F40000602FE2040404080404040200109090612
:103F500002FE8080808080808080800309090602C4
:103F6000FE804040402040404080040202060103A1
:103F700050A0FFFFFFFFFFFFFFFFFFFFFFFFFFFF5F
:103F8000FFFFFFFFFFFFFFFFFFFFFFFFFFFFFFFF41
:103F9000FFFFFF0000000600010107070602FE8088
:103FA0000080808080800408080601FF2020708047
:103FB000807020200607070600003840F8202044C3
:103FC000FC05050506000188705070880507070686
:103FD00000008850F820F820700109090602FE80D0
:103FE00080800000808080800408080601FF7080C7
:103FF0006090906010E0030101060205A00607072B
:104000000600003048B4A4B4483004050506010198
:10401000E010D000F00603030600016CD86C050325
:1040200003060002F80808040101060103F0060770
:10403000070600003048BCB4AC483004010106015A
:1040400005F00403030601046090600506060600FF
:10405000002020F82000F803040406020360A040BA
:10406000E0030404060203E04020C002020206024C
:104070000540800607070600FED8484848744040BF
:104080000608080600FF7CA8A8682828286C0102FA
:104090000206020280800303030601FE4020C003E3
:1040A0000404060203C04040E00405050601016067
:1040B000906000F0060303060101D86CD8060707DC
:1040C000060000C04448F42C5C8406070706000084
:1040D000C04448FC34489C060707060000E044281A
:1040E000D42C5C840407070600FE200020204090AA
:1040F000600609090600002010007028487848CCA6
:104100000609090600001020007028487848CC06EF
:1041100009090600002050007028487848CC06099C
:10412000090600002850007028487848CC06080886
:1041300006000050007028487848CC06090906009F
:10414000001028107028487848CC060606060000A3
:104150007C305C70909C0408080601FE60908080B2
:10416000906020C0050909060000201000F8487082
:104170004048F8050909060000102000F848704082
:1041800048F8050909060000205000F8487040482A
:10419000F80508080600005000F848704048F80587
:1041A0000909060000402000F820202020F8050919
:1041B00009060000102000F820202020F805090939
:1041C000060000205000F820202020F805080806EE
:1041D00000005000F820202020F805060606000008
:1041E000F048E84848F0060909060000285000DCBD
:1041F00048685848C804090906010040200060903A
:1042000090909060040909060100204000609090A1
:104210009090600409090601002050006090909081
:10422000906004090906010050A0006090909090F1
:1042300060040808060100A000609090909060055E
:104240000505060001885020508806060606000075
:104250003448586848B0060909060000201000CC10
:104260004848484830060909060000102000CC489C
:1042700048484830060909060000102800CC484884
:104280004848300608080600005000CC4848484816
:1042900030050909060000102000D8885020207041
:1042A000050606060000C070487040E006060606D7
:1042B00000003048584454C8050808060000402053
:1042C000006010709068050808060000102000606B
:1042D00010709068050808060000205000601070FB
:1042E000906805080806000050A0006010709068F3
:1042F0000507070600005000601070906805090966
:104300000600002050200060107090680605050629
:1043100000006C947C90EC0407070601FE6090801E
:10432000906020C00408080601004020006090F062
:1043300080700408080601002040006090F0807042
:1043400004080806010040A0006090F08070040797
:1043500007060100A0006090F080700508080600C4
:104360000040200060202020F8050808060000100A
:10437000200060202020F8050808060000205000DA
:1043800060202020F805070706000050006020206C
:1043900020F8040808060100D060A070909090609A
:1043A000060808060000285000B0484848EC0408F9
:1043B0000806010040200060909090600408080604
:1043C0000100102000609090906004080806010031
:1043D00040A000609090906004080806010050A082
:1043E000006090909060040707060100A0006090B4
:1043F0009090600505050600012000F800200606E3
:10440000060600000438586848B006080806000090
:10441000201000D84848483406080806000010203C
:1044200000D848484834060808060000205000D844
:10443000484848340607070600005000D848484856
:1044400034050A0A0600FE102000D84848483020EB
:10445000C00509090600FEC040704848487040E0A9
:104460000509090600FE5000D84848483020C00021
:10447000507611241FBECFEFD1E2DEBFCDBF00E0EA
:104480000CBF14E0A0E0B2E0EEE0F0E201E00BBF10
:1044900002C007900D92AC3DB107D9F72BE0ACED0F
:1044A000B4E001C01D92A930B207E1F712E2C9E3FE
:1044B000D2E200E006C021970109802FFE010E9490
:1044C000A48FC833D10780E00807A9F70E947F783E
:1044D0000C9405900C940000089580E00895CF920C
:1044E000DF92EF92FF92CF93DF93EC01072E000C47
:1044F000880B990B0E942D8E6B017C0120E030E02F
:1045000040E45FE30E94DD8E20E030E048E452E4C6
:104510000E94928D0E94FA8DC617D707D4F020E032
:1045200030E040EA5FE3C701B6010E94DD8E20E083
:1045300030E048E452E40E94928D20E030E040E810
:104540005FE30E942A8D0E94FA8D21E06C177D079F
:104550000CF420E0822F90E0DF91CF91FF90EF905C
:10456000DF90CF9008958F929F92AF92BF92CF929B
:10457000DF92EF92FF920F931F93CF93DF93FC0193
:1045800020813181E0918D08F0918E0801E010E0EA
:104590002E173F070CF040C0D901AA0FBB1FE091B6
:1045A0008B08F0918C08EA0FFB1FA080B180890175
:1045B000009510950170112720FD20C02CE93FEFD8
:1045C000EA016B017C014901840E951EB401C5010D
:1045D00086DF892BB1F48C0E9D1EB401C5017FDFEF
:1045E000892B41F5BE01680D791DC50178DF23E0F7
:1045F00030E0892B41F40FEF1FEF0EC024E630E0CE
:10460000DFCF21E030E0F6018081918101968217B1
:1046100093079CF491838083C801DF91CF911F9110
:104620000F91FF90EF90DF90CF90BF90AF909F9051
:104630008F90089522E030E0E6CF11821082F701DA
:10464000808191810196E6CF2F923F924F925F92A7
:104650006F927F928F929F92AF92BF92CF92DF9292
:10466000EF92FF920F931F93CF93DF9300D000D070
:10467000CDB7DEB78AE599E090938C0880938B08DC
:104680008091220A90E090938E0880938D0880910B
:104690005609853009F0ABC580915C0990915D09A0
:1046A000885891098D35910508F054C08091220AEF
:1046B000843021F580915E0990915F09809747973A
:1046C000E8F4809160099091610909970997B0F425
:1046D00010928A08109289088FEF9FEFDC01809377
:1046E000850890938608A0938708B093880881E096
:1046F00090E090938208809381086CC38091220A95
:10470000843440F180915E0990915F09825491094F
:104710008E9700F530E020E080E090E0DC01F901C8
:10472000E05AF64F408151814950510949305105B5
:1047300088F4F901EE59F64F4081518147515109F2
:104740004231510528F1408151814650510947308D
:10475000510580F18091220A8A3108F460C080916D
:104760005A0990915B09843F914048F510928A085C
:10477000109289088FEF9FEFDC018093850890935A
:104780008608A0938708B093880889E090E0B1CFAD
:10479000880F991FAA1FBB1F81602C5F3F4F2038D5
:1047A000310509F0BCCF20E230E030938A08209335
:1047B000890895CF880F991FAA1FBB1FEECF809144
:1047C0005C0990915D0985974B9748F5E5E5F9E01F
:1047D00082E090E040E050E0BA01A091220A9C0102
:1047E0002F5F3F4FA217130609F00CF4F1C021858B
:1047F0003285275031092730310508F0E9C023857B
:104800003485235131092F30310508F4D4C0238574
:1048100034852A5031092930310508F4D4C08091FB
:10482000220A8A3108F43FC080915A0990915B09AD
:104830008032934008F49ACF80915C0990915D0991
:10484000C697869780F580915E0990915F09C6971B
:10485000869748F5E5E5F9E083E090E040E050E038
:10486000BA01A091220A9C012F5F3F4FA2171306A5
:1048700009F00CF4D3C0238534852C5031092B303A
:10488000310508F0CBC025853685255231092B31FD
:10489000310508F4B6C0258536852C5031092A30FB
:1048A000310508F4B6C08091220A823238F1809135
:1048B0005C0990915D090697079700F5E5E5F9E039
:1048C00082E090E040E050E0BA01DC0111962091D6
:1048D000220A2A171B0609F00CF4CCC02185328568
:1048E0002E5131092731310508F4AFC021853285B9
:1048F0002C5031092B30310508F4B6C08091220AC2
:104900008D3008F405C181E090E09C838B831A828E
:10491000198249E753E0BE016F5F7F4FCE010396D6
:1049200022DE892B09F0F4C049E753E0BE016F5F36
:104930007F4FCE01039617DE8C01019709F0E8C086
:1049400049E753E0BE016F5F7F4FCE0103960BDE58
:104950005C01892B09F0DCC0C12CD12C760120919F
:10496000220A8B819C812817190609F00CF4A4C037
:1049700049E753E0BE016F5F7F4FCE010396F3DD41
:104980004C0149E753E0BE016F5F7F4FCE010396B4
:10499000EADDB1E08B16910409F085C0892B09F09E
:1049A000B7C0CC0CDD1CEE1CFF1C6894C0F8EFEF08
:1049B000AE1ABE0AD4CF440F551F661F771F416041
:1049C000029634960ACF440F551F661F771FF8CF03
:1049D00001979595879590938A08809389080C97FD
:1049E0002CF410928A081092890819CF40938508F8
:1049F00050938608609387087093880882E090E05F
:104A000078CE440F551F661F771F4160029634967B
:104A100028CF440F551F661F771FF8CF0197959534
:104A2000879590938A08809389080C972CF41092AC
:104A30008A081092890837CF4093850850938608DA
:104A40006093870870938808A0CE440F551F661F97
:104A5000771F4160238534853496235031092530F2
:104A6000310538F4029631CF440F551F661F771F6A
:104A7000F1CFCD0101979595879590938A08809302
:104A8000890840972CF410928A081092890836CF32
:104A90004093850850938608609387087093880830
:104AA0008AE090E026CE892899F5019789F5CC0C0B
:104AB000DD1CEE1CFF1C7BCFB0928A08A0928908F7
:104AC000C0928508D0928608E0928708F092880804
:104AD00083E090E09093820880938108C801269635
:104AE0000FB6F894DEBF0FBECDBFDF91CF911F91FF
:104AF0000F91FF90EF90DF90CF90BF90AF909F907D
:104B00008F907F906F905F904F903F902F9008957F
:104B100080918D0890918E08181619060CF081C0AE
:104B2000E0918B08F0918C0881E090E09C838B836E
:104B30008281938189974E9708F073C082E090E05C
:104B40009C838B83848195810B970A9708F069C0B9
:104B500083E090E09C838B831A8219824CEB51E0B6
:104B6000BE016F5F7F4FCE010396FDDC7C01892B78
:104B700009F057C04CEB51E0BE016F5F7F4FCE0193
:104B80000396F1DC8C01019709F04BC0412C512CAC
:104B9000320120918D0830918E088B819C81821783
:104BA00093070CF0E4C04CEB51E0BE016F5F7F4F08
:104BB000CE010396D8DC5C01F3E0EF16F10431F18D
:104BC0004CEB51E0BE016F5F7F4FCE010396CBDC13
:104BD0006C0123E0E216F10459F44CEB51E0BE0104
:104BE0006F5F7F4FCE010396BEDCC816D906C9F4AD
:104BF000A114B10409F4ADC0AA94AB2891F4CD2856
:104C000081F4440C551C661C771CADC04CEB51E084
:104C1000BE016F5F7F4FCE010396A5DCA816B906D3
:104C200079F2E0918B08F0918C0882819381C6978C
:104C3000869778F5848195814B97459750F5DF01EC
:104C400016967F0126ECE20EF11C20E030E040E0F9
:104C500050E060E070E080E090E00D911C911197D1
:104C60000950110908301105A0F412960D911C91FC
:104C70001397015111090D30110508F487C01296E0
:104C80000D911C911397045011090530110508F47A
:104C9000A4C082819381895791098335910568F574
:104CA0008091220A893348F184819581CA97899736
:104CB00020F59F012A5F3F4FC12CD12C760143E0A4
:104CC00050E0D9016D917C9111976A50710969305A
:104CD000710598F412966D917C9113976651710944
:104CE0006131710508F47DC012966D917C9166501A
:104CF00071096730710508F4A3C08091220A8232DD
:104D000009F0A3C0828193810A97099708F09DC09A
:104D1000A091220AB0E0A150B048AA0FBB1FAE0F6D
:104D2000BF1F8D919C910A97099708F08EC0109231
:104D30008A08109289088FEF9FEFDC018093850825
:104D400090938608A0938708B093880888E090E045
:104D5000D0CCCA94CD2809F064CF440C551C661CF5
:104D6000771C689440F8AFEFEA1AFA0A12CFF09273
:104D70008A08E092890840928508509286086092DD
:104D800087087092880884E090E0A4CE01E00E9439
:104D9000BC8F21601496AE15BF0509F05ECF20933D
:104DA000850830938608409387085093880800E26E
:104DB0000E94D78F209383083093840887E090E087
:104DC000909382088093810880E390E090938A0812
:104DD0008093890801E010E081CE01E00E94BC8F41
:104DE000D9CFD701C601880F991FAA1FBB1F6C011D
:104DF0007D016894C0F84E5F5F4F2C5F3F4F4B338F
:104E0000510509F05ECF9F012A583F4FD9012D91DE
:104E10003C912A5031092930310508F06ECF2CE140
:104E200030E030938A0820938908C0928508D09298
:104E30008608E0928708F09288088CE090E059CCD0
:104E4000CC0CDD1CEE1CFF1CD6CF828193818957D0
:104E500091098335910560F58091220A813240F1F4
:104E600084819581CA97899718F59F012A5F3F4FE2
:104E7000C12CD12C760143E050E0D9016D917C9199
:104E800011976A5071096930710590F412966D910D
:104E90007C911397665171096131710598F11296F1
:104EA0006D917C91665071096730710508F457C0A7
:104EB000828193818C549109C59708F084C08091B8
:104EC000220A843009F050C08481958180974797E9
:104ED00008F04AC0868197810997099708F044C075
:104EE00010928A08109289088FEF9FEFDC0180935F
:104EF000850890938608A0938708B09388088BE074
:104F000090E0F7CBD701C601880F991FAA1FBB1FDE
:104F10006C017D016894C0F84E5F5F4F2C5F3F4F7E
:104F20004332510509F0A9CF9F012A5B3F4FD901B8
:104F30002D913C912A5031092930310508F0B8CF24
:104F400020E130E030938A0820938908C0928508D8
:104F5000D0928608E0928708F0928808F7CECC0CB1
:104F6000DD1CEE1CFF1CD8CF8091220A843458F13E
:104F70008481958189549109C39728F59F012A5FFF
:104F80003F4FBF016A577F4FC12CD12C7601D90109
:104F90004D915C911197495051094930510598F450
:104FA00012964D915C91139746515109413151052B
:104FB00008F4C0C012964D915C914650510947309B
:104FC000510508F4D6C08091220A8634C0F182814E
:104FD00093810C970B9798F5848195810997099790
:104FE00070F5868197818C974F9748F580859185DC
:104FF00089974D9720F59F01265F3F4FC12CD12CFB
:10500000760145E050E0D9016D917C9111976C508B
:1050100071096B30710598F412966D917C9113971C
:105020006E5171096731710508F4A8C012966D912F
:105030007C91695071096930710508F4CEC0809186
:105040008D0890918E089E838D8306970CF4CAC0BC
:105050008F010E5F1F4F85ECC82E8DE9D82E8CE195
:10506000E82E81E8F82E93E0292E312CD8011496F1
:105070006D917C911597AD90BC9090E080E00E947E
:105080002B8E2B013C01B50190E080E00E942B8E1D
:105090004B015C012DEC3CEC4CE45FE30E94DD8EA7
:1050A0009B01AC01C301B2010E948E8DF0E0E0E0F3
:1050B00087FD14C02DEC3CEC4CE45FE3C301B2016E
:1050C0000E94DD8E9B01AC01C501B4010E948E8D52
:1050D000E2E0F0E087FD02C0E1E0F0E0A701960128
:1050E00063E971E080E091E00E94408F6F01FF0F63
:1050F000EE08FF08C626D726E826F926BFEF2B1AAA
:105100003B0A0E5F1F4FED81FE81E215F30509F0AA
:10511000ADCFC0928508D0928608E0928708F092C1
:10512000880880E290E090938A08809389088FEF46
:105130009FEFDFCAD701C601880F991FAA1FBB1FA7
:105140006C017D016894C0F82C5F3F4F261737072C
:1051500009F01DCF20E230E030938A0820938908BF
:10516000C0928508D0928608E0928708F09288085D
:10517000C6CECC0CDD1CEE1CFF1CE6CFD701C60151
:10518000880F991FAA1FBB1F6C017D016894C0F88E
:105190004E5F5F4F2C5F3F4F4534510509F033CFD1
:1051A0009F0126573F4FD9012D913C912C50310939
:1051B0002B30310508F043CF20E230E030938A08ED
:1051C00020938908C0928508D0928608E0928708CB
:1051D000F09288088DE090E08CCACC0CDD1CEE1CAF
:1051E000FF1CD6CF82E0809356091092220A10E06D
:1051F00000E074CC2091D30A3091D40A28173907E3
:1052000099F19093D40A8093D30A009739F12091B1
:10521000E60AFC01211129C03596E491E093E70AE2
:105220000C96FC0184918093E80A8091E70A082E8D
:10523000000C990B2091E80A821B910927FD939598
:105240002091E90A203441F0829FC001112426E018
:10525000969587952A95E1F78093EA0A8DE692E282
:105260009093E50A8093E40A0895213031F43F9643
:10527000E491E093E70A4096D4CF3D96E491E09321
:10528000E70A0E96CECFAF92BF92CF92DF92EF9207
:10529000FF920F931F93CF93DF93DC0128E030E060
:1052A00081E0AA24AA94B12C0FE010E043E2E42E9E
:1052B000F12C57EDC52ED12C9C911196ED91FC91BE
:1052C0001297592F5095462F4823A1F1F894428107
:1052D000452342834181492B4183E7012197F1F71F
:1052E0004281942B92837894F6013197F1F7880FDD
:1052F0002150310909F7F8941196ED91FC9112971C
:1053000091818C918095892381831196ED91FC91F7
:10531000129792818C918095892382837894DF9172
:10532000CF911F910F91FF90EF90DF90CF90BF90A2
:10533000AF900895F8944281452342834181492BDF
:105340004183E5012197F1F74281942B9283789470
:10535000F801CBCFFC01538D448D252F30E0842FF5
:1053600090E0821B930B541710F0CF96089501978D
:105370000895FC01918D828D981761F0A28DAE0F7A
:10538000BF2FB11D5D968C91928D9F5F9F73928F01
:1053900090E008958FEF9FEF0895FC01918D828D2D
:1053A000981731F0828DE80FF11D858D90E00895FA
:1053B0008FEF9FEF0895FC01918D228D892F90E052
:1053C000805C9F4F821B91098F7399270895FC0180
:1053D000A48DA80FB92FB11DA35ABF4F2C91848D56
:1053E00090E001968F739927848FA689B7892C93B3
:1053F000A089B1898C91837080648C93938D848D06
:10540000981306C00288F389E02D80818F7D808308
:105410000895EF92FF920F931F93CF93DF93EC01C8
:1054200081E0888F9B8D8C8D98131AC0E889F9894B
:10543000808185FF15C09FB7F894EE89FF8960834E
:10544000E889F98980818370806480839FBF81E0CF
:1054500090E0DF91CF911F910F91FF90EF90089511
:10546000F62E0B8D10E00F5F1F4F0F731127E02EEC
:105470008C8D8E110BC00FB607FCFACFE889F98925
:10548000808185FFF5CFCE01A2DFF2CFEB8DEC0F4F
:10549000FD2FF11DE35AFF4FF0829FB7F8940B8F59
:1054A000EA89FB8980818062D0CFCF93DF93EC01C2
:1054B000888D8823B1F0AA89BB89E889F9898C9104
:1054C00085FD03C0808186FD0CC00FB607FCF7CFB9
:1054D0008C9185FFF2CF808185FFEDCFCE0177DF04
:1054E000EACFDF91CF9108958FE998E064DF21E062
:1054F000892B09F420E0822F089580E090E0892B29
:1055000021F0F2DF81110E94000080E090E0892B01
:1055100049F080E090E0892B29F00E940000811181
:105520000E94000080E090E0892B49F080E090E04C
:10553000892B29F00E94000081110E94000080E068
:1055400090E0892B49F080E090E0892B29F00E94BF
:10555000000081110C940000089580E991E0089505
:1055600008950895AF92BF92CF92DF92EF92FF928B
:105570000F931F93CF93DF936C017B018B01040F7B
:10558000151FEB015E01AE18BF08C017D10759F017
:105590006991D601ED91FC910190F081E02DC60159
:1055A0001995892B79F7C501DF91CF911F910F9143
:1055B000FF90EF90DF90CF90BF90AF900895815013
:1055C000823108F05AC0E82FF0E08827E551F54D08
:1055D0008F4F0C94A48F0B2B0F2BFD2A032B072B23
:1055E0003D2B122B182B1C2B222B262B2A2B302B3E
:1055F000342B3D2B382B3E2B422B809180008F7714
:10560000809380000895809180008F7DF9CF8091F4
:105610008000877FF5CF84B58F7784BD089584B5EA
:105620008F7DFBCF8091B0008F778093B00008957D
:105630008091B0008F7DF9CF809190008F7780931B
:1056400090000895809190008F7DF9CF8091900017
:10565000877FF5CF8091A0008F778093A000089579
:105660008091A0008F7DF9CF8091A000877FF5CF3A
:10567000809120018F7780932001089580912001EF
:105680008F7DF9CF80912001877FF5CFCF93DF9376
:10569000282F30E0F901E556F64E8491F901E550E6
:1056A000F64ED491F901EF5BF54EC491CC2399F0FD
:1056B000811185DFEC2FF0E0EE0FFF1FEF57F64E64
:1056C000A591B491EC91ED2381E090E009F480E0A4
:1056D000DF91CF91089580E090E0FACF1F93CF93B0
:1056E000DF93282F30E0F901E556F64E8491F90159
:1056F000E550F64ED491F901EF5BF54EC491CC2301
:10570000A1F0162F81115BDFEC2FF0E0EE0FFF1FF1
:10571000E959F64EA591B4918FB7F894EC91111117
:1057200008C0D095DE23DC938FBFDF91CF911F910E
:105730000895DE2BF8CFCF93DF9390E0FC01E55086
:10574000F64E24918F5B954EFC0184918823C9F01D
:1057500090E0880F991FFC01EF51F64EA591B4918E
:10576000FC01E959F64EC591D49161110DC09FB766
:10577000F8948C91209582238C9388812823288308
:105780009FBFDF91CF910895623051F49FB7F89495
:105790003C91822F809583238C93E8812E2BEFCF31
:1057A0008FB7F894EC912E2B2C938FBFEACF1F93D9
:1057B000CF93DF93182FEB0161E0BDDF209731F429
:1057C00060E0812FDF91CF911F9188CFCF3FD1052E
:1057D00011F461E0F6CFE12FF0E0E556F64EE491EA
:1057E000E150E23108F0B3C0F0E08827E550F44D15
:1057F0008F4F0C94A48F0D2C152C1A2C242C2E2C8E
:10580000A72C382C402C482C522C5C2C662C752C48
:105810007F2CA72C892C932C9D2C84B5806884BD6B
:10582000C7BDDF91CF911F91089584B5806284BD7B
:10583000C8BDF7CF80918000806880938000D093AE
:105840008900C0938800EDCF8091800080628093B2
:105850008000D0938B00C0938A00E3CF80918000BA
:10586000886080938000D0938D00C0938C00D9CF46
:105870008091B00080688093B000C093B300D1CF16
:105880008091B00080628093B000C093B400C9CF13
:1058900080919000806880939000D0939900C0938D
:1058A0009800BFCF80919000806280939000D09349
:1058B0009B00C0939A00B5CF809190008860809340
:1058C0009000D0939D00C0939C00ABCF8091A0002E
:1058D00080688093A0008091A0008F7B8093A000BF
:1058E000D093A900C093A8009CCF8091A0008062B3
:1058F0008093A000D093AB00C093AA0092CF809178
:10590000A00088608093A000D093AD00C093AC004D
:1059100088CF80912001806880932001D093290155
:10592000C09328017ECF8091200180628093200166
:10593000D0932B01C0932A0174CF809120018860FD
:1059400080932001D0932D01C0932C016ACFC038E1
:10595000D1050CF03ECF34CF3FB7F8948091660765
:1059600090916707A0916807B091690726B5A89B39
:1059700005C02F3F19F00196A11DB11D3FBFBA2FE1
:10598000A92F982F8827BC01CD01620F711D811DA1
:10599000911D42E0660F771F881F991F4A95D1F726
:1059A00008954F925F926F927F929F92AF92BF92B3
:1059B000CF92DF92EF92FF920F931F93CF93DF93DB
:1059C00000D0CDB7DEB7F0903C0980913F099091AF
:1059D0004009A0914109B0914209892B8A2B8B2B58
:1059E000D1F0BADF00919B0810919C0820919D088E
:1059F00030919E08601B710B820B930B00913F0945
:105A000010914009209141093091420960177107B6
:105A100082079307D0F2A0DF60939B0870939C08E5
:105A200080939D0890939E08E0914709F091480962
:105A3000309759F0409143095091440960914509CC
:105A4000709146098F2D1995F82E009199081091A3
:105A50009A084F2C512C712C612C0115110509F459
:105A60005EC0D8011C96EC901C9780913D099091E6
:105A70003E098436910510F41C961C92D801ED91D4
:105A8000FC91A280B38019821A821B82FF2089F1C7
:105A9000F8013696D12CC12C2191222319F1928044
:105AA000992001F130E050E040E02F5F3F4F4F4F31
:105AB0005F4FC301B2010E94408F9B01AC01892D51
:105AC00090E0B0E0A0E0BC01CD016F5F7F4F8F4F51
:105AD0009F4F0E94408FA1E0B0E0AC0FBD1FAC0D06
:105AE000BD1D8C93BFEFCB1ADB0A83E0C816D1042F
:105AF00099F6D8011D964D915C911E9712966D9165
:105B00007C919E012F5F3F4FC801F5011995D80187
:105B10001C96EC921C9714960D911C919ECF80912F
:105B20009708909198089C012F5F3F4F30939808F9
:105B30002093970849970CF445C08FB7F8942091AB
:105B40008F083091900840919108509192088FBF32
:105B5000E0919708F091980888EE93E0E89FB001F3
:105B6000E99F700DF89F700D1124072E000C880B13
:105B7000990BC0909308D0909408E0909508F0900D
:105B800096082C193D094E095F090E94828F3093B7
:105B90003E0920933D0910929808109297082FB75C
:105BA000F89480918F0890919008A0919108B091FD
:105BB00092082FBF8093930890939408A093950820
:105BC000B09396080F900F900F90DF91CF911F9197
:105BD0000F91FF90EF90DF90CF90BF90AF909F908C
:105BE0007F906F905F904F9008958F929F92AF92A9
:105BF000BF92CF92DF92EF92FF924B015C01ACDE3D
:105C00006B017C01A9DE6C197D098E099F09683E34
:105C1000734081059105B0F321E0821A9108A10833
:105C2000B10888EEC80E83E0D81EE11CF11C811477
:105C30009104A104B10431F7FF90EF90DF90CF9071
:105C4000BF90AF909F908F900895CF92DF92EF9288
:105C5000FF920F931F93CF93DF93EC018FB7F894CC
:105C6000C0908F08D0909008E0909108F090920832
:105C70008FBF88810BDD2981892B09F087C0211115
:105C80005DC08C819D81AE81BF81B701A601481B9B
:105C9000590B6A0B7B0B88899989B0E0A0E08417C7
:105CA0009507A607B70708F049C01A821B8281E052
:105CB0008983C886D986EA86FB868A899B89892B4F
:105CC000E9F58C899D89892BC9F581E090E055C063
:105CD0008C899D89009719F490E080E04EC048853A
:105CE00059856A857B8597018601041B150B260B58
:105CF000370BB901A801B0E0A0E084179507A6070B
:105D0000B70750F78C859D85AE85BF85B701A60185
:105D1000481B590B6A0B7B0B8E899F89B0E0A0E072
:105D200084179507A607B707B8F681E08B83CC8662
:105D3000DD86EE86FF8682E090E01FC08A818111B9
:105D4000C7CF8A899B89009719F2488559856A854A
:105D50007B8597018601041B150B260B370BB901B8
:105D6000A801B0E0A0E084179507A607B70708F0E0
:105D7000AFCF81E08A8383E090E0DF91CF911F91E4
:105D80000F91FF90EF90DF90CF900895222309F4B8
:105D9000A3CF88859985AA85BB85B701A601481B35
:105DA000590B6A0B7B0B88899989B0E0A0E08417B6
:105DB0009507A607B70708F08FCF1982CC82DD823E
:105DC000EE82FF828A899B89892B29F48C899D899F
:105DD000892B09F481CF8A8181117ECF8B8191E05B
:105DE000892790E0CACF62E0FC018081A4CCFC014D
:105DF00061819081492F50E08281282F30E0EBE5CE
:105E0000F9E181E0861730F47491270F311D8F5F1F
:105E10003196F8CF633020F0937011F42F5F3F4F2D
:105E20006DE671E0469FC001479F900D569F900D13
:105E3000112405964D5F5F4F5695479556954795AA
:105E4000840F951F820F931F67E070E00C945B8FA7
:105E50000F931F93CF93DF93FC01A681B781C58178
:105E6000D0E033E0D695C7953A95E1F7362F3770F5
:105E7000E0E8F0E08F0102C0159507953A95E2F74A
:105E8000FC018281481B4C9FC0014D9F900D112445
:105E9000669566956695680F792F711DA60FB71FD9
:105EA0008C91E02F222339F0E82BEC93DF91CF91F6
:105EB0001F910F910895E095E823F7CFFB014181F1
:105EC000DC0112962C911297421760F013962C91D8
:105ED0001397241738F0608115962C91621710F4EF
:105EE0002481B6CF0895FC0180819281980F92831E
:105EF0002181921760F494819F5F94839381890F2D
:105F0000821710F08FEF820F838381E0089580E085
:105F10000895FC0112828081815083831482089548
:105F2000DB01ED91FC9119940F931F93CF93DF93B5
:105F30001F92CDB7DEB70091D10A1091D20AE0913D
:105F4000000BF091010B82E0199530E020E04AE06F
:105F5000B8018FEC9AE0E4DF182FE091000BF0918C
:105F6000010B83E01995E091000BF091010B80E0AB
:105F70001995112399F16091D10A7091D20A9E016D
:105F80002F5F3F4F46E48FEC9AE0CADF8981809310
:105F9000CF0A6091D10A7091D20A9E012F5F3F4FC4
:105FA00047E48FEC9AE0BCDF89818093D00A60914E
:105FB000D10A7091D20A30E020E048E48FEC9AE0F8
:105FC000AFDF8093DA0A6091D10A7091D20A22E0A1
:105FD0003BE047E18FEC9AE0A3DF11E0812F0F90C7
:105FE000DF91CF911F910F910895CF93DF9380910F
:105FF000080B811104C081E08093080B95DFC091EC
:10600000D10AD091D20AE091000BF091010B82E00D
:106010001995E091000BF091010B81E0199530E0AA
:1060200020E044E1BE018FEC9AE07ADF22E03BE021
:1060300047E1BE018FEC9AE073DFE091000BF09135
:10604000010B80E0DF91CF9119940F931F93CF93B1
:10605000E091DD0AF091DE0A309719F08FEC9AE0BA
:1060600019950091D10A1091D20AE091000BF0919C
:10607000010B82E01995E091000BF091010B81E09A
:10608000199530E020E045E1B8018FEC9AE048DF57
:10609000C82F882339F022E03BE047E1B8018FECBC
:1060A0009AE03EDFE091000BF091010B80E0199542
:1060B0008C2FCF911F910F910895EF92FF920F9324
:1060C0001F93CF93DF93082F162FC42FD42FF82EB2
:1060D000F40EEE24EA948F2D8D1BD83078F58C2F9A
:1060E000887F800F9C2F96959695969528EF929F86
:1060F000C00D1124CC23B1F197E0C9276091D10ADA
:106100007091D20A8093EB0A1093EC0A1092EE0A77
:10611000CF5FC7708FEF90E001C0880FCA95EAF794
:106120008093ED0A2BEE3AE04BE38FEC9AE0DF919F
:10613000CF911F910F91FF90EF90F2CE6091D10A15
:106140007091D20A8093EB0A1093EC0A1092EE0A37
:10615000E092ED0A2BEE3AE04BE38FEC9AE0E0DEC2
:10616000D850B9CFDF91CF911F910F91FF90EF9051
:1061700008950F931F93CF93DF93182FC62F042FEB
:10618000D62FD20F402F6C2F812F97DFCF5FCD13EB
:10619000F9CFDF91CF911F910F910895EBECFAE0C9
:1061A0006681778180A38EE281A381E083A380EF63
:1061B00082A32BEE3AE04BE38FEC9AE0B1CE0B9644
:1061C000FC01849108950A96FC0184910895FC01D4
:1061D00084910895FCDF882321F0823011F083E060
:1061E000089586E00895FC01E60FF11D849190E08A
:1061F000982F88273196E4918E0F911D089568E0BD
:10620000F2CF66E0F0CF2EE93FE0009709F4089561
:10621000F9013197F1F70197F8CF30914407409198
:1062200043075091420760914107A0913F07B09109
:106230004007E0913D07F0913E079FB790933C07E0
:10624000F8949C91392B9C91492398E087FF0EC0CC
:106250003C93880F2081262320832081252B2083B7
:106260009150A1F780913C078FBF08954C93F1CFD7
:10627000CF93C62F811118C088EFCFDF8C2F807F7E
:10628000CCDF8C2F8295807FC8DF88E290E0FC0114
:106290003197F1F7FC013197F1F7FC013197F1F7F4
:1062A0000197F1F7CF910895813041F78AEFE5CF5B
:1062B00090E0FC01EF5BF54EE491F0E0EE0FFF1F84
:1062C000E959F64E259134913093400720933F07CA
:1062D00070E0FB01EF5BF54EE491F0E0EE0FFF1F85
:1062E000E959F64E2591349130933E0720933D07AE
:1062F0008550964EFC018491809344076550764EFC
:10630000FB0164916093420760956093410780951B
:10631000809343070895860F911DFC0183A18F3F51
:1063200011F0642FDBC90895EF92FF920F931F9332
:10633000CF93DF93EC01142F79016150673008F09F
:1063400035C0E62FF0E08827E755FE4C8F4F0C94C0
:10635000A48FB0312B32E531DE31F231F631283203
:106360007E0183E2E80EF11C8E01005D1F4FF701F4
:1063700081917F018F3F39F061E0DDD961E0F70164
:1063800031978081ABD9E016F10689F740E062E0F1
:10639000CE01C1DF41E064E0CE01BDDF40E065E059
:1063A000CE01B9DF6FA188A583DF1EA281E0DF9156
:1063B000CF911F910F91FF90EF9008958BA160E016
:1063C0008F3FA1F3CE01A7DFF1CF411103C040E021
:1063D00062E0F8CF41E062E0CE019DDF6FA188A5C9
:1063E00067DFE4CF642F8EA143DFE0CF8EA1811160
:1063F00014C088EF12DFC8E2D0E0111112C088E2A9
:1064000090E0FC013197F1F7FC013197F1F7FC01C5
:106410003197F1F70197F1F7C9CF813061F78AEF32
:10642000E9CFF7018081807FF8DEF70181917F015C
:106430008295807FF2DE1150CE010197F1F7DDCF1A
:10644000F70164918EA114DFFFEFEF1AFF0A1150DC
:106450001111F6CFABCF4EA3A9CFDB011496ED916E
:10646000FC9130E020E065E01994DB011496ED9199
:10647000FC9130E020E062E01994DB011496ED918C
:10648000FC9130E020E063E019949F92AF92BF92BC
:10649000CF92DF92EF92FF920F931F93CF93DF93F0
:1064A0007C018B01942E69012AE0421749F185E1B4
:1064B000481709F482C0F801C281D381F2E39F1624
:1064C00009F41BC1F91508F4BEC025E1921609F4C0
:1064D00018C187E1981609F426C194E19912E2C027
:1064E000EE81FF818D8124E0829FC00111248E0FF7
:1064F0009F1F11928E179F07E1F7CE010ADDD2C0D0
:10650000DB011496ED91FC9130E020E043E061E086
:10651000199580E094E4A92E99E1B92EF501C49172
:1065200081110FC081E0CF3F41F04C2FB801C7016E
:1065300094DF882309F4BFCF80E0BFEFAB1ABB0A1A
:10654000EDCF4FEFCF3F91F3CE3F09F4B4CFC03F33
:1065500098F7C03E30F04C2F4F70B801C70185DF6F
:10656000EBCFC03D30F04C2F4F70B801C70185DF35
:10657000E3CFC03CE8F0D8011496ED91FC9130E0F7
:1065800020E040E064E0C7011995C295C07FCE5F6E
:10659000D0E0CE0138DED8011496ED91FC9130E0C8
:1065A00020E041E064E0C7011995CE012CDEC4CFA4
:1065B000C7FDC2CF8C2F90E0F9CFFB01A280B38042
:1065C00040E0C70152DF41E0B801C70156DFD50105
:1065D0001296CC9112971696AD90BC90D0E2DC0F3B
:1065E00040E0B801C70141DF4EE3B801C70135DF24
:1065F000C03208F54C2F4068B801C7012EDF40E8D3
:10660000B801C7012ADF41E0B801C7012EDFD80178
:106610001496ED91FC91950140E166E0C701199552
:10662000B0E1AB0EB11CCF5FCD13DACF40E0B801C3
:10663000C70123DF40CF40EE4C0F4068B801C701CF
:106640000CDF48E8DDCFA6E49A1609F476C0B7E47B
:106650009B1609F476C0EBE39E1224C0D601119676
:106660009C91119713968C9138E0390F813031F05D
:10667000833011F0392F02C0392F985021E04B811F
:10668000491708F420E041E0391708F040E091E0B4
:106690005A81351708F490E0322F342B932379F484
:1066A000242369F481E0DF91CF911F910F91FF9036
:1066B000EF90DF90CF90BF90AF909F900895F6013C
:1066C000128100E0F12C843048F490E0FC01E95A9A
:1066D000FC4FF0808D5A9C4FDC010C9117FF03C0DA
:1066E000B601CE01EBDBF60180818F0D80838181C5
:1066F000800F8183110F91F7D5CFB601CE01DEDB7C
:10670000D1CFCE01F0DB882371F2EE81FF818D8144
:10671000A4E08A9FC00111248E0F9F1F11928E1733
:106720009F07E1F7BFCFF60110828A8181838D81B7
:10673000815082838B818383B5CF8D81D6018C93E9
:10674000B1CF8981F6018083ADCF0F93FC01015059
:10675000040F84A996A9941788F0081710F4041759
:1067600078F42150260F83A995A9961758F0281779
:1067700060F481E0261720F40F910895081778F748
:1067800080E0FACF2817A8F7FBCF81E0F5CFFF9282
:106790000F931F93CF93DF93C82FD62F142FF22E72
:1067A000022F242F462F682F8FEC9AE0CEDF88230C
:1067B00051F02F2D412F6D2F8C2FDF91CF911F91F5
:1067C0000F91FF90D6CCDF91CF911F910F91FF9049
:1067D00008953F924F925F926F927F928F929F9215
:1067E000AF92BF92CF92DF92EF92FF920F931F93DF
:1067F000CF93DF93D82FC62FB42EF22E4801022F4D
:10680000242F462F682F8FEC9AE09FDF882309F40E
:106810005FC00C2F0F0D88EF8B0DC82EC694C69449
:10682000C694D12C9FEFC91AD90A97E0E92EEB0C38
:10683000E694E694E694F12C27E0522E5D0E32E0C9
:10684000432E3B2C350C887FA82ED85F152D3401A4
:10685000F30184916091D10A7091D20A1093EB0AEE
:10686000C093EC0A4092EE0A8093ED0A2BEE3AE0D8
:106870004BE38FEC9AE054DBFFEF6F1A7F0A185F4F
:10688000832D811B883020F7F401EC0DFD1D8B2D2D
:106890008770782EC1F014916D2E6A0C10FF0EC017
:1068A0006091D10A7091D20A6092EB0AC093EC0A0F
:1068B0002BEE3AE042E38FEC9AE032DB63947A9479
:1068C00016957110EBCF8E0C9F1CCF5FC013BECFFF
:1068D000DF91CF911F910F91FF90EF90DF90CF90BC
:1068E000BF90AF909F908F907F906F905F904F90F0
:1068F0003F9008950F9304E026E24EE264E38FECAC
:106900009AE023DF882369F046E26EE284E3D5DB78
:1069100084E344DC89E542DC46E261E384E30F91F1
:10692000CCCB0F91089520911907260F3327331FE1
:1069300021323105ECF420915708FC0190E080E011
:10694000243069F082E00895A09119072191AC01EB
:106950004750594FA40FB52FB11D2C9301968617A0
:1069600098F380911907680F6093190780E00895E4
:1069700081E008951092570881E0809356081092A4
:10698000310861E084E10E946E2B61E085E10E94A4
:106990006E2BE9EBF0E080818E7F808380818D7F9C
:1069A000808388E48093B80085E48093BC000895D8
:1069B000CF93DF9391E09093F8068823B1F0C091D4
:1069C000B800D091BA008091BC008A7B8093BC0053
:1069D00060E084E10E946E2B60E085E10E946E2BF6
:1069E000C9DFD093BA00C093B800DF91CF9108956A
:1069F000CF92DF92EF92FF920F931F93CF93DF938B
:106A0000D091800881E0D13208F09BC0C0917F080E
:106A10000E94AC2C6B017C018091570881116CC0E5
:106A200082E08093570881E0809356088FEF80932F
:106A3000550810925408D0935308AFE5B8E0E3E34B
:106A4000F8E080E0D8138CC01092320880913208B0
:106A5000CC0FC82BC093320880913108813009F0E7
:106A600083C0109231080E94AC2C6B017C01809194
:106A700032088093BB008091590890915A08A091E8
:106A80005B08B0915C08892B8A2B8B2BA1F00E94AC
:106A9000AC2C0091590810915A0820915B08309154
:106AA0005C086C197D098E099F09061717072807CE
:106AB000390708F442C08091BC0083FDD8CF85EC33
:106AC0008093BC000E94AC2C6B017C018091570824
:106AD000823009F44BC0809155088F3F09F468C09B
:106AE00080915508803209F465C080915508803343
:106AF00009F462C084E025C08091590890915A0839
:106B0000A0915B08B0915C08892B8A2B8B2B09F430
:106B100083CF0E94AC2C0091590810915A08209103
:106B20005B0830915C086C197D098E099F09061776
:106B300017072807390708F06FCF8091580838DF0A
:106B400085E010925E081092800810925D08DF9137
:106B5000CF911F910F91FF90EF90DF90CF9008950C
:106B60009D9191938F5F6ECF85EEAACF809159084A
:106B700090915A08A0915B08B0915C08892B8A2BF0
:106B80008B2B09F4A3CF0E94AC2C009159081091D3
:106B90005A0820915B0830915C086C197D098E09B8
:106BA0009F09061717072807390708F08FCFC5CFA9
:106BB00080E0C7CF82E0C5CF83E0C3CF0895E091E6
:106BC000700780916F07E81730F4F0E0EB5BF84F47
:106BD000808190E008958FEF9FEF08959091700766
:106BE00080916F072FEF3FEF981748F4E92FF0E0FF
:106BF000EB5BF84F208130E09F5F90937007C901F5
:106C0000089580916F0790917007891B990B0895E3
:106C1000CF92DF92EF92FF920F931F93CF93DF9368
:106C20007C01CB018A0120915D08222389F0EB01D0
:106C30006B01C40ED51ECC15DD0561F06991D7013D
:106C4000ED91FC910190F081E02DC7011995F3CFF2
:106C5000642F69DEC801DF91CF911F910F91FF90E2
:106C6000EF90DF90CF900895CF93DF931F92CDB731
:106C7000DEB7698320915D082223F9F02091800816
:106C8000203258F021E030E0FC013383228390E091
:106C900080E00F90DF91CF91089580915E08E82FFA
:106CA000F0E0E15AF74F998190838F5F80935E08FF
:106CB0008093800881E090E0ECCF61E0CE01019606
:106CC00032DEF8CF1F93CF93DF93EC0181E0809306
:106CD0005D0888E680937F0810925E081092800815
:106CE00060E089E499E0C0DF2D811AE0822F612FF6
:106CF0000E944F8F682F660F680F660F620F89E43E
:106D000099E0B2DF2C81822F612F0E944F8F682F74
:106D1000660F680F660F620F89E499E0A5DF2B818B
:106D2000822F612F0E944F8F682F660F680F660FAA
:106D3000620F89E499E098DF60E089E499E094DFEC
:106D40002A81822F612F0E944F8F682F660F680F54
:106D5000660F620F89E499E087DF2981822F612F16
:106D60000E944F8F682F660F680F660F620F89E4CD
:106D700099E07ADF2881822F612F0E944F8F682F40
:106D8000660F680F660F620F89E499E06DDF60E0BF
:106D900089E499E069DFDF91CF911F9129CEAF920D
:106DA000BF92CF92DF92EF92FF920F931F93CF93F8
:106DB000DF93DC0128E030E080E041E067E070E054
:106DC00093E2A92EB12C0FEC10E09C911196ED915D
:106DD000FC911297F8945181592B5183F280E92E3E
:106DE000E094FE20F282EB012197F1F751815E21C0
:106DF0005183E5012197F1F750817894F80131979B
:106E0000F1F7952309F0842B440F21503109E9F65D
:106E1000DF91CF911F910F91FF90EF90DF90CF9076
:106E2000BF90AF900895FC0190810180F281E02D28
:106E3000F8948181292F20958223818378943DE7DE
:106E400043E050E0315029F1DA011197F1F78081E8
:106E50008923C1F3F8948281822382838181892BE3
:106E600081837894ABE7B7E01197F1F7F8948181CB
:106E700082238183A3E1B1E01197F1F78081982308
:106E800081E009F080E07894E3E6F6E03197F1F7ED
:106E9000089580E008951F93CF93DF93EC01162FA0
:106EA00060E0812F0E949B2B612F70E0FB01E55079
:106EB000F64EE491E883FB01EF5BF54EE491F0E0E0
:106EC000EE0FFF1FEF57F64E859194919A838983B9
:106ED0001B861D861C861A86198618861F821E82AE
:106EE0001D821C821B82DF91CF911F9108950F9309
:106EF0001F93CF93DF932091EE062F5F322F3770D1
:106F00003093EE0620FF2BC020E831FD2064347062
:106F100009F02062205FFC01EC01239600E011E003
:106F20006485662329F070E0C8010E946F8F6F5F4F
:106F30006187322F369F030E30E0311D112431114D
:106F400010C01682662311F0615061873196EC17EC
:106F5000FD0731F7DF91CF911F910F91089520E048
:106F6000D4CF31503683EECF6F927F928F929F9223
:106F7000AF92BF92CF92DF92EF92FF920F931F9347
:106F8000CF93DF933C01EB010E94AC2CF3012785EA
:106F90003089621B730B6A307105B0F3F894E88195
:106FA000F981509105015260409105014D7F409358
:106FB0000501EA848F812E2D281B822F2F83DF84E9
:106FC000AA81BB816D857C85FE846F5F7F5FF394B2
:106FD0009E813885B984AB84118120E0C32E022FB5
:106FE000322F3181112788943111380F08F43FEF87
:106FF0008195889460FD130F1795889461FD130F98
:107000001795889462FD130F1795889463FD130FED
:107010001795889464FD130F1795889465FD130FD9
:107020001795889466FD130F1795889467FD130FC5
:1070300017958894232F6111212F8E0D122F002C6C
:1070400050930501002C17FF409305013081222742
:10705000889400C000C0409305013111390F00C071
:1070600050930501002C16FF4093050108F43FEFF3
:107070009195889400C000C04093050170FD230FD6
:1070800000C050930501002C15FF40930501279582
:10709000889471FD230F00C000C04093050127951F
:1070A000889400C050930501002C14FF4093050103
:1070B00072FD230F2795889400C000C040930501FE
:1070C00073FD230F00C050930501002C13FF409364
:1070D00005012795889474FD230F00C000C04093DC
:1070E00005012795889400C050930501002C12FFDC
:1070F0004093050175FD230F2795889400C000C0BB
:107100004093050176FD230F00C050930501002C2C
:1071100011FF409305012795889477FD230F00C048
:1071200000C0409305012795889400C05093050145
:10713000002C10FF40930501132F7111122F9B0D8E
:1071400000C000C04093050100C000C0509305017D
:10715000002C17FF4093050132812227889400C03C
:1071600000C04093050131113C0D00C05093050152
:10717000002C16FF4093050108F43FEFED0DF11DC3
:1071800000C000C040930501F0FC230F00C05093E5
:107190000501002C15FF4093050127958894F1FC0B
:1071A000230F00C000C0409305012795889400C0BC
:1071B00050930501002C14FF40930501F2FC230FAE
:1071C0002795889400C000C040930501F3FC230F6D
:1071D00000C050930501002C13FF40930501279533
:1071E0008894F4FC230F00C000C04093050127954C
:1071F000889400C050930501002C12FF40930501B4
:10720000F5FC230F2795889400C000C0409305012A
:10721000F6FC230F00C050930501002C11FF409392
:10722000050127958894F7FC230F00C000C0409308
:1072300005012795889400C050930501002C10FF8C
:1072400040930501132FF110122FC19400C000C00C
:1072500040930501CA0C00C0002C50930501002C7E
:1072600017FF4093050131812227889400C000C098
:10727000409305013111380F00C050930501002CD7
:1072800016FF4093050108F43FEF8195889400C0F4
:1072900000C04093050160FD230F00C0509305011D
:1072A000002C15FF409305012795889461FD230F5D
:1072B00000C000C0409305012795889400C05093FA
:1072C0000501002C14FF4093050162FD230F279553
:1072D000889400C000C04093050163FD230F00C0E7
:1072E00050930501002C13FF4093050127958894C6
:1072F00064FD230F00C000C04093050127958894CA
:1073000000C050930501002C12FF4093050165FD5C
:10731000230F2795889400C000C04093050166FDA7
:10732000230F00C050930501002C11FF409305016D
:107330002795889467FD230F00C000C04093050186
:107340002795889400C050930501002C10FF4093AE
:107350000501132F6111122F8E0D00C000C0409344
:107360000501119709F06CCE4A815B8120EE31E076
:10737000DA010E94AC8FDC01CB01F4E0B695A79551
:1073800097958795FA95D1F730E020E0B901EAE9C1
:107390004E9F040E611D5E9F600D711D1124650FCF
:1073A000711D860F971FA11DB11D893E43E09407F3
:1073B000A105B10508F434C0885E9340A109B10964
:1073C00042E0B695A795979587954A95D1F747E0FE
:1073D000849F080E211D949F200D311D1124290F1B
:1073E000311D6091ED0670E0860F971F820F931F8D
:1073F00040918F0850919008609191087091920887
:10740000292F3327420F531F611D711D40938F0891
:107410005093900860939108709392088093ED06C2
:1074200078940E94AC2CF301708B6787DF91CF9129
:107430001F910F91FF90EF90DF90CF90BF90AF9092
:107440009F908F907F906F900895E4E0F1E08081AD
:107450008260808308950F931F93CF93DF93CDB7FE
:10746000DEB762970FB6F894DEBF0FBECDBF8C01BA
:10747000F901DC011C968C917A8369835C834B83D0
:107480005E834D8390819D8791819E8792819F87A6
:107490008130E9F4CE0101962ADD83E0888B1A8AD7
:1074A000198AD801ED91FC910484F585E02DBE0187
:1074B0006F5F7F4FC801199562960FB6F894DEBFD3
:1074C0000FBECDBFDF91CF911F910F9108951C8604
:1074D0001B861A86198618861F82DFCF0F931F938B
:1074E000CF93DF93CDB7DEB762970FB6F894DEBFC8
:1074F0000FBECDBF8C01F901DC011C968C917A8303
:1075000069835C834B835E834D8390819D879181EA
:107510009E8792819F878130E1F4CE010196E7DC5E
:10752000188A1A8A198AD801ED91FC910484F5858C
:10753000E02DBE016F5F7F4FC801199562960FB6AF
:10754000F894DEBF0FBECDBFDF91CF911F910F9199
:1075500008951C861B861A86198618861F82E0CF1E
:10756000EF92FF920F931F93CF93DF9360E08DE034
:107570000E946E2B10922C0810922B086CE271E086
:1075800080E090E00E94F52DD0E0C1E0FF24F3946C
:1075900082E0E82E64E670E080E090E00E94F52D45
:1075A00080912B0890912C080196823091050CF067
:1075B00071C090932C0880932B080E94F52FF092B5
:1075C000EF0A04E415E120E440E860E080E001D93E
:1075D000F092EF0AC13009F067C0D11102C01092D9
:1075E000EF0A27E047E065E283E1D1D827E049E0F0
:1075F00065E288E2CCD80E9425308111E0CF0E945C
:107600002423892B39F2E09256091092220A61E074
:107610008DE00E946E2B8091850890918608A09144
:107620008708B0918808853D2BE4920720E9A207DE
:107630002EE0B207A9F185352BEC920720E9A207CD
:107640002EE0B20779F111E084309A41A041BE40AA
:1076500009F010E06CE271E080E090E00E94F52D0E
:10766000E09256091092220A60E08DE00E946E2B93
:10767000112309F48FCF68EC70E080E090E00E9465
:10768000F52D8C2F90E0DF91CF911F910F91FF90FE
:10769000EF900895DF2510922C0810922B088DCFC3
:1076A000C2E0D1CFC1E0D5CFD11102C01092EF0A14
:1076B00027E047E065E282E46AD827E047E065E238
:1076C00089E598CF682F8CE20C946E2B1F93CF9393
:1076D000DF932091F2063091F3061FEF129FC00155
:1076E000139F900D1124C4E6D0E0BE010E946F8F5D
:1076F00088E00E94D72B2091F0063091F106129F6E
:10770000C001139F900D1124BE010E946F8F8CE069
:10771000DF91CF911F910C94D72B8091F70688238E
:1077200009F445C061E082E00E946E2B8091E8067A
:10773000811110C086E090E09093100880930F08AC
:1077400081E090E090931603809315038093E80600
:1077500010920A028091F60661E0811101C060E09A
:1077600083E00E946E2B8091F50661E0811101C0DB
:1077700060E084E00E946E2B8091F40661E081114C
:1077800006C085E00E94462B892B21F060E085E051
:107790000E946E2B8091930761E0811105C080915A
:1077A000920781111DC060E086E00C946E2B60E0B2
:1077B00082E00E946E2B80910A028111CBCF87E07C
:1077C00090E09093100880930F0881E090E09093F0
:1077D0001603809315031092E80680930A02BACF2D
:1077E00008958091F807811189C180910B032FEFD3
:1077F000829FC001112464E670E00E946F8F87E0D1
:107800000E94D72B80911908813009F05BC08091CC
:10781000E506882309F4B4C0E091E306F091E4069C
:107820003196F093E406E093E3064091E10650912F
:10783000E20620917307309174074115510521F438
:107840003093F3062093F2066CE3649FC001659FBA
:10785000900D1124B9010E946F8F4CED469FC0011D
:10786000479F900D11246FEF70E00E946F8F6E178D
:107870007F070CF085C08091F2069091F306019687
:107880009093F3068093F2061092E4061092E306BA
:107890002817390734F43093F3062093F206109238
:1078A00019082091F2063091F3064FEF429FC00174
:1078B000439F900D112464E670E00E946F8F88E072
:1078C0000E94D72B80911908823009F059C080910D
:1078D000E506811155C02091E3063091E4062F5F43
:1078E0003F4F3093E4062093E3064091E106509128
:1078F000E2064115510521F41092F3061092F206AA
:107900006CE3649FC001659F900D11246091730723
:10791000709174070E946F8F4CED469FC001479F86
:10792000900D11246FEF70E00E946F8F6217730744
:107930003CF58091F2069091F30601979093F3063F
:107940008093F2061092E4061092E30618161906C8
:1079500034F01092F3061092F2061092190820915A
:10796000F2063091F3064FEF429FC001439F900D06
:10797000112464E670E00E946F8F88E00E94D72B8C
:1079800080911808813009F05BC08091E00688235F
:1079900009F4B7C0E091DE06F091DF063196F0936E
:1079A000DF06E093DE064091DC065091DD06209173
:1079B0007107309172074115510521F43093F1069A
:1079C0002093F0066CE3649FC001659F900D112425
:1079D000B9010E946F8F4CED469FC001479F900DEB
:1079E00011246FEF70E00E946F8F6E177F070CF00D
:1079F00088C08091F0069091F10601969093F1066F
:107A00008093F0061092DF061092DE0628173907E1
:107A100034F43093F1062093F00610921808209168
:107A2000F0063091F1064FEF429FC001439F900D49
:107A3000112464E670E00E946F8F8CE00E94D72BC7
:107A400080911808823009F05CC08091E0068111B5
:107A500058C02091DE063091DF062F5F3F4F3093F4
:107A6000DF062093DE064091DC065091DD064115CD
:107A7000510521F41092F1061092F0066CE3649F18
:107A8000C001659F900D112460917107709172077C
:107A90000E946F8F4CED469FC001479F900D1124AF
:107AA0006FEF70E00E946F8F6217730754F580913B
:107AB000F0069091F10601979093F1068093F006FD
:107AC0001092DF061092DE061816190634F0109296
:107AD000F1061092F006109218082091F0063091ED
:107AE000F1064FEF429FC001439F900D112464E6C1
:107AF00070E00E946F8F8CE00C94D72B80910A036A
:107B000076CE089590E080E00895FC018585968505
:107B10000895CF93DF9300D000D0CDB7DEB7AB018F
:107B20001C821D821E82DC01ED91FC910190F0818E
:107B3000E02D19821A821B829E012F5F3F4FBE01EA
:107B40006C5F7F4F199526960FB6F894DEBF0FBE77
:107B5000CDBFDF91CF9108953F924F925F926F9288
:107B60007F928F929F92AF92BF92CF92DF92EF92CD
:107B7000FF920F931F93CF93DF93EC01162FDCAC92
:107B80005BAC5C0124E0A20EB11CE98DFA8DC5014D
:107B90001995982EE884F984C7010E94E730082FD0
:107BA000888599850E94EA30782E88248A9401304D
:107BB00011F48FE0882E888599850E94E330082F84
:107BC000888599850E94DF30C82E888599850E9416
:107BD000FF30113670F0009761F0E80EF91E01E6F3
:107BE000C116B8F41C8A1F8A188E1D8A1E8A80E06E
:107BF0005BC0888599850E940131113430F000976F
:107C000021F0E80EF91E01E4EBCF81E1E80EF11C52
:107C1000E7CFC01638F3872D90E0F70124912F3F6E
:107C200039F4FFEFEF1AFF0AC016E1F20F5FF5CF4C
:107C3000101368C0888599850E94E73097012F5FEF
:107C40003F4FF701882319F0823009F044C0849136
:107C50008F8BF9012491288FF7013396E491EC8BF7
:107C6000F7013496E491ED8BF7013596E491EE8BB4
:107C7000E114F10409F4BBCF888599850E94EA30AC
:107C8000782ECF88388C8D89580E1D2D13198E892A
:107C9000181B190D032D2C2D412F652DC5010E9498
:107CA000A533811138C08C899BAD890F8BAF81E0E2
:107CB00090E0DF91CF911F910F91FF90EF90DF90B7
:107CC000CF90BF90AF909F908F907F906F905F907C
:107CD0004F903F9008958491982F9F7092509E8B63
:107CE00082958F708D8BF9012491822F8F70888FF0
:107CF00022952F702F8BF7013296E491E295EF7069
:107D0000EC8BB6CF3296E491E821E80FF92FF11D04
:107D1000EE0EFF1E89CFE70CF11C07E00C0D069557
:107D200006950695310E4E01F0E28F0E911C602EE5
:107D3000712C131509F4B7CF452C670112C0F60159
:107D400084916E817F8148A219A31BA28AA394010A
:107D50004BE3C5010E94902FFFEFCF1ADF0A28E006
:107D6000420E8C2D8E19801750F3E60CF71C1F5F06
:107D7000E0CF682F8BEC9AE0EFCE8EBD00000DB403
:107D800007FEFDCF8EB50895F8CFCF93DF93C82FB0
:107D9000D62F90E080E096DC80E28C0FC03238F085
:107DA0008FE18C0F833070F0CF3F61F08C2FE5DFD7
:107DB000C82F8D2FE9DF81E090E084DC8C2FDF91EC
:107DC000CF9108958C2FD9DFC82FF5CFCF93C82F2F
:107DD00090E080E077DC8C2FD7DF80E0CEDFC82F0B
:107DE00081E090E06FDC8C2FCF910895089590E0B2
:107DF00080E008958F929F92AF92BF92DF92EF92B0
:107E0000FF920F931F93CF93DF937C0181E08093C8
:107E10005D0888E680937F0810925E0810928008C3
:107E200060E089E499E00E9434360E94F8340E94B0
:107E3000AC2C4B015C0180915708811165C081E039
:107E400080935708809356089FEF9093550810929F
:107E5000540896E09093530880933208809132083A
:107E6000806D8093320880913108813009F0FFC025
:107E7000109231080E94AC2C4B015C0180913208B9
:107E80008093BB008091590890915A08A0915B089B
:107E9000B0915C08892B8A2B8B2BA1F00E94AC2C13
:107EA0000091590810915A0820915B0830915C08A4
:107EB000681979098A099B090617170728073907DE
:107EC00008F443C08091BC0083FDD8CF85EC80933B
:107ED000BC000E94AC2C4B015C01809157088130A2
:107EE00009F4C7C080915408873008F0E4C080913D
:107EF0005408A3E3B8E0E5E4F7E090E0981751F107
:107F00002D9121939F5FFACF8091590890915A0843
:107F1000A0915B08B0915C08892B8A2B8B2B09F40C
:107F20008ACF0E94AC2C0091590810915A082091D8
:107F30005B0830915C08681979098A099B09061762
:107F400017072807390708F076CF809158080E9454
:107F5000D83480E01092700780936F0789E499E02D
:107F60000E94EE358F77282F30E094E035952795E5
:107F70009A95E1F7922F990F990FC22FC91BCC0F39
:107F8000C80F89E499E00E94EE359C0144E03595E4
:107F900027954A95E1F72F703327922F990F990F64
:107FA000D22FD91BDD0FD80F89E499E00E94EE355E
:107FB0009C0154E0359527955A95E1F72F703327AA
:107FC000922F990F990F122F191B110F180F89E477
:107FD00099E00E94EE3589E499E00E94EE359C011B
:107FE00064E0359527956A95E1F72F703327922F36
:107FF000990F990F022F091B000F080F89E499E0D0
:108000000E94EE359C0174E0359527957A95E1F74D
:108010002F703327922F990F990FD22ED91ADD0C7A
:10802000D80E89E499E00E94EE359C01E4E0359594
:108030002795EA95E1F72F703327922F990F990F23
:10804000291B220F820FF7018083D18202831383C1
:10805000D483C583C701DF91CF911F910F91FF900A
:10806000EF90DF90BF90AF909F908F90089585EE36
:108070002ECF8091590890915A08A0915B08B09139
:108080005C08892B8A2B8B2B09F427CF0E94AC2C00
:108090000091590810915A0820915B0830915C08B2
:1080A000681979098A099B090617170728073907EC
:1080B00008F013CF4ACF87E01CCFBF92CF92DF9258
:1080C000EF92FF920F931F93CF93DF9300D000D0D6
:1080D000CDB7DEB7CE0101968DDEFC808F2D90E00E
:1080E0009093300880932F080D8110E010932E0894
:1080F00000932D088E8190E090932C0880932B089C
:108100008A8190E090932A08809329088B8190E0DF
:108110009093280880932708898190E08053984F96
:108120009093260880932508CE0101960E94F72E91
:1081300090E0009709F4FBC09093240880932308F3
:1081400024E6F29E000D111D11241093E706009302
:10815000E60680919207811102C0109293078091E8
:10816000EF06882319F081E080939307409123085C
:1081700050912408415F5F4F60919307E5E7F2E07B
:1081800070E0E12CD12CF12C84E69F01240F351FE7
:10819000D9019C91913009F069C09081913001F52D
:1081A0009481258130E0989F200D311D1124021704
:1081B0001307B4F09681278130E0989F200D311D80
:1081C00011240217130764F49381933009F4BCC09F
:1081D00008F0B0C0913009F4BCC0923009F4B1C0CD
:1081E0009181913001F59085218530E0989F200D97
:1081F000311D112402171307B4F09285238530E056
:10820000989F200D311D11240217130764F49381E8
:10821000933009F4ABC008F09FC0913009F4ABC0B3
:10822000923009F4A0C09281913001F594852585A2
:1082300030E0989F200D311D112402171307B4F070
:108240009685278530E0989F200D311D1124021757
:10825000130764F49381933009F49AC008F08EC038
:10826000913009F49AC0923009F48FC07796B2E049
:10827000EF3FFB0709F089CFF092F706D092F606A0
:10828000E092F5067093F4066093930746DA109235
:10829000F807B090050321E0B212A6C09091060342
:1082A00084E6E0900703F12C989FE00CF11C112468
:1082B00090910803C0900903D12C989FC00CD11C49
:1082C0001124CE14DF040CF072C00E151F059CF0B3
:1082D000083389E018077CF480910A03AFEF8A9F86
:1082E000C001112464E670E00E946F8F87E00E9455
:1082F000D72BB092F8070C151D050CF071C08091BA
:108300000A03BFEF8B9FC001112464E670E00E9456
:108310006F8F87E00E94D72B81E08093F807EC14E1
:10832000FD04F4F50E151F050CF04AC059C087E096
:1083300090E002CF943059F0953009F051CF61E0D0
:108340004FCFDD24D3944CCFEE24E39449CF71E09A
:1083500047CFFF24F39444CF943059F0953009F07F
:1083600062CF61E060CFDD24D3945DCFEE24E3944F
:108370005ACF71E058CFFF24F39455CF943059F081
:10838000953009F073CF61E071CFDD24D3946ECFC7
:10839000EE24E3946BCF71E069CFFF24F39466CFB2
:1083A00080910A03BFEF8B9FC001112423C0EC14FE
:1083B000FD04D4F40E151F059CF00C151D0584F466
:1083C00080910A032FEF829FC001112464E670E0C0
:1083D0000E946F8F87E00E94D72B81E08093F8077F
:1083E0008091F8078111DCCF80910B03AFEF8A9F5A
:1083F000C001112464E670E00E946F8F87E00E9444
:10840000D72B26960FB6F894DEBF0FBECDBFDF91F7
:10841000CF911F910F91FF90EF90DF90CF90BF9081
:108420000895DF92EF92FF920F931F93CF93DF9304
:1084300082E0809356091092220A61E08DE00E944A
:108440006E2B8091850890918608A0918708B09145
:1084500088088E349045A041BE4089F410921008DF
:1084600010920F08CCE9D7E01FEF188319831A8305
:108470000E94D12C239687E0C63FD807B1F78091A0
:10848000850890918608A0918708B09188084E973A
:10849000A041BE4081F41092100810920F08CCE960
:1084A000D7E0188219821A820E94D12C239687E085
:1084B000C63FD807B1F78091850890918608A091B2
:1084C0008708B09188088E3F904EA041BE4009F0C9
:1084D0005AC080910F0890911008892B81F4CCE943
:1084E000D7E0A2E8FA2E06E41AEFF88209831A838D
:1084F0000E94D12C239687E0C63FD807B1F7809120
:108500000F0890911008019781F4CCE9D7E0F2E8C8
:10851000FF2E06E41AEFF88209831A830E94D12CF9
:10852000269627E0C63FD207B1F780910F089091B9
:108530001008029781F4CCE9D7E0E2E8FE2E06E4C9
:108540001AEFF88209831A830E94D12C2C9687E0B7
:10855000CC3FD807B1F780910F089091100806978B
:1085600031F481E090E09093100880930F0880919F
:108570000F0890911008079731F481E090E09093F4
:10858000100880930F088091850890918608A0912B
:108590008708B09188088E3E904FA041BE4009F0F8
:1085A0005AC080910F0890911008892B81F4CCE972
:1085B000D7E074EBF72E0EE61EEBF88209831A83E0
:1085C0000E94D12C239687E0C63FD807B1F780914F
:1085D0000F0890911008019781F4CCE9D7E064EB83
:1085E000F62E0EE61EEBF88209831A830E94D12C28
:1085F000269627E0C63FD207B1F780910F089091E9
:108600001008029781F4CCE9D7E054EBF52E0EE682
:108610001EEBF88209831A830E94D12C2C9687E0E6
:10862000CC3FD807B1F780910F08909110080697BA
:1086300031F481E090E09093100880930F088091CE
:108640000F0890911008079731F481E090E0909323
:10865000100880930F088091850890918608A0915A
:108660008708B0918808843F2AEE920720E1A2078C
:108670002EE0B207A9F422E030E0309317082093EF
:108680001608883726E6920720E1A2072EE0B207F7
:10869000F1F485E090E0909317088093160852C09B
:1086A000883F26EE920720E1A2072EE0B20721F4D0
:1086B00021E020931508E5CF8F3921E0920720E9CA
:1086C000A2072EE0B20751F521E02093130885316F
:1086D0009B48A049BE40B1F58091F9079091FA07F7
:1086E0008130910509F069C02091F70631E0232718
:1086F0002093F7068630910509F072C080911B0225
:1087000090911C02019797FD02C00C948B4C109223
:108710001C0210921B020E94663B14C08E3520E49E
:10872000920720E1A2072EE0B207D9F587E090E09A
:108730009093100880930F0881E090E090931603C7
:10874000809315038091850890918608A0918708F1
:10875000B091880885399B40A049BE4009F0C0C04F
:108760008091F9079091FA078130910509F075C061
:108770002091F70631E023272093F70686309105F4
:1087800009F07EC080911B0290911C0201968536F3
:10879000910514F084E690E090931C0280931B02F4
:1087A0009DC08E3D20EC920720E1A2072EE0B2078B
:1087B00009F067CF86E090E0BBCF8230910539F4B5
:1087C0002091F60631E023272093F60693CF8330DD
:1087D0009105B9F42091F50631E023272093F506A1
:1087E00087309105B9F48091F2069091F3060197D4
:1087F00097FD02C00C94974C1092F3061092F2066B
:108800008ACF84309105B9F42091F40631E0232712
:108810002093F4068830910511F00C94914C8091CE
:10882000F0069091F106019797FD12C09093F10622
:108830008093F00670CF8530910509F05BCF809171
:10884000930791E08927809393070E948D3B7ACF0D
:108850001092F1061092F0065ECF8230910539F445
:108860002091F60631E023272093F60687CF833048
:108870009105C1F42091F50631E023272093F506F8
:1088800087309105C9F48091F2069091F306019624
:108890008536910514F084E690E09093F30680937A
:1088A000F2061CC08430910509F058C02091F406EE
:1088B00031E023272093F4068830910511F00C94C1
:1088C0009D4C8091F0069091F106019685369105B8
:1088D0000CF051C09093F1068093F0060E94663B25
:1088E0008091850890918608A0918708B0918808AA
:1088F0008E389049A041BE4091F410929307109297
:10890000EF0660E086E00E946E2B70E060E08CE095
:108910000E94D72B70E060E088E00E94D72B809106
:10892000850890918608A0918708B09188088535C0
:108930002BEC920720E9A2072EE0B207F9F4809110
:10894000F9079091FA0701971816190614F088E0B4
:1089500090E09093FA078093F90742C08530910523
:1089600009F00CCF8091930791E0892780939307BA
:108970000E948D3BB5CF84E690E0ACCF853D2BE4E3
:10898000920720E9A2072EE0B20709F06DC7809197
:10899000F9079091FA07019689309105D4F281E0A8
:1089A00090E09093FA078093F90780918508909161
:1089B0008608A0918708B091880888359644A04120
:1089C000BE4071F481E0809393078093EF0661E0ED
:1089D00086E00E946E2B64E670E08CE00E94D72B4C
:1089E0008091850890918608A0918708B0918808A9
:1089F000883D964CA041BE4071F481E0809393077E
:108A00008093EF0661E086E00E946E2B6AEF70E0D3
:108A100088E00E94D72B8091850890918608A091CC
:108A20008708B09188088D3422EB92072FEFA207B8
:108A3000B10509F030C781E090E090931008809371
:108A40000F089093160380931503809185089091E9
:108A50008608A0918708B09188088F34904BAF4F5B
:108A6000B10589F41092100810920F08CCE9D7E0F4
:108A70001FEF188319831A830E94D12C239687E055
:108A8000C63FD807B1F78091850890918608A091DC
:108A90008708B09188088F369049AF4FB10529F506
:108AA000809111039091120324E130E08436910506
:108AB00064F42AE030E0823391053CF421E030E0B8
:108AC0008A30910514F025E030E0820F931F813F3A
:108AD00091050CF01AC790931203809311038091B3
:108AE000110380933C090E94D12C809185089091BC
:108AF0008608A0918708B09188088734984BAF4FBB
:108B0000B10529F5809111039091120324E130E021
:108B10008436910564F42AE030E0823391053CF418
:108B200021E030E08A30910514F025E030E0821B2E
:108B3000930B181619060CF0EBC690931203809352
:108B400011038091110380933C090E94D12C8091E4
:108B5000850890918608A0918708B091880887368B
:108B60009849AF4FB10509F051C080910F0890911D
:108B70001008892B69F4CCE9D7E01FEF188319821C
:108B80001A820E94D12C239687E0C63FD807B1F7FE
:108B900080910F0890911008019769F4CCE9D7E013
:108BA0001FEF188319821A820E94D12C269627E083
:108BB000C63FD207B1F780910F0890911008029735
:108BC00069F4CCE9D7E01FEF188319821A820E945A
:108BD000D12C2C9687E0CC3FD807B1F780910F08B5
:108BE00090911008069731F481E090E0909310087E
:108BF00080930F0880910F0890911008079731F427
:108C000081E090E09093100880930F088091850890
:108C100090918608A0918708B09188088732984D76
:108C2000AF4FB10509F051C080910F089091100825
:108C3000892B69F4CCE9D7E010E8188219831A82ED
:108C40000E94D12C239687E0C63FD807B1F78091C8
:108C50000F0890911008019769F4CCE9D7E010E86B
:108C6000188219831A820E94D12C269627E0C63FCB
:108C7000D207B1F780910F0890911008029769F41C
:108C8000CCE9D7E010E8188219831A820E94D12C0F
:108C90002C9687E0CC3FD807B1F780910F089091D0
:108CA0001008069731F481E090E0909310088093CB
:108CB0000F0880910F0890911008079731F481E018
:108CC00090E09093100880930F0880918508909110
:108CD0008608A0918708B091880887379848AF4FD9
:108CE000B10509F051C080910F0890911008892BAF
:108CF00069F4CCE9D7E01FEF188219821A830E9429
:108D0000D12C239687E0C63FD807B1F780910F0892
:108D100090911008019769F4CCE9D7E01FEF188211
:108D200019821A830E94D12C269627E0C63FD207CB
:108D3000B1F780910F0890911008029769F4CCE97F
:108D4000D7E01FEF188219821A830E94D12C2C962B
:108D500087E0CC3FD807B1F780910F0890911008B9
:108D6000069731F481E090E09093100880930F080B
:108D700080910F0890911008079731F481E090E0FE
:108D80009093100880930F08809185089091860831
:108D9000A0918708B09188088735984AAF4FB105F0
:108DA00009F051C080910F0890911008069731F496
:108DB00081E090E09093100880930F0880910F0855
:108DC00090911008079731F481E090E0909310089B
:108DD00080930F0880910F0890911008892B69F4F7
:108DE000CCE9D7E01FEF188319831A830E94D12C96
:108DF000239687E0C63FD807B1F780910F0890917E
:108E00001008019769F4CCE9D7E01FEF18831983A4
:108E10001A830E94D12C269627E0C63FD207B1F7CD
:108E200080910F0890911008029769F4CCE9D7E07F
:108E30001FEF188319831A830E94D12C2C9687E088
:108E4000CC3FD807B1F78091850890918608A09112
:108E50008708B09188088731984EAF4FB10509F067
:108E600054C080910F0890911008892B71F4CCE9BF
:108E7000D7E00FEF12E3088319831A820E94D12CE6
:108E8000239687E0C63FD807B1F780910F089091ED
:108E90001008019771F4CCE9D7E00FEF12E30883D3
:108EA00019831A820E94D12C269627E0C63FD2074A
:108EB000B1F780910F0890911008029771F4CCE9F6
:108EC000D7E00FEF12E3088319831A820E94D12C96
:108ED0002C9687E0CC3FD807B1F780910F0890918E
:108EE0001008069731F481E090E090931008809389
:108EF0000F0880910F0890911008079731F481E0D6
:108F000090E09093100880930F08809185089091CD
:108F10008608A0918708B0918808873B9844AF4F96
:108F2000B10509F051C080910F0890911008892B6C
:108F300069F4CCE9D7E01FEF188219831A830E94E5
:108F4000D12C239687E0C63FD807B1F780910F0850
:108F500090911008019769F4CCE9D7E01FEF1882CF
:108F600019831A830E94D12C269627E0C63FD20788
:108F7000B1F780910F0890911008029769F4CCE93D
:108F8000D7E01FEF188219831A830E94D12C2C96E8
:108F900087E0CC3FD807B1F780910F089091100877
:108FA000069731F481E090E09093100880930F08C9
:108FB00080910F0890911008079731F481E090E0BC
:108FC0009093100880930F088091850890918608EF
:108FD000A0918708B091880887399846AF4FB105AE
:108FE00009F060C080910F0890911008892B81F4DE
:108FF000CCE9D7E044E6F42E0EE11CEDF8820983BB
:109000001A830E94D12C239687E0C63FD807B1F778
:1090100080910F0890911008019799F4CCE9D7E05E
:1090200006EF17E094E6D92E2EE1E22E3CEDF32E6A
:10903000D882E982FA820E94D12C26960C171D074D
:10904000B9F780910F0890911008029799F4CCE934
:10905000D7E00CEF17E0A4E6DA2EBEE1EB2E8CEDA4
:10906000F82ED882E982FA820E94D12C2C960C1715
:109070001D07B9F780910F0890911008069731F4F9
:1090800081E090E09093100880930F0880910F0882
:1090900090911008079731F481E090E090931008C8
:1090A00080930F088091850890918608A091870889
:1090B000B09188088D3F9240AF4FB10509F063C071
:1090C00080910F0890911008892B99F4CCE9D7E092
:1090D00006EF17E0DD24DA94E0E5EE2EF4E1FF2E52
:1090E000D882E982FA820E94D12C23960C171D07A0
:1090F000B9F780910F0890911008019799F4CCE985
:10910000D7E006EF17E0DD24DA9460E5E62E74E19F
:10911000F72ED882E982FA820E94D12C26960C176B
:109120001D07B9F780910F0890911008029799F4E4
:10913000CCE9D7E00CEF17E0DD24DA9440E5E42E2B
:1091400054E1F52ED882E982FA820E94D12C2C9625
:109150000C171D07B9F780910F089091100806971A
:1091600031F481E090E09093100880930F08809193
:109170000F0890911008079731F481E090E09093E8
:10918000100880930F088091850890918608A0911F
:109190008708B09188088D3C9243AF4FB10509F024
:1091A00063C080910F0890911008892B99F4CCE945
:1091B000D7E006EF17E09BE3D92E23E8E22E3DEB44
:1091C000F32ED882E982FA820E94D12C23960C17C2
:1091D0001D07B9F780910F0890911008019799F435
:1091E000CCE9D7E006EF17E0ABE3DA2EB3E8EB2EDD
:1091F0008DEBF82ED882E982FA820E94D12C269635
:109200000C171D07B9F780910F089091100802976D
:1092100099F4CCE9D7E00CEF17E07BE3D72EE3E835
:10922000EE2EFDEBFF2ED882E982FA820E94D12C2D
:109230002C960C171D07B9F780910F089091100814
:10924000069731F481E090E09093100880930F0826
:1092500080910F0890911008079731F481E090E019
:109260009093100880930F0880918508909186084C
:10927000A0918708B09188088F3D9042AF4FB1050B
:1092800009F05DC080910F0890911008892B89F436
:10929000CCE9D7E006EF17E06BE8E62EFF24FA945E
:1092A000E8821982FA820E94D12C23960C171D079E
:1092B000B9F780910F0890911008019789F4CCE9D3
:1092C000D7E006EF17E05BE8E52EFF24FA94E8828A
:1092D0001982FA820E94D12C26960C171D07B9F725
:1092E00080910F0890911008029789F4CCE9D7E09B
:1092F0000CEF17E04BE8E42EFF24FA94E882198281
:10930000FA820E94D12C2C960C171D07B9F7809178
:109310000F0890911008069731F481E090E0909347
:10932000100880930F0880910F08909110080797FC
:1093300031F481E090E09093100880930F088091C1
:10934000850890918608A0918708B09188088F3A87
:109350009045AF4FB10509F060C080910F08909122
:109360001008892B81F4CCE9D7E03AEFF32E04E61C
:109370001AE0F88209831A830E94D12C239687E091
:10938000C63FD807B1F780910F0890911008019758
:1093900099F4CCE9D7E006EF17E08AEFD82E94E6EF
:1093A000E92E2AE0F22ED882E982FA820E94D12C9C
:1093B00026960C171D07B9F780910F089091100899
:1093C000029799F4CCE9D7E00CEF17E0FAEFDF2E23
:1093D000A4E6EA2EBAE0FB2ED882E982FA820E9445
:1093E000D12C2C960C171D07B9F780910F0890917E
:1093F0001008069731F481E090E090931008809374
:109400000F0880910F0890911008079731F481E0C0
:1094100090E09093100880930F08809185089091B8
:109420008608A0918708B091880887389847AF4F81
:10943000B10509F05DC080910F0890911008892B4B
:1094400089F4CCE9D7E006EF17E0E1E6EE2EFF2441
:10945000FA941882E982FA820E94D12C23960C1782
:109460001D07B9F780910F0890911008019789F4B2
:10947000CCE9D7E006EF17E071E6E72EFF24FA9477
:109480001882E982FA820E94D12C26960C171D07B9
:10949000B9F780910F0890911008029789F4CCE9F0
:1094A000D7E00CEF17E061E6E62EFF24FA9418826D
:1094B000E982FA820E94D12C2C960C171D07B9F76D
:1094C00080910F0890911008069731F481E090E0A8
:1094D0009093100880930F0880910F0890911008C6
:1094E000079731F481E090E09093100880930F0883
:1094F0008091850890918608A0918708B09188088E
:109500008F389047AF4FB10509F063C080910F08C5
:1095100090911008892B99F4CCE9D7E006EF17E079
:1095200030E5D32E4AE0E42E5AE5F52ED882E982C2
:10953000FA820E94D12C23960C171D07B9F780914F
:109540000F0890911008019799F4CCE9D7E006EF45
:1095500017E080E5D82E9AE0E92E2AE5F22ED8828F
:10956000E982FA820E94D12C26960C171D07B9F7C2
:1095700080910F0890911008029799F4CCE9D7E0F8
:109580000CEF17E0F0E5DF2EAAE0EA2EBAE5FB2E9D
:10959000D882E982FA820E94D12C2C960C171D07E2
:1095A000B9F780910F0890911008069731F481E087
:1095B00090E09093100880930F0880910F0890918D
:1095C0001008079731F481E090E0909310088093A1
:1095D0000F088091850890918608A0918708B09126
:1095E0008808873C9843AF4FB10509F057C0809178
:1095F0000F0890911008892B99F4CCE9D7E006EF79
:1096000017E06DEFD62E79EEE72EE0E1FE2ED88240
:10961000E982FA820E94D12C23960C171D07B9F714
:1096200080910F0890911008019799F4CCE9D7E048
:1096300006EF17E03DEFD32E49EEE42E50E1F52E74
:10964000D882E982FA820E94D12C26960C171D0737
:10965000B9F780910F0890911008029799F4CCE91E
:10966000D7E00CEF17E08DEFD82E99EEE92E20E130
:10967000F22ED882E982FA820E94D12C2C960C1705
:109680001D07B9F780910F0890911008069731F4E3
:1096900081E090E09093100880930F0880918508F6
:1096A00090918608A0918708B0918808873D9842DC
:1096B000AF4FB10509F057C080910F089091100885
:1096C000892B99F4CCE9D7E006EF17E0F7E8DF2E15
:1096D000AEECEA2EBAEFFB2ED882E982FA820E9423
:1096E000D12C23960C171D07B9F780910F08909184
:1096F0001008019799F4CCE9D7E006EF17E067E886
:10970000D62E7EECE72EEAEFFE2ED882E982FA8290
:109710000E94D12C26960C171D07B9F780910F08CF
:1097200090911008029799F4CCE9D7E00CEF17E07C
:1097300037E8D32E4EECE42E5AEFF52ED882E9828C
:10974000FA820E94D12C2C960C171D07B9F7809134
:109750000F0890911008069731F481E090E0909303
:10976000100880930F088091850890918608A09139
:109770008708B09188088F30904FAF4FB10509F03E
:109780005DC080910F0890911008892B89F4CCE975
:10979000D7E026EFE22E27E0F22E16E90AE0188342
:1097A00009831A830E94D12C2396EC16FD06B9F783
:1097B00080910F0890911008019789F4CCE9D7E0C7
:1097C00096EFE92E97E0F92E16E90AE0188309834F
:1097D0001A830E94D12C2696EC16FD06B9F78091CB
:1097E0000F0890911008029789F4CCE9D7E08CEF2C
:1097F000E82E87E0F82E16E90AE0188309831A8319
:109800000E94D12C2C96EC16FD06B9F780910F081A
:1098100090911008069731F481E090E09093100841
:1098200080930F0880910F0890911008079731F4EA
:1098300081E090E09093100880930F0864E670E058
:1098400080E090E00E94F52D82E08093560910920E
:10985000220A60E08DE0DF91CF911F910F91FF9080
:10986000EF90DF900C946E2B84379A46A041BE4057
:1098700009F09BC88091F9079091FA07181619060C
:109880000CF0AEC81092FA071092F9070E945D40E2
:109890000E94663B8AC88F3F91052FEFA207B10552
:1098A00049F482E090E09093100880930F0881E0E3
:1098B00090E0C7C8873A28E592072FEFA207B105C5
:1098C00019F486E090E0EFCF8F3C20E392072FEF72
:1098D000A207B10519F487E090E0E5CF8730984FF3
:1098E000AF4FB10509F0B1C81092100810920F08DF
:1098F000CCE9D7E0188219821A820E94D12C2396D3
:1099000087E0C63FD807B1F7A0C880EF90E0E3C872
:1099100081E090E012C990931C0280931B020C948A
:109920008B43069714F40C9425440C948B4390932A
:10993000F3068093F2060C948B4306970CF418C838
:109940000C946E442F923F924F925F926F927F924F
:109950008F929F92AF92BF92CF92DF92EF92FF923F
:109960000F931F93CF93DF9300D000D0CDB7DEB716
:10997000CE0101960E94FA3EFC808F2D90E09093DC
:10998000300880932F088D81082F10E010932E0847
:1099900000932D088E8190E090932C0880932B08E3
:1099A0008A8190E090932A08809329088B8190E027
:1099B0009093280880932708898190E08053984FDE
:1099C0009093260880932508CE0101960E94F72ED9
:1099D00090E0009709F457C09093240880932308DF
:1099E000C80124E6F29E800D911D11249093E70694
:1099F0008093E6064090230850902408AEE04A0E7B
:109A0000511CF0901808909019084091DC06509174
:109A1000DD0620917107309172072090E1063090A9
:109A2000E2066091730770917407009175071091B9
:109A30007607EDE1F2E0812CE12CB4E67B2E6F019C
:109A4000C40CD51CD601DC90B1E0DB1271C0D08013
:109A5000DB123AC0B580C680D12CB79CC00CD11C9B
:109A600011248C159D05A9F4B280A3E0BA1671F0FB
:109A7000B4E0BB1609F497C0A2E0BA120AC0A2E093
:109A80009A2EE12C06C087E090E0A6CFA2E0FA2E45
:109A9000812C6380A480B12C679CA00CB11C112484
:109AA0008A159B058CF08C159D0574F4D280B2E06C
:109AB000DB1609F47BC0A3E0DA1609F481C0B1E03B
:109AC000DB1202C0038510E0D180A1E0DA1230C0C1
:109AD000B184C284D12CB79CC00CD11C11248C152C
:109AE0009D0559F4B280B2E0BB1609F472C0A3E040
:109AF000BA1203C0B2E0FB2E812C6780A084B12C87
:109B0000679CA00CB11C11248A159B058CF08C1548
:109B10009D0574F4D280B2E0DB1609F45EC0A3E0C8
:109B2000DA1609F464C0B1E0DB1202C0058510E06A
:109B30007696A2E0E537FA0709F081CFE092E506D4
:109B4000909219088092E006F09218081093760718
:109B5000009375073092E2062092E1067093740735
:109B6000609373075093DD064093DC0630937207D1
:109B70002093710726960FB6F894DEBF0FBECDBFB7
:109B8000DF91CF911F910F91FF90EF90DF90CF90D9
:109B9000BF90AF909F908F907F906F905F904F900D
:109BA0003F902F900895B2E0FB2E73CFA4852A2E0C
:109BB000312C638570E099249394EE24E39484CF50
:109BC000448550E0238530E0FF24F3948824839477
:109BD0007BCFA2E09A2EE12C90CFA6852A2E312CA5
:109BE000658570E099249394EE24E394A1CF468593
:109BF00050E0258530E0FF24F3948824839498CFA7
:109C00000E940190FB0101900020E9F73197AF011C
:109C1000461B570BDC01ED91FC910280F381E02D96
:109C200019948F929F92AF92BF920F931F93CF93ED
:109C3000DF93CDB7DEB7A1970FB6F894DEBF0FBEA6
:109C4000CDBF19A2423008F44AE08E010F5D1F4FCC
:109C5000842E912CB12CA12CA50194010E94828FFD
:109C6000E62FB901CA01EA30FCF4E05DD801EE93B9
:109C70008D01232B242B252B79F790E080E0109782
:109C800021F0BD018BEC9AE0BDDFA1960FB6F894F0
:109C9000DEBF0FBECDBFDF91CF911F910F91BF905F
:109CA000AF909F908F900895E95CE0CFCF92DF92C4
:109CB000EF92FF92CF93DF936C01990FEE08FF08AC
:109CC000F7FE16C08DE20E94B93EEC0166277727A9
:109CD000CB016C197D098E099F094AE0A2DF8C0F28
:109CE0009D1FDF91CF91FF90EF90DF90CF9008956F
:109CF0004AE0C701B601DF91CF91FF90EF90DF906E
:109D0000CF908FCF682F70E090E080E04AE089CF5D
:109D1000CF93DF93BC018FE998E074DFEC016DEA2B
:109D200073E08FE998E06EDF8C0F9D1FDF91CF917C
:109D300008951092EC0683EB9AE00E94252E813064
:109D4000910541F1029769F18BE99AE00E94252E75
:109D50008130910559F1029781F183E89AE00E94E0
:109D6000252E8130910571F1029799F18BE69AE0E9
:109D70000E94252E8230910509F44FC08330910551
:109D800069F1019771F589E194E0C2DF84E0809385
:109D9000EC0627C080EB93E0BBDF81E08093EC060C
:109DA000D3CF8FEB93E0B4DF8BE0F8CF83ED93E07C
:109DB000AFDF82E08093EC06D0CF82EE93E0A8DFA5
:109DC0008CE0F8CF86EF93E0A3DF83E08093EC068E
:109DD000CDCF85E094E09CDF8DE0F8CF88E294E081
:109DE00097DF83E59AE00E94252E81309105D1F01E
:109DF0000297F9F08BE39AE00E94252E81309105BD
:109E0000E9F0029711F183E29AE00E94252E813059
:109E1000910501F1029729F108958CE394E078DF30
:109E20008EE0B5CF80E594E073DF85E08093EC06AB
:109E3000E1CF8FE594E06CDF8FE0F8CF83E794E02B
:109E400067DF86E08093EC06DECF82E894E060DF97
:109E500080E1F8CF86E994E05BDF87E08093EC0651
:109E6000089585EA94E054DF81E1F8CFBC018BECE2
:109E70009AE0C8CE2F923F924F925F926F927F925C
:109E80008F929F92AF92BF92CF92DF92EF92FF920A
:109E90000F931F93CF93DF93C1E0D1E08DE0382E75
:109EA00097E1292E2AE0422E512C66246A94712CC7
:109EB00045E0E42EF12C5EEFC52ED12C6BE3A62EEF
:109EC000B12C77E1872E912C68EC70E080E090E077
:109ED0000E94F52D0E94F52FD093EF0A04E41DE0B7
:109EE00020E440E860E080E00E94E9338FE395E2FF
:109EF0000E94FA283092060B2092070B80911002E4
:109F000090911102B2010E946F8FCB01CFDE809140
:109F1000100290911102B2010E946F8FC7DE89EB8F
:109F200094E0A4DF80910E0290910F02B2010E9492
:109F30006F8FCB01BBDE80910E0290910F02B201B8
:109F40000E946F8FB3DE80910D020CE21DE088232A
:109F500011F004E11DE02CE040E16CE08AE30E9496
:109F6000E9338091EB060CEF1CE0882311F004EE3E
:109F70001CE02CE040E16CE08CE40E94E93320918D
:109F80000B0230910C024AED4203C001439F900D39
:109F90001124B3010E946F8F8B010A5D1F4F0E9435
:109FA0007A3424E0402F6EE284E30E94C73380912C
:109FB0001802882331F021E04AE065E286E00E9441
:109FC000C73380911702882331F021E048E065E231
:109FD00083E10E94C73380911602882331F021E08B
:109FE0004AE065E28EE10E94C73380911502882322
:109FF00031F021E048E065E28BE20E94C7338091B6
:10A000001402882331F021E048E065E286E30E94F3
:10A01000C73380911302882331F021E04AE065E2E2
:10A0200081E40E94C73380911202882331F021E03D
:10A030004AE065E28EE40E94C733C13009F048C0AF
:10A0400021E040E168E18DE00E94C7330E942530A5
:10A05000811142CF0E942423892B09F435CF82E05D
:10A06000809356091092220A61E08DE00E946E2BC7
:10A070008091850890918608A0918708B091880802
:10A0800085312BE8920720E9A2072EE0B20709F0FC
:10A09000D2C0C13009F068C0209110023091110285
:10A0A0002150310937FF6FC1909211028092100246
:10A0B000853D2BE4920720E9A2072EE0B20709F0C4
:10A0C000D3C0CF5F10E0CD3009F0A4C1C1E0A2C180
:10A0D000C23029F421E040E168E185E2B5CFC33028
:10A0E00029F421E04EE068E18AE3AECF21E04CE0C4
:10A0F00068E1C43079F1C53029F421E04AE067E233
:10A1000086E0A2CFC63029F421E048E067E283E18F
:10A110009BCFC73029F421E04AE067E28EE194CF7B
:10A12000C83029F421E048E067E28BE28DCFC930E6
:10A1300029F421E048E067E286E386CFCA3029F4BB
:10A1400021E04AE067E281E47FCFCB3029F421E0CF
:10A150004AE067E28EE478CFCC3009F077CF21E097
:10A160004FE264E382E070CFC23069F420910E02C6
:10A1700030910F022150310937FF33C1B0920F02E5
:10A18000A0920E0295CFC33009F002C120910D02BA
:10A19000222319F010920D028BCFD0930D0288CF9D
:10A1A0002091EB06222319F01092EB0681CFD09379
:10A1B000EB067ECF20911802222319F0109218028C
:10A1C00077CFD093180274CF20911702222319F071
:10A1D000109217026DCFD09317026ACF209116020A
:10A1E000222319F01092160263CFD093160260CF8B
:10A1F00020911502222319F01092150259CFD09305
:10A20000150256CF20911402222319F01092140245
:10A210004FCFD09314024CCF20911202222319F079
:10A220001092120245CFD093120242CFD0920C026C
:10A23000C0920B023DCF85394BE0940740E9A4075B
:10A240004EE0B40709F0D2C0C13021F520911002D0
:10A25000309111022F5F3F4F283131050CF404C1BA
:10A26000109211021092100285359B4CA049BE40FD
:10A2700009F483C064E670E080E090E00E94F52D70
:10A2800082E0809356091092220A60E08DE00E94DD
:10A290006E2B1ACEC23079F420910E0230910F024B
:10A2A0002F5F3F4F2C3331050CF40DC110920F027C
:10A2B00010920E02D9CFC33009F0DBC020910D02FD
:10A2C000222319F010920D02CFCFD0930D02CCCFE4
:10A2D0002091EB06222319F01092EB06C5CFD09304
:10A2E000EB06C2CF20911802222319F01092180217
:10A2F000BBCFD0931802B8CF20911702222319F0B8
:10A3000010921702B1CFD0931702AECF2091160250
:10A31000222319F010921602A7CFD0931602A4CFD1
:10A3200020911502222319F0109215029DCFD0938F
:10A3300015029ACF20911402222319F010921402D0
:10A3400093CFD093140290CF20911302222319F0BF
:10A3500010921302ADCED0931302AACE2091120216
:10A36000222319F0109212027FCFD09312027CCFD9
:10A37000F0920C02E0920B0277CFC15010E009F08E
:10A3800049C0CCE047C0309311022093100290CE18
:10A39000C43009F405CFC53009F40CCFC63009F438
:10A3A00013CFC73009F41ACFC83009F421CFC93010
:10A3B00009F428CFCA3041F2CB3009F42DCFCC308C
:10A3C00009F076CE20910B0230910C02265F3F4FB0
:10A3D0002F3F31050CF02ACF30930C0220930B0253
:10A3E00067CE30930F0220930E0262CE84302AE1B2
:10A3F000920720E1A2072EE0B20749F084374AE62F
:10A40000940740E1A4074EE0B40709F051CE109242
:10A41000130811E064E670E080E090E00E94F52D02
:10A4200082E0809356091092220A60E08DE00E943B
:10A430006E2B112309F448CD6CE271E080E090E0CE
:10A44000DF91CF911F910F91FF90EF90DF90CF9010
:10A45000BF90AF909F908F907F906F905F904F9044
:10A460003F902F900C94F52D309311022093100201
:10A47000FBCEC43009F42CCFC53009F433CFC6303D
:10A4800009F43ACFC73009F441CFC83009F448CFB6
:10A49000C93009F44FCFCA3009F456CFCB3009F494
:10A4A0005DCFCC3009F0E0CE20910B0230910C0250
:10A4B0002A503109253031050CF45ACF30930C0263
:10A4C00020930B02D1CE30930F0220930E02CCCEFC
:10A4D0002F923F924F925F926F927F928F929F92B4
:10A4E000AF92BF92CF92DF92EF92FF920F931F93A2
:10A4F000CF93DF93CDB7DEB762970FB6F894DEBF88
:10A500000FBECDBFCE010D960E94FA3EE889F0E065
:10A51000F0933008E0932F08698970E070932E085B
:10A5200060932D088A8990E090932C0880932B08E3
:10A530004E8550E050932A08409329082F8530E03B
:10A5400030932808209327088D8590E08053984FFA
:10A550009093260880932508789734F0E8E0F0E09F
:10A56000F0933008E0932F086C33710524F01092BB
:10A570002E0810922D084D30510534F041E050E086
:10A5800050932A08409329082032310534F021E005
:10A5900030E030932808209327088433984034F023
:10A5A0008AED97E09093260880932508332433940E
:10A5B0003AE0E32EF12CCC24C394D12C5EE1452E5D
:10A5C000512C6FE1A62EB12C7BE3872E912CE7E175
:10A5D0006E2E712C68EC70E080E090E00E94F52D0A
:10A5E000CE0107960E94FA3E8C8590E090932C084D
:10A5F00080932B080E94F52F20E3222E61E06093C8
:10A60000EF0A04EE18E020E440E860E080E00E94F9
:10A61000E9338FE395E20E94FA287AE07093060B03
:10A620008CE18093070B80912F0890913008B7013F
:10A630000E946F8FCB013ADB80912F0890913008F8
:10A64000B7010E946F8F32DB89EB94E00FDC8091C1
:10A650002D0890912E08B7010E946F8FCB0126DB49
:10A6600080912D0890912E08B7010E946F8F1EDBFC
:10A6700089EB94E0FBDB80912B0890912C08B701CB
:10A680000E946F8FCB0112DB80912B0890912C08D8
:10A69000B7010E946F8F0ADB98E09093060B20921F
:10A6A000070B8091270890912808B7010E946F8FAF
:10A6B000CB01FCDA8091270890912808B7010E940D
:10A6C0006F8FF4DA8BEB94E0D1DB809129089091C5
:10A6D0002A08B7010E946F8FCB01E8DA8091290820
:10A6E00090912A08B7010E946F8FE0DA8BEB94E01B
:10A6F000BDDB8091250890912608D8DA21E040E161
:10A700006EE18AE0321639F062E0361253C021E081
:10A7100040E16EE182E20E94C7330E942530811140
:10A720006DCF0E94242300E0892B09F424C182E02C
:10A73000809356091092220A61E08DE00E946E2BF0
:10A740008091850890918608A0918708B09188082B
:10A7500085319B48A049BE4071F471E037124AC070
:10A7600080912F0890913008019797FFFAC370925B
:10A77000300860922F088091850890918608A091FA
:10A780008708B091880885399B40A049BE4009F0F0
:10A79000A0C061E0361241C180912F08909130082D
:10A7A0000196883191050CF436C41092300810924D
:10A7B0002F088FC073E0371205C021E040E162E34B
:10A7C00088E0A9CF84E0381205C021E040E162E3CF
:10A7D00080E2A1CF95E0391205C021E040E262E3BA
:10A7E00088E399CF26E0321298CF21E040E16EE174
:10A7F0008AE391CF82E038120CC080912D089091AD
:10A800002E08019797FF02C490922E0880922D087F
:10A81000B2CF93E03912AAC32091270830912808BB
:10A820002150310930932808209327088091290866
:10A8300090912A088130910509F4E3C38330910592
:10A8400079F08530910561F0AC01475051094230F3
:10A85000510530F08A30910519F08C30910539F4AA
:10A860001216130624F0B0922808A09227089C0123
:10A870002D7F2430310519F02930310559F420910C
:10A880002708309128081216130624F05092280841
:10A8900040922708029709F06ECF80912708909187
:10A8A0002808181619060CF466CF6DE170E0709355
:10A8B0002808609327085FCF8091290890912A0883
:10A8C0000197181619060CF085C090932A088093FA
:10A8D00029088091850890918608A0918708B091F9
:10A8E000880884309A41A041BE4009F006C12091F9
:10A8F0002B0830912D0840912F0850912708609126
:10A9000029088091250890912608803D77E09707D7
:10A9100010F0805D974089836A835B834C833D831D
:10A920002E83CE0101960E9462361092150801E036
:10A930008091850890918608A0918708B091880839
:10A9400084372AE6920720E1A2072EE0B20709F039
:10A95000FBC01092150801E064E670E080E090E032
:10A960000E94F52D82E0809356091092220A60E041
:10A970008DE00E946E2BDDD91091EC06153011F0A0
:10A980001F3071F461E03612FAC080912F08909167
:10A990003008019797FF94C37092300860922F0897
:10A9A000143019F01E3009F0E9C181E0381609F4BD
:10A9B000D8C192E039123CC280912D0890912E08A6
:10A9C00001968C3391050CF4DAC310922E08109284
:10A9D0002D08D4C18CE090E078CF8091250890912B
:10A9E000260801978A3D27E092072CF090932608CD
:10A9F000809325086ECF63E378E070932608609318
:10AA00002508B9CE1092300810922F08D9C20196AD
:10AA100090932E0880932D08D3C272E037120EC097
:10AA200080912D0890912E0801968C3391050CF49D
:10AA300042C310922E0810922D084BCF83E038129B
:10AA4000EFC220912708309128082F5F3F4F3093A5
:10AA50002808209327088091290890912A0881309E
:10AA6000910591F08330910579F08530910561F081
:10AA7000AC01475051094230510550F08A309105E0
:10AA800019F08C30910559F42032310524F41AC0A4
:10AA90002032310524F0D0922808C09227089C016A
:10AAA0002D7F2430310519F02930310559F42091DA
:10AAB0002708309128082F31310524F0D09228083A
:10AAC000C0922708029709F004CF8091270890913F
:10AAD00028084E970CF4FDCED0922808C092270883
:10AAE000F8CE8091290890912A0801968D30910521
:10AAF00034F490932A088093290800E019CFD0926B
:10AB00002A08C0922908F9CF80912508909126083B
:10AB10000196843328E092072CF4909326088093C2
:10AB20002508EBCF6AED77E070932608609325083F
:10AB3000D0CE1092300810922F089CC201969093AC
:10AB40002E0880932D0896C2853D6BE4960760E938
:10AB5000A6076EE0B60739F4339477E03712FCCEDF
:10AB600033243394F9CE85359B4CA049BE4009F07F
:10AB7000F3CE3A943110F0CE96E0392EEDCE72E05D
:10AB800037120CC080912D0890912E08019797FFE5
:10AB9000E7C290922E0880922D0802CF83E03812EF
:10ABA00094C2209127083091280821503109309310
:10ABB0002808209327088091290890912A08AC0141
:10ABC0004D7F4130510599F08530910561F0BC0110
:10ABD000675071096230710550F08A30910519F0A3
:10ABE0008C309105A9F4121613065CF003C01216FE
:10ABF000130624F0B0922808A0922708843091050B
:10AC000089F08630910539F04930510559F403C077
:10AC100084309105B1F72091270830912808121649
:10AC2000130694F4029709F0BBCE80912708909107
:10AC30002808181619060CF4B3CE6DE170E0709375
:10AC4000280860932708ACCE509228084092270825
:10AC5000E9CF8091290890912A08019718161906C2
:10AC6000ACF490932A0880932908143009F09ACE06
:10AC70008091290890912A0801968D3091050CF059
:10AC800033C190932A088093290878C08CE090E023
:10AC9000E8CF809125089091260801978A3D27E00A
:10ACA00092070CF062C263E378E070932608609329
:10ACB0002508143009F076CE84E03816C9F295E004
:10ACC000391609F416C126E0321258C080912B08BB
:10ACD00090912C088497CCF080912D0890912E08AB
:10ACE0008B33910509F02EC180912F089091300887
:10ACF00010922E0810922D080196883191050CF0C3
:10AD00001CC19093300880932F0810922C08109249
:10AD10002B0820912D0830912F0840912708509141
:10AD200029088091250890912608803D67E09607C4
:10AD300010F0805D974089835A834B833C832D8339
:10AD40001E82CE0101960E94623618C01092300811
:10AD500010922F08E4C1019690932E0880932D083D
:10AD6000DEC180912F0890913008019688319105BD
:10AD70000CF400C21092300810922F08133011F01A
:10AD80001D3009F560912B0850912D0840912F0836
:10AD90003091270820912908809125089091260854
:10ADA000803D77E0970710F0805D974089832A8384
:10ADB0003B834C835D836E83CE0101960E94623695
:10ADC0001092150801E0113011F01B3019F41092A7
:10ADD000150801E0163011F0103129F4339487E0A2
:10ADE000381609F4B5C0123011F01C3029F43A9429
:10ADF000311002C086E0382E002309F4EBCB6296B6
:10AE00000FB6F894DEBF0FBECDBFDF91CF911F917B
:10AE10000F91FF90EF90DF90CF90BF90AF909F90F9
:10AE20008F907F906F905F904F903F902F900895FC
:10AE300023E0321241CF20912708309128082F5F5C
:10AE40003F4F30932808209327088091290890913C
:10AE50002A0881309105B1F08330910579F0853071
:10AE6000910561F0AC01475051094230510530F075
:10AE70008A30910519F08C30910539F52032310571
:10AE800024F40BC020323105D4F0D0922808C092AF
:10AE900027088430910509F077C1029709F06ECF39
:10AEA00080912708909128084E970CF467CFD09294
:10AEB0002808C092270862CF8630910549F09C018E
:10AEC0002D7F2930310521F0E8CF84309105A1F79D
:10AED00020912708309128082F313105F4F2D092C3
:10AEE0002808C0922708D9CFD0922A08C0922908F2
:10AEF00045CF80912508909126080196843368E01B
:10AF000096072CF4909326088093250837CF8AED76
:10AF100097E09093260880932508133009F039C1F3
:10AF200060912B0850912D0840912F0830912708EF
:10AF3000209129088AED97E037CF109230081092BF
:10AF40002F08E3CE019690932E0880932D08DDCE36
:10AF5000123009F44FCF332433941C3009F04CCF16
:10AF600049CF9093300880932F0805CC94E0391690
:10AF700009F4A2CC25E0321609F42FCD66E0361292
:10AF8000FACB80912B0890912C088497CCF080917B
:10AF90002D0890912E088B33910509F038CD8091C2
:10AFA0002F089091300810922E0810922D080196CB
:10AFB000883191050CF026CD9093300880932F08AE
:10AFC00010922C0810922B0820912D0830912F08F8
:10AFD00040912708509129088091250890912608D2
:10AFE000803D77E0970710F0805D974089835A8312
:10AFF0004B833C832D831E82CE0101960E946236D4
:10B00000BACB121613060CF445CC2DCC90932E0817
:10B0100080932D08B0CB9093300880932F0859CCA3
:10B0200074E0371609F45DCD85E0381609F46CCD6F
:10B0300096E039124ECC80912B0890912C08849781
:10B04000CCF080912D0890912E088B33910509F05A
:10B0500075CD80912F089091300810922E08109293
:10B060002D080196883191050CF063CD909330083E
:10B0700080932F0810922C0810922B0820912D08F5
:10B0800030912F0840912708509129088091250878
:10B0900090912608803D77E0970710F0805D9740FB
:10B0A00089835A834B833C832D831E82CE01019674
:10B0B0000E9462360ECC90932E0880932D0809CC06
:10B0C0009093300880932F086BCC24E0321609F45B
:10B0D000C0CD65E0361609F4DCCD76E0371260CCE1
:10B0E00080912B0890912C088497CCF080912D08AA
:10B0F00090912E088B33910509F02DCE80912F0869
:10B100009091300810922E0810922D0801968831E7
:10B1100091050CF01BCE9093300880932F0810926D
:10B120002C0810922B0820912D0830912F08409167
:10B130002708509129088091250890912608803D84
:10B1400077E0970710F0805D974089835A834B839F
:10B150003C832D831E82CE0101960E946236A9CDCA
:10B1600090932E0880932D081BCC909326088093F3
:10B1700025089FCD9093300880932F08FFCD9093A2
:10B180002E0880932D08FACD8630910509F097CED0
:10B1900084CE1D3009F017CEC3CEFF920F931F93BC
:10B1A000CF93DF93FF24F394F092EF0A07E81EE1B8
:10B1B00020E440E860E080E00E94E9331092EF0A6A
:10B1C0008FE395E20E94FA288EE18093060B8BE0D4
:10B1D0008093070B80912F0890913008CAE0D0E04F
:10B1E000BE010E946F8FCB010E94564E80912F08A6
:10B1F00090913008BE010E946F8F0E94564E89EBDD
:10B2000094E00E94364F80912D0890912E08BE0147
:10B210000E946F8FCB010E94564E80912D08909115
:10B220002E08BE010E946F8F0E94564E89EB94E05B
:10B230000E94364F80912B0890912C08BE010E94ED
:10B240006F8FCB010E94564E80912B0890912C0855
:10B25000BE010E946F8F0E94564EF092EF0A87E85F
:10B2600092E20E94FA288AE28093060B84E280939D
:10B27000070B80910F08909110088730910509F015
:10B2800017C28091FB079091FC0764ED7FEF0E944D
:10B290006F8F6C597F4F70931C0260931B028091DB
:10B2A0001B0290911C020E94564E409175075091CE
:10B2B000760757FF02C04D5F5F4F559547955595EF
:10B2C00047954093E9065093EA0621E060E28DE05D
:10B2D0000E94C73380911B0290911C0297FD039638
:10B2E00095958795959587959093EA068093E906BD
:10B2F00080910F0890911008892B21F41092EA0692
:10B300001092E90622E04091E90661E28DE00E9498
:10B31000C7338AE28093060B8CE28093070B8091FF
:10B32000F2069091F3060E94564E40917307509199
:10B33000740757FF02C04D5F5F4F55954795559570
:10B3400047954093E9065093EA0621E068E28DE0D4
:10B350000E94C7334091F2065091F30657FF02C096
:10B360004D5F5F4F55954795559547954093E90635
:10B370005093EA0622E069E28DE00E94C7338AE238
:10B380008093060B84E38093070B8091F0069091E5
:10B39000F1060E94564E409171075091720757FF77
:10B3A00002C04D5F5F4F5595479555954795409322
:10B3B000E9065093EA0621E060E38DE00E94C7337E
:10B3C0004091F0065091F10657FF02C04D5F5F4F6C
:10B3D00055954795559547954093E9065093EA064C
:10B3E00022E061E38DE00E94C7338EEE9AE30E9473
:10B3F000FA28C5E4C093060B14E11093070B8DEBFC
:10B4000094E00E94364FDEE5D093060B1093070BB5
:10B41000809102030E94824E80EC94E00E94364F9D
:10B42000809101030E94824EC093060B1EE110938F
:10B43000070B82EC94E00E94364FD093060B1093DA
:10B44000070B809100030E94824E80EC94E00E94E2
:10B45000364F8091FF020E94824E12E41093060B39
:10B4600009E20093070B85EC94E00E94364F8BE5D0
:10B470008093060B0093070B809104030E94824E79
:10B4800080EC94E00E94364F809103030E94824E2C
:10B490001093060B84E38093070B89EC94E00E94E1
:10B4A000364FC093060BCEE3C093070B8DEC94E0B0
:10B4B0000E94364F80911A08811106C1D093060B65
:10B4C000C093070B80911C0890911D080E94564E56
:10B4D0008091F706882331F024E044E065E187E0BD
:10B4E0000E94C7338091F606882331F024E044E0BF
:10B4F00065E183E10E94C7338091F506882331F02E
:10B5000024E044E065E18FE10E94C7338091F406B6
:10B51000882331F024E044E065E18BE20E94C733E8
:10B5200080919307882331F024E044E065E187E3CC
:10B530000E94C7338091F9079091FA07019789F427
:10B54000809120088111CEC01092EF0A21E048E0DE
:10B550006CE185E00E94C733809120088111109230
:10B56000EF0A8091F9079091FA07029789F4809188
:10B5700020088111BBC01092EF0A21E048E06CE185
:10B5800081E10E94C7338091200881111092EF0A57
:10B590008091F9079091FA07039789F48091200828
:10B5A0008111A8C01092EF0A21E048E06CE18DE122
:10B5B0000E94C7338091200881111092EF0A809178
:10B5C000F9079091FA07049789F480912008811176
:10B5D00095C01092EF0A21E048E06CE189E20E94F8
:10B5E000C7338091200881111092EF0A8091F907EA
:10B5F0009091FA07059789F480912008811182C003
:10B600001092EF0A21E048E06CE185E30E94C73325
:10B610008091200881111092EF0A8091F907909192
:10B62000FA07069789F48091200881116FC0109263
:10B63000EF0A21E048E065E283E00E94C733809191
:10B64000200881111092EF0A8091F9079091FA0772
:10B65000079789F48091200881115CC01092EF0A4D
:10B6600021E048E06DE283E00E94C733809120082A
:10B6700081111092EF0A8091F9079091FA070897CB
:10B6800089F480912008811149C01092EF0A21E0CD
:10B6900048E065E383E00E94C73380912008811170
:10B6A0001092EF0ADF91CF911F910F91FF900895B3
:10B6B000069709F0F4CD8091FD079091FE076DE1AA
:10B6C00070E00E946F8FE7CD89E58093060BC093F1
:10B6D000070B80ED94E00E94364F8091F607909121
:10B6E000F707F4CE81E08093EF0A30CF81E08093BA
:10B6F000EF0A43CF81E08093EF0A56CF81E0809339
:10B70000EF0A69CF81E08093EF0A7CCF81E08093DC
:10B71000EF0A8FCF81E08093EF0AA2CF81E0809380
:10B72000EF0AB5CF85ED8093BC00809159089091C8
:10B730005A08A0915B08B0915C080796A11DB11D45
:10B7400023E0B695A795979587952A95D1F72091EF
:10B75000BC0024FD03C01092570808954091590879
:10B7600050915A0860915B0870915C08452B462BFC
:10B77000472B69F30097A105B10541F025E32A9510
:10B78000F1F700000197A109B109E1CF80915808B4
:10B790000C94D8341F93CF93DF93EC01162F0E94A3
:10B7A000138D181739F0612FCE01DF91CF911F91C2
:10B7B0000C941B8DDF91CF911F9108952F923F9292
:10B7C0004F925F926F927F928F929F92AF92BF92B1
:10B7D000CF92DF92EF92FF920F931F93CF93DF935D
:10B7E000CDB7DEB76A970FB6F894DEBF0FBECDBFF8
:10B7F0002091190230911A02388F2F8B10922C0849
:10B8000010922B0841E050E05A8F498F912C87E12C
:10B81000E82EFF24F3948091190290911A02019767
:10B82000E89EF001E99EF00D1124EB58FD4F2081B8
:10B83000422F50E05A8B498B2181422F50E05C8B84
:10B840004B8B2281422F50E05E8B4D8BA3802A2DA3
:10B8500030E0388B2F872481A22EB12C2581422FF6
:10B8600050E05A8349832681422F50E05C834B830A
:10B870002781422F50E05E834D832085422F50E088
:10B8800058874F832185422F50E05A874987228568
:10B89000422F50E05C874B872385422F50E05E8724
:10B8A0004D872484312C4584512C6684712CC784A7
:10B8B000D12C21E03089311101C020E02093180201
:10B8C000E89EF001E99EF00D1124EB58FD4F21E0B8
:10B8D0003189311101C020E020931702E89EF00168
:10B8E000E99EF00D1124EB58FD4F21E03289311112
:10B8F00001C020E020931602E89EF001E99EF00DC1
:10B900001124EB58FD4F21E03389311101C020E0B3
:10B9100020931502E89EF001E99EF00D1124EB58EA
:10B92000FD4F21E03489311101C020E02093140241
:10B93000E89EF001E99EF00D1124EB58FD4F21E047
:10B940003589311101C020E020931302E89EF001F7
:10B95000E99EF00D1124EB58FD4F81E0968991117D
:10B9600001C080E08093120264E670E080E090E025
:10B970000E94F52D80912B0890912C0801969093B0
:10B980002C0880932B08029754F08091200851E0F6
:10B9900085278093200810922C0810922B080E9473
:10B9A000F52FF092EF0A04E411E120E440E860E0B2
:10B9B00080E00E94E9338EEE9AE30E94FA2882E347
:10B9C0008093060B99E09093070B80911902909158
:10B9D0001A020E94564E1092EF0AE0E7E093060B1F
:10B9E000F9E0F093070B8F8598890E94564EF092EC
:10B9F000EF0A28E12093060B30E23093070B4AE070
:10BA0000A416B10424F483ED94E00E94364FC501DE
:10BA10000E94564E89EB94E00E94364F89819A81AC
:10BA20000A9724F483ED94E00E94364F89819A812D
:10BA30000E94564EF092EF0A94E59093060BE0E2D6
:10BA4000E093070B2B813C812A30310524F483EDF0
:10BA500094E00E94364F8B819C810E94564E89EB68
:10BA600094E00E94364F4D815E814A30510524F4A6
:10BA700083ED94E00E94364F8D819E810E94564E48
:10BA800058E15093060B8BE28093070BEF81F8850A
:10BA90003A9724F483ED94E00E94364F8F81988585
:10BAA0000E94564E89EB94E00E94364F29853A85D4
:10BAB0002A30310524F483ED94E00E94364F8985C5
:10BAC0009A850E94564EF092EF0A34E53093060BA9
:10BAD0004BE24093070B8B859C850A9724F483EDFA
:10BAE00094E00E94364F8B859C850E94564E89EBD0
:10BAF00094E00E94364FED85FE853A9724F483ED5D
:10BB000094E00E94364F8D859E850E94564EF8E146
:10BB1000F093060B26E32093070B3AE0231631043B
:10BB200024F483ED94E00E94364FC1010E94564EEA
:10BB300089EB94E00E94364F4AE04416510424F405
:10BB400083ED94E00E94364FC2010E94564EF0925F
:10BB5000EF0A54E55093060B86E38093070B9AE0B7
:10BB60006916710424F483ED94E00E94364FC301FA
:10BB70000E94564E89EB94E00E94364FEAE0CE16C2
:10BB8000D10424F483ED94E00E94364FC6010E9454
:10BB9000564E80911802882331F021E04BE064E199
:10BBA0008AE00E94C73380911702882331F021E098
:10BBB0004BE064E18AE10E94C7338091160288233A
:10BBC00031F021E04BE064E18AE20E94C7338091CA
:10BBD0001502882331F021E04CE064E189E30E9402
:10BBE000C73380911402882331F021E04CE064E1F6
:10BBF00089E40E94C73380911302882331F021E049
:10BC00004CE064E189E50E94C733809112028823E9
:10BC100031F021E04CE064E189E60E94C7332989D4
:10BC20003A89232BA1F41092EF0A29E04CE767E14F
:10BC300082E00E94C733F092EF0A33E03093060BA4
:10BC400040E24093070B85ED94E00E94364F8B89CC
:10BC50009C89892BA1F41092EF0A29E04CE762E25B
:10BC600082E00E94C733F092EF0A93E09093060BB4
:10BC7000EBE2E093070B85ED94E00E94364F2D89AF
:10BC80003E89232BA1F41092EF0A29E04CE76DE2E4
:10BC900082E00E94C733F092EF0A33E03093060B44
:10BCA00046E34093070B85ED94E00E94364F898D63
:10BCB0009A8D019709F068C080912008811190C584
:10BCC0001092EF0A29E046E061E082E30E94C73368
:10BCD00080912008882309F486C51092EF0A92E328
:10BCE0009093060BE9E0E093070B80911902909185
:10BCF0001A020E94564E498D5A8D4630510509F060
:10BD000075C080912008811180C51092EF0A21E052
:10BD10004CE066E189E30E94C733E98DFA8D3B97D9
:10BD200009F075C08091200881117EC51092EF0A3C
:10BD300021E04AE061E289E10E94C733298D3A8D12
:10BD40002031310509F075C08091200881117BC533
:10BD50001092EF0A21E04AE06CE289E10E94C733C9
:10BD6000498D5A8D4531510509F075C080912008E3
:10BD7000811178C51092EF0A21E04AE067E389E17A
:10BD800023C1988F8F8B47CD298D3A8D2230310575
:10BD9000E1F480912008882309F428C51092EF0A65
:10BDA00029E046E061E080E70E94C73380912008E7
:10BDB00081111FC51092EF0A30E73093060B49E05E
:10BDC0004093070B8F85988994CF898D9A8D03971F
:10BDD00009F051C08091200881110EC51092EF0A20
:10BDE00021E04BE066E18AE00E94C733898D9A8D9D
:10BDF000079709F051C080912008811109C5109260
:10BE0000EF0A21E04CE066E189E40E94C733298D06
:10BE10003A8D2C30310509F050C0809120088111F5
:10BE200006C51092EF0A21E04AE061E28BE20E942F
:10BE3000C733498D5A8D4131510509F050C0809169
:10BE40002008811103C51092EF0A21E04AE06CE25C
:10BE50008BE20E94C733898D9A8D469709F051C0B5
:10BE600080912008811101C51092EF0A21E04AE07B
:10BE700067E38BE2A9C0E98DFA8D349709F051C0D0
:10BE8000809120088111BBC41092EF0A21E04BE0A1
:10BE900066E18AE10E94C733E98DFA8D389709F08F
:10BEA0000CC1809120088111B6C41092EF0A21E0E4
:10BEB0004CE066E189E50E94C733298D3A8D2D302B
:10BEC000310509F00CC1809120088111B3C4109292
:10BED000EF0A21E04AE061E285E50E94C733498D1F
:10BEE0005A8D4231510509F00CC180912008811111
:10BEF000B0C41092EF0A21E04AE06CE285E50E94AE
:10BF0000C733898D9A8D479709F00CC1809120081D
:10BF10008111AEC41092EF0A21E04AE067E385E5A3
:10BF200053C0298D3A8D2530310509F0E4CE80913A
:10BF30002008811167C41092EF0A21E04BE066E10E
:10BF40008AE20E94C733498D5A8D4A30510509F063
:10BF5000E4CE80912008811164C41092EF0A89898F
:10BF60009A8921E042E1892B09F045E061E283E012
:10BF70000E94C733898D9A8D0F9709F0DFCE80918B
:10BF8000200881115DC41092EF0AEB89FC8921E041
:10BF900042E1EF2B09F045E06CE283E00E94C733F9
:10BFA000E98DFA8D749709F0DBCE8091200881111C
:10BFB00056C41092EF0A2D893E89232B09F0C2C086
:10BFC00021E042E167E383E00E94C733F092EF0A89
:10BFD0000E9425308111E5CC0E942423892B09F48D
:10BFE0002AC582E0809356091092220A61E08DE012
:10BFF0000E946E2B8091850890918608A0918708F9
:10C00000B09188088531FBE89F07F0E9AF07FEE0B3
:10C01000BF0709F078C4298D3A8D2130310509F028
:10C0200094C02091190230911A0221503109121640
:10C0300013060CF423C4498D5A8D50931A02409371
:10C040001902498D5A8D4630510509F09DC0209145
:10C050001502222309F428C110921502298D3A8D68
:10C060002B30310509F09CC031E0A31AB10818F457
:10C0700047E1A42EB12C298D3A8D2031310509F0EC
:10C08000A1C04F8158854150510958874F834F3F78
:10C090005F4F21F427E130E038872F83298D3A8DD7
:10C0A0002531310509F0A1C031E0231A310808F02B
:10C0B0002AC437E1232E312C26C4298D3A8D29300C
:10C0C000310509F040CF809120088111A7C310925B
:10C0D000EF0A21E04CE066E189E60E94C733498D12
:10C0E0005A8D4E30510509F045CF809120088111BD
:10C0F000A4C31092EF0A21E04AE061E287E60E94C1
:10C10000C733898D9A8D439709F04ACF80912008D3
:10C110008111A2C31092EF0A21E04AE06CE287E6A7
:10C120000E94C733E98DFA8D789709F04FCF80913F
:10C1300020088111A0C31092EF0A21E04AE067E3D2
:10C1400087E642CF21E045E03DCFE98DFA8D329779
:10C1500079F42F85388921503109388B2F871216B1
:10C1600013060CF46ECF41E050E0588B4F8769CF37
:10C17000E98DFA8D339709F086C3209118022223A6
:10C1800009F441C010921802E98DFA8D379709F031
:10C1900044C020911402222309F489C01092140291
:10C1A000E98DFA8D3C9709F045C029813A812150EB
:10C1B00031093A8329832F3F3F4F21F42BE330E0AD
:10C1C0003A832983298D3A8D2131310509F044C004
:10C1D00049855A85415051095A8749874F3F5F4FDA
:10C1E00021F44BE350E05A874987E98DFA8D769721
:10C1F00009F045C0F1E04F1A510808F084C32BE361
:10C20000422E512C80C3F0921802BECF209117020B
:10C21000222309F443C010921702298D3A8D283049
:10C22000310509F04AC020911302222309F442C0CB
:10C2300010921302E98DFA8D3D9709F04AC02B81C7
:10C240003C81215031093C832B832F3F3F4F21F408
:10C2500047E150E05C834B83298D3A8D22313105D3
:10C2600009F049C04B855C85415051095C874B877B
:10C270004F3F5F4F21F4E7E1F0E0FC87EB87498D0A
:10C280005A8D4731510509F049C051E0651A7108CE
:10C2900008F039C307E1602E712C35C3F092170204
:10C2A000BCCFF092160201C3F0921502D7CEF092E5
:10C2B000140276CFF0921302BDCF498D5A8D4930CA
:10C2C000510509F0F2C2209112022223B1F110921D
:10C2D0001202E98DFA8D3E9709F0F6C22D813E815A
:10C2E000215031093E832D832F3F3F4F21F4EBE353
:10C2F000F0E0FE83ED83298D3A8D2331310509F07D
:10C30000F2C24D855E85415051095E874D874F3F92
:10C310005F4F21F42BE330E03E872D87298D3A8D46
:10C320002831310509F0EFC231E0C31AD10808F015
:10C33000EAC21BE3C12ED12CE6C2F0921202C9CF91
:10C34000498D5A8D4230510509F040C0EF85F8897A
:10C350003196F88BEF87369724F025E030E0388B64
:10C360002F87298D3A8D26303105E1F52091150270
:10C37000222309F4BCC010921502E98DFA8D3B9777
:10C38000E9F5FFEFAF1ABF0A28E1A216B1040CF0DD
:10C390008EC3E98DFA8D7097F1F52F8138852F5F67
:10C3A0003F4F38872F83283131050CF08CC3E98D3E
:10C3B000FA8D7597F1F5FFEF2F1A3F0A28E1221643
:10C3C00031040CF400C3312C212CFDC2498D5A8D4F
:10C3D0004330510509F0B5C2209118022223D1F152
:10C3E00010921802498D5A8D47305105E9F5209178
:10C3F0001402222309F47EC010921402498D5A8D32
:10C400004C305105E9F5E981FA813196FA83E983E7
:10C41000FC970CF04FC3498D5A8D4131510509F0FD
:10C420003FC0E985FA853196FA87E987FC970CF0D9
:10C430004DC3498D5A8D4631510509F041C05FEF1A
:10C44000451A550AECE34E1651040CF4BCC2512CAB
:10C45000412CB9C2F0921802C5CF209117022223B5
:10C4600009F43FC010921702E98DFA8D389709F050
:10C4700047C020911302222309F43FC010921302F7
:10C48000298D3A8D2D30310509F046C04B815C81F4
:10C490004F5F5F4F5C834B83483151050CF00DC3F8
:10C4A000298D3A8D2231310509F045C04B855C85D7
:10C4B0004F5F5F4F5C874B87483151050CF009C3D4
:10C4C000298D3A8D2731310509F044C03FEF631AB9
:10C4D000730A48E1641671040CF475C2712C612C66
:10C4E00072C2F0921702C0CFF09216023CC2F092D4
:10C4F000150243CFF092140281CFF0921302C0CF05
:10C50000298D3A8D2930310509F02DC22091120272
:10C51000222381F110921202E98DFA8D3E9709F0E3
:10C5200032C22D813E812F5F3F4F3E832D832C33BE
:10C5300031050CF0C5C2E98DFA8D739709F033C24D
:10C540002D853E852F5F3F4F3E872D872C3331054C
:10C550000CF0C2C2E98DFA8D789709F034C2FFEF72
:10C56000CF1ADF0A2CE3C216D1040CF42CC2D12C52
:10C57000C12C29C2F0921202CFCFE98DFA8D7097AB
:10C5800041F42B893C89232B09F035C2E4E1F0E02A
:10C590000CC0498D5A8D4531510551F48D899E89C4
:10C5A000E1E0F0E0892B09F026C2FA8FE98F23C27F
:10C5B000298D3A8D2931310509F01DC221E030E085
:10C5C0003A8F298F18C285353BEC930730E9A307D2
:10C5D0003EE0B30779F5498D5A8D415051095A8F84
:10C5E000498F4E30510539F489899A89EAE0F0E0A3
:10C5F000892BD9F200C2298D3A8D2331310551F4AE
:10C600004B895C89452B09F0F6C18FE090E09A8F49
:10C61000898FF1C1E98DFA8DEF2B09F0ECC12D89DD
:10C620003E8944E150E0232B11F048E150E05A8F5D
:10C63000498FE1C184309A41A041BE4009F0DBC17D
:10C640000E94B03A019709F0C6C0809119029091FA
:10C650001A029C0121503109E29EF001E39EF00D87
:10C660001124EB58FD4F298920833B8931834D8963
:10C6700042835F855383A482298125833B8136834E
:10C680004D8147835F815087298521873B8532878C
:10C690004D854387248645866686C7862091180285
:10C6A000208B20911702218B20911602228B209142
:10C6B0001502238B20911402248B20911302258BC9
:10C6C00020911202268B019781F405E712E0912C4C
:10C6D000812CF80161918F01C4015CD8FFEF8F1AA2
:10C6E0009F0A27E182169104A1F780911902909187
:10C6F0001A02029789F40CE812E0F7E18F2E912CD0
:10C70000F80161918F01C40145D8FFEF8F1A9F0A8C
:10C710002EE282169104A1F78091190290911A02DB
:10C72000039789F403EA12E0EEE28E2E912CF801D1
:10C7300061918F01C4012ED8FFEF8F1A9F0A25E463
:10C7400082169104A1F78091190290911A02049720
:10C7500089F40AEB12E075E4872E912CF8016191BF
:10C760008F01C40117D8FFEF8F1A9F0A2CE582169C
:10C770009104A1F78091190290911A02059789F40A
:10C7800001ED12E06CE5862E912CF80161918F018C
:10C79000C40100D8FFEF8F1A9F0A23E78216910485
:10C7A000A1F78091190290911A02069791F408EE70
:10C7B00012E053E7852E912CF80161918F01C4019D
:10C7C0000E94CA5BFFEF8F1A9F0A2AE88216910423
:10C7D00099F70E945D4010921408992493940BC11C
:10C7E000F092EF0A6FCAF092EF0A79CAF092EF0A5C
:10C7F000D7CAF092EF0AE0CAF092EF0AF1CAF092BB
:10C80000EF0A44CBF092EF0A98CBF092EF0A7FCA7E
:10C81000F092EF0AF6CAF092EF0A49CBF092EF0AD3
:10C8200058CCF092EF0A9BCBF092EF0A81CAF092BB
:10C83000EF0AF9CAF092EF0A4CCBF092EF0A5BCC08
:10C84000F092EF0AA2CBF092EF0A84CAF092EF0ABC
:10C85000FCCAF092EF0A4FCBF092EF0A5DCCF09257
:10C86000EF0AA9CBF092EF0A87CAF092EF0AFECA4C
:10C87000F092EF0A51CBF092EF0A5FCC30931A029C
:10C8800020931902DECBE98DFA8D349709F4BECCE2
:10C89000298D3A8D2530310509F0D3CB2091160230
:10C8A000222309F4FECC10921602E98DFA8D3A97F4
:10C8B00009F0D4CB21E049895A89452B09F020E0C1
:10C8C000E22FF0E0FA8BE98BE98DFA8D3F9709F0C2
:10C8D000D2CB21E04B895C89452B09F020E0E22F87
:10C8E000F0E0FC8BEB8B298D3A8D2431310509F07A
:10C8F000D5CB21E04D895E89452B09F020E0E22F60
:10C90000F0E0FE8BED8B85395BE0950750E9A507DC
:10C910005EE0B50709F057C0E98DFA8D319709F04F
:10C920000FCD2091190230911A022F5F3F4F27300F
:10C93000310514F026E030E030931A0220931902FA
:10C9400010CD498D5A8D4430510509F486CDE98DBD
:10C95000FA8D359709F005CD20911602222309F4AE
:10C96000C3CD10921602498D5A8D4A30510509F0F7
:10C9700004CD21E0E989FA89EF2B09F020E0422F6C
:10C9800050E05A8B498B498D5A8D4F30510509F033
:10C9900000CD21E0EB89FC89EF2B09F020E0422F4C
:10C9A00050E05C8B4B8B498D5A8D4431510509F019
:10C9B000FECC21E0ED89FE89EF2B09F020E0422F2B
:10C9C00050E05E8B4D8B853D3BE4930730E9A30738
:10C9D0003EE0B30709F0F7CD498D5A8D4F5F5F4FA9
:10C9E0005A8F498F4B30510509F0C7CD89899A89F3
:10C9F000892B09F40ACE8091850890918608A09130
:10CA00008708B091880884379A46A041BE4021F437
:10CA1000109214089924939464E670E080E090E00A
:10CA20000E94F52D82E0809356091092220A60E060
:10CA30008DE00E946E2B0E94994E8091EC06813011
:10CA400011F08B3021F41092140899249394809162
:10CA5000190290911A02EF89F88D8E179F0709F03D
:10CA600090C960E08DE00E946E2B992011F40C9427
:10CA7000B45C6CE271E080E090E06A960FB6F894E6
:10CA8000DEBF0FBECDBFDF91CF911F910F91FF9001
:10CA9000EF90DF90CF90BF90AF909F908F907F905E
:10CAA0006F905F904F903F902F900C94F52DB12C8C
:10CAB000A12C6FCC1A821982AECC1C821B82F0CCC6
:10CAC0001E821D8238CD18861F8271CC1A86198667
:10CAD000B0CC1C861B86F4CC1E861D863BCD2F92C7
:10CAE0003F924F925F926F927F928F929F92AF92FE
:10CAF000BF92CF92DF92EF92FF920F931F93CF934B
:10CB0000DF93CDB7DEB765970FB6F894DEBF0FBEE3
:10CB1000CDBF10922C0810922B0860E08DE00E948F
:10CB20006E2B21E0298780910503811101C01986B0
:10CB300080910603882E912C80910703482E512C5A
:10CB400080910803E82FF0E0FA83E98380910903DC
:10CB5000282F30E03C832B83E0900A03F12CC09017
:10CB60000B03D12C6624639480910C03811101C0C6
:10CB7000612C20900D03312C80910E03E82FF0E002
:10CB8000FE83ED83A0900F03B12C80911003282F1A
:10CB900030E038872F8381E090E09D8B8C8B772469
:10CBA0007394EAE1EE9DC001EF9D900D112464E6BF
:10CBB00070E00E946F8F688B798B6E87EC9DC0014F
:10CBC000ED9D900D112464E670E00E946F8F6A8BDA
:10CBD0007B8B6F873985232F30E03B872A87862D13
:10CBE00090E09D878C8780912B0890912C0801966E
:10CBF00090932C0880932B08029754F08091200882
:10CC000091E089278093200810922C0810922B081D
:10CC10007092EF0A04EE14E020E440E860E080E067
:10CC20000E94E9331092EF0A8EEE9AE30E94FA28EE
:10CC3000E4E4E093060BF9E0F093070B8A859B850B
:10CC40000E94564E7092EF0A2EE62093060B38E2B1
:10CC50003093070B8C859D850E94564E88E180930A
:10CC6000060B94E19093070BEAE08E16910424F4EE
:10CC700083ED94E00E94364FC4010E94564E89EB2A
:10CC800094E00E94364FFAE04F16510424F483EDED
:10CC900094E00E94364FC2010E94564E7092EF0AF5
:10CCA00024E52093060B34E13093070B89819A81A8
:10CCB0000A9724F483ED94E00E94364F89819A818B
:10CCC0000E94564E89EB94E00E94364FEB81FC8126
:10CCD0003A9724F483ED94E00E94364F8B819C8137
:10CCE0000E94564E87E892E20E94FA28FAE0EF1678
:10CCF000F1040CF0A4C024E32093060B3CE1309334
:10CD0000070BC7010E94564EE889E093E906F989AE
:10CD1000F093EA0623E04E8568E184E10E94C73380
:10CD20002AE0C216D1040CF091C086E78093060B6E
:10CD30003CE13093070BC6010E94564E9A899093AE
:10CD4000E906EB89E093EA0623E04F8568E184E594
:10CD50000E94C7338EEE9AE30E94FA28F8E1F0931E
:10CD6000060B24E32093070BC1010E94564E80EC72
:10CD700094E00E94364F8D819E810E94564E89ED2F
:10CD800094E00E94364F8EEE9AE30E94FA2834E532
:10CD90003093060B84E38093070BC5010E94564E27
:10CDA00080EC94E00E94364F8F8198850E94564E09
:10CDB00089ED94E00E94364FEC89FD89319709F0A6
:10CDC0004CC080912008811153C31092EF0A29E0D2
:10CDD00046E061E084E40E94C73380912008882304
:10CDE00009F449C31092EF0AF4E4F093060B29E02A
:10CDF0002093070B8A859B850E94564EEC89FD89FE
:10CE0000369709F04BC080912008811143C31092DE
:10CE1000EF0A21E04FE06DE182E00E94C733EC8928
:10CE2000FD893B9709F04BC080912008811144C3D4
:10CE30001092EF0A21E04BE065E385E509C180E34C
:10CE40008093060B9CE19093070B5BCF80E7809368
:10CE5000060B8CE18093070B6ECF8C899D8902971E
:10CE600069F480912008811109C31092EF0A21E032
:10CE70004AE065E189E10E94C733C0CFEC89FD89B2
:10CE8000339771F5809120088111FBC21092EF0A4F
:10CE900021E04AE065E18BE20E94C7332C893D899D
:10CEA0002730310579F5809120088111F6C2109262
:10CEB000EF0A21E04FE06DE181E40E94C7332C8945
:10CEC0003D892C30310509F03FC080912008811147
:10CED000F6C21092EF0A21E046E065E385E6B8C0AD
:10CEE0002C893D892430310509F082C080912008C9
:10CEF0008111CAC21092EF0A21E04AE065E185E59E
:10CF00000E94C7338C899D89089709F092C080914F
:10CF100020088111C5C21092EF0A29E046E060E2C4
:10CF20008EE60E94C73380912008882309F4BBC293
:10CF30001092EF0A9EE69093060BE8E2E093070B4F
:10CF40008C859D850E94564E7092EF0A0E94253076
:10CF500081115ECE0E942423892B09F444CE82E005
:10CF6000809356091092220A61E08DE00E946E2B98
:10CF70008091850890918608A0918708B0918808D3
:10CF800085319B48A049BE4009F0BDC08C899D8970
:10CF9000019709F060C09985972599872C893D896B
:10CFA0002630310509F06FC031E0E31AF10810F4C2
:10CFB000F12CE12C2FEF2E9DC0012F9D900D1124FF
:10CFC00064E670E00E946F8F87E00E94D72B8C8907
:10CFD0009D890B9709F06EC091E0A91AB108E4E1B0
:10CFE000AE16B1040CF08FC054E1A52EB12C8BC04D
:10CFF0008C899D89059709F001CF809120088111C6
:10D0000046C21092EF0A21E04AE065E187E60E94FD
:10D01000C7338C899D890A9709F001CF8091200838
:10D02000811147C21092EF0A21E046E065E389E2F0
:10D030000FC02C893D892930310559F7809120088E
:10D04000811134C21092EF0A21E04AE065E389E1E0
:10D050000E94C73379CFEC89FD89329749F4F1E01A
:10D060008F1A910808F09ACF97E1892E912C96CFCC
:10D070008C899D89039779F591E0491A510818F434
:10D080008BE3482E512CEC89FD893797A9F5F1E007
:10D09000CF1AD10810F4D12CC12C2FEF2C9DC00138
:10D0A0002D9D900D112464E670E00E946F8F87E043
:10D0B0000E94D72B2C893D892C30310521F58F8199
:10D0C0009885019798878F830196E9F429E030E0ED
:10D0D00038872F8318C02C893D892430310509F009
:10D0E00056C089819A8101979A838983019621F498
:10D0F00027E130E03A8329838C899D89089709F0DC
:10D1000069C091E069268091850890918608A09178
:10D110008708B091880885399B40A049BE4009F036
:10D12000C1C08C899D89019709F064C09985E1E0AF
:10D130009E279987EC89FD89369709F077C0FFEF24
:10D14000EF1AFF0A25E6E216F1041CF044E6E42E8D
:10D15000F12C2FEF2E9DC0012F9D900D112464E620
:10D1600070E00E946F8F87E00E94D72BEC89FD89C9
:10D170003B9709F076C0FFEFAF1ABF0AA214B304C1
:10D180000CF490C0510121E0A21AB1088BC02C8987
:10D190003D892530310509F001CF8B819C810197B4
:10D1A0009C838B83019621F48BE390E09C838B839B
:10D1B0008C899D890A9709F00ACFED81FE8131970C
:10D1C000FE83ED83319609F09ECFE9E0F0E0FE8327
:10D1D000ED8399CFEC89FD89399751F7F1E02F1A4A
:10D1E0003108A214B3040CF48ECF15012FEF221ACC
:10D1F000320A89CF2C893D892230310559F43FEF1D
:10D20000831A930A88E1881691040CF493CF912C29
:10D21000812C90CFEC89FD89339789F5FFEF4F1A68
:10D220005F0A2CE3421651040CF04CC18C899D8995
:10D23000079789F59FEFC91AD90AE5E6CE16D104FA
:10D240001CF034E6C32ED12C2FEF2C9DC0012D9D58
:10D25000900D112464E670E00E946F8F87E00E94B9
:10D26000D72B8C899D890C97E9F4EF81F88531964D
:10D27000F887EF833A97B4F018861F8213C08C8921
:10D280009D89049759F5E981FA813196FA83E983FA
:10D2900078970CF01AC12C893D8928303105E1F5C9
:10D2A00031E063268091850890918608A0918708D7
:10D2B000B0918808853DFBE49F07F0E9AF07FEE0E9
:10D2C000BF07D1F52C893D892F5F3F4F3D8B2C8BBC
:10D2D0002D30310509F4FFC010E08BC02C893D8949
:10D2E0002530310509F026CF8B819C8101969C83E6
:10D2F0008B83CC970CF0ECC02C893D892A3031050A
:10D3000009F034CF8D819E8101969E838D830A978B
:10D310004CF21E821D82C6CF8C899D89099761F7C8
:10D320009FEF291A390AE4E22E1631040CF4BACF21
:10D3300023E2222E312CB6CF85353BEC930730E922
:10D34000A3073EE0B30761F48C899D8901979D8B0B
:10D350008C8B892B09F6ECE0F0E0FD8BEC8BBCCFDD
:10D3600084309A41A041BE4009F0B6CF0E94B03A45
:10D370000197B1F529852093050380920603409219
:10D3800007033981309308038B8180930903E0926E
:10D390000A03C0920B0360920C0320920D039D813F
:10D3A00090930E03A0920F03EF81E093100325E00A
:10D3B00033E03B872A8702EE10E0EA85FB85619126
:10D3C000FB87EA87C8010E94CA5B0F5F1F4F0E3EB2
:10D3D000110599F764EF71E080E090E00E94F52D6F
:10D3E0001092110810921708109216080E945D40C2
:10D3F00011E08091850890918608A0918708B091EE
:10D40000880884379A46A041BE4039F4109211082A
:10D41000109217081092160811E064E670E080E0A0
:10D4200090E00E94F52D82E0809356091092220A26
:10D4300060E08DE00E946E2B112309F4B2CB65965B
:10D440000FB6F894DEBF0FBECDBFDF91CF911F9115
:10D450000F91FF90EF90DF90CF90BF90AF909F9093
:10D460008F907F906F905F904F903F902F90089596
:10D470007092EF0AACCC7092EF0AB6CC7092EF0AC1
:10D48000F6CC7092EF0A04CD7092EF0A35CD70920F
:10D49000EF0AB9CD7092EF0ABCCC7092EF0A09CDB9
:10D4A0007092EF0A3ACD7092EF0A44CD7092EF0A73
:10D4B000CBCD7092EF0AB8CD7092EF0ABBCC7092D0
:10D4C000EF0A09CD512C412CB1CE1A821982E3CE3C
:10D4D0001C821B8211CF21E030E03D8B2C8BFCCED7
:10D4E0002F923F924F925F926F927F928F929F9274
:10D4F000AF92BF92CF92DF92EF92FF920F931F9362
:10D50000CF93DF93CDB7DEB7A5970FB6F894DEBF04
:10D510000FBECDBF20910802309109023F8B2E8BA8
:10D5200010922C0810922B0841E050E05DA34CA310
:10D530001D8A96E1E92EFF24F394809108029091D0
:10D5400009020197E89EF001E99EF00D1124E35EC7
:10D55000FD4F2081422F50E05A8B498B2181422F71
:10D5600050E05C8B4B8B2281422F50E0588B4F87D1
:10D570002381222E312C2481422F50E05A8349836B
:10D580002581422F50E05C834B832681422F50E05F
:10D590005E834D832781422F50E058874F8320853B
:10D5A000422F50E05A8749872185422F50E05C87FF
:10D5B0004B872285422F50E05E874D874384512C54
:10D5C0006484712CC584D12CA684B12C21E03785CC
:10D5D000311101C020E020931802E89EF001E99E7D
:10D5E000F00D1124E35EFD4F21E03089311101C0BF
:10D5F00020E020931702E89EF001E99EF00D11242F
:10D60000E35EFD4F21E03189311101C020E020931C
:10D610001602E89EF001E99EF00D1124E35EFD4F35
:10D6200021E03289311101C020E020931502E89EEB
:10D63000F001E99EF00D1124E35EFD4F21E03389F6
:10D64000311101C020E020931402E89EF001E99E10
:10D65000F00D1124E35EFD4F21E03489311101C04A
:10D6600020E020931302E89EF001E99EF00D1124C2
:10D67000E35EFD4F81E09589911101C080E08093C8
:10D68000120264E670E080E090E00E94F52D809147
:10D690002B0890912C08019690932C0880932B08CE
:10D6A000029754F08091200851E08527809320084C
:10D6B00010922C0810922B080E94F52F2AE1249D2D
:10D6C000C001259D900D112464E670E00E946F8FCB
:10D6D0006C8F7D8F688F269DC001279D900D112432
:10D6E0006CE370E00E946F8F6E8F7F8F698F2C9D2F
:10D6F000C0012D9D900D112464E670E00E946F8F93
:10D7000068A379A36A8F2A9DC0012B9D900D1124D7
:10D710006CE370E00E946F8F6AA37BA36B8F09E0BC
:10D72000902E8FE1882EF092EF0A04EE10E020E4B4
:10D7300040E860E080E00E94E9338EEE9AE30E94C8
:10D74000FA2882E38093060B9092070B80910802DF
:10D75000909109020E94564E1092EF0A95E790931D
:10D76000060B9092070B8F8598890E94564EF09277
:10D77000EF0AE8E1E093060B8092070BFAE02F1620
:10D78000310424F483ED94E00E94364FC1010E94DD
:10D79000564E89EB94E00E94364F29813A812A3017
:10D7A000310524F483ED94E00E94364F89819A81FB
:10D7B0000E94564EF092EF0A34E53093060B8092A9
:10D7C000070B4B815C814A30510524F483ED94E0D2
:10D7D0000E94364F8B819C810E94564E89EB94E0CB
:10D7E0000E94364F8D819E810A9724F483ED94E048
:10D7F0000E94364F8D819E810E94564E87E892E2AC
:10D800000E94FA289AE0491651040CF08FC1E4E313
:10D81000E093060BF7E2F093070BC2010E94564E0D
:10D820004C8D4093E9065D8D5093EA0623E0488DC8
:10D8300063E280E10E94C7338AE0681671040CF04D
:10D840007CC19CE69093060BE7E2E093070BC301D3
:10D850000E94564E3E8D3093E9064F8D4093EA0666
:10D8600023E0498D63E28AE40E94C7335AE0C5167B
:10D87000D1040CF069C184E38093060B88E38093A4
:10D88000070BC6010E94564EE8A1E093E906F9A1F4
:10D89000F093EA0623E04A8D64E380E10E94C733F7
:10D8A0002AE0A216B1040CF053C13CE63093060BFB
:10D8B00088E38093070BC5010E94564E5AA15093EE
:10D8C000E9068BA18093EA0623E04B8D64E38AE4AA
:10D8D0000E94C7338EEE9AE30E94FA2898E1909353
:10D8E000060BE0E3E093070B2F8138852A303105E2
:10D8F00024F483ED94E00E94364F8F8198850E9436
:10D90000564E89EB94E00E94364F49855A854A303D
:10D91000510524F483ED94E00E94364F89859A8561
:10D920000E94564EF092EF0A54E55093060B80E3A6
:10D930008093070BEB85FC853A9724F483ED94E004
:10D940000E94364F8B859C850E94564E89EB94E051
:10D950000E94364F2D853E852A30310524F483ED13
:10D9600094E00E94364F8D859E850E94564E809190
:10D970001802882331F021E04BE064E18AE00E9444
:10D98000C73380911702882331F021E04BE064E136
:10D990008AE10E94C73380911602882331F021E08A
:10D9A0004BE064E18AE20E94C7338091150288232C
:10D9B00031F021E04CE064E189E30E94C7338091BB
:10D9C0001402882331F021E04CE064E189E40E94F4
:10D9D000C73380911302882331F021E04CE064E1E9
:10D9E00089E50E94C73380911202882331F021E03B
:10D9F0004CE064E189E60E94C73349895A89452B86
:10DA000099F41092EF0A23E14CE766E182E00E946C
:10DA1000C733F092EF0A83E08093060B8092070BE6
:10DA200085ED94E00E94364F8B899C89892BA1F467
:10DA30001092EF0A20E14CE769E282E00E94C733CE
:10DA4000F092EF0A83E08093060B81E38093070B4B
:10DA500085ED94E00E94364FECA1FDA1319709F0CD
:10DA60007BC0809120088111C4C51092EF0A29E083
:10DA700046E061E082E30E94C7338091200888235A
:10DA800009F4BAC51092EF0AF2E3F093060B9092F4
:10DA9000070B80910802909109020E94564E2CA11A
:10DAA0003DA12630310509F089C0809120088111FF
:10DAB000B5C51092EF0A21E04CE066E189E30E94CF
:10DAC000C7338CA19DA10B9709F08AC080912008D3
:10DAD0008111B3C51092EF0A21E04AE060E289E1CA
:10DAE0000E94C7338CA19DA1409709F08AC0809104
:10DAF00020088111B1C51092EF0A21E045E067E2EC
:10DB000083E40E94C733ECA1FDA1759709F08FC093
:10DB1000809120088111AFC51092EF0A21E04AE000
:10DB200061E387E667C19F8B8E8B07CD2EE2209342
:10DB3000060B37E23093070B70CEF7E6F093060B37
:10DB400027E22093070B83CE9EE29093060B96CE9E
:10DB500047E64093060BACCE2CA13DA12230310507
:10DB6000D9F480912008882309F449C51092EF0A5E
:10DB700029E046E061E085E70E94C73380912008F4
:10DB8000811140C51092EF0A35E73093060B909251
:10DB9000070B8F85988981CF4CA15DA1433051053A
:10DBA00009F056C08091200881112FC51092EF0A0C
:10DBB00021E04BE066E18AE00E94C7334CA15DA101
:10DBC0004730510509F055C080912008811129C5C1
:10DBD0001092EF0A21E04CE066E189E40E94C7332D
:10DBE000ECA1FDA13C9709F055C08091200881115E
:10DBF00027C51092EF0A21E04AE060E28BE20E9422
:10DC0000C733ECA1FDA1719709F056C0809120089F
:10DC1000811125C51092EF0A2B893C89232B09F02D
:10DC200061C121E042E162E383E00E94C7332CA19D
:10DC30003DA12631310509F051C0809120088111A4
:10DC40001DC51092EF0A21E04AE068E382E0D2C0ED
:10DC50008CA19DA1049709F052C0809120088111E8
:10DC6000D7C41092EF0A21E04BE066E18AE10E94FE
:10DC7000C7338CA19DA1089709F08CC08091200822
:10DC80008111D2C41092EF0A21E04CE066E189E5EF
:10DC90000E94C7332CA13DA12D30310509F08BC066
:10DCA000809120088111CFC41092EF0A21E04AE050
:10DCB00060E285E50E94C7334CA15DA14231510568
:10DCC00009F08AC0809120088111CCC41092EF0A1B
:10DCD00021E04AE061E389E10E94C7334CA15DA1E4
:10DCE0004731510509F088C0809120088111C9C4CD
:10DCF0001092EF0A21E045E068E383E47BC0ECA1E9
:10DD0000FDA1359709F0CBCE80912008811183C405
:10DD10001092EF0A21E04BE066E18AE20E94C733ED
:10DD20002CA13DA12A30310509F0CBCE80912008ED
:10DD3000811180C41092EF0A49895A8921E0452B4C
:10DD400009F0CEC042E160E283E00E94C7334CA1FB
:10DD50005DA14F30510509F0C5CE80912008811199
:10DD600078C41092EF0A21E04AE067E282E00E9464
:10DD7000C7334CA15DA14431510509F0C4CE809157
:10DD80002008811175C41092EF0A21E04AE061E396
:10DD900085E530C0ECA1FDA1399709F0C1CF809194
:10DDA0002008811144C41092EF0A21E04CE066E1A2
:10DDB00089E60E94C7332CA13DA12E30310539F6EA
:10DDC00080912008811142C41092EF0A21E04AE0BC
:10DDD00060E287E60E94C7338CA19DA1439749F674
:10DDE00080912008811141C41092EF0A21E04AE09D
:10DDF00061E38BE20E94C733F092EF0A0E94253064
:10DE0000811191CC0E942423892B09F4C4C282E0A1
:10DE1000809356091092220A61E08DE00E946E2BD9
:10DE20008091850890918608A0918708B091880814
:10DE300085315BE8950750E9A5075EE0B50709F075
:10DE4000B0C0ECA1FDA1E130F10509F04FC0209177
:10DE500008023091090221503109121613060CF400
:10DE600013C4F0930902E0930802ECA1FDA13697D8
:10DE700009F05DC020911502222309F400C110921F
:10DE800015022CA13DA12B30310509F05DC031E018
:10DE9000231A310818F427E1222E312C4CA15DA160
:10DEA0004031510509F062C055E0651A710877FEEE
:10DEB00002C0712C612C2CA13DA12531310509F046
:10DEC00064C04D855E85415051095E874D874F3F47
:10DED0005F4F09F066C02BE330E03E872D8761C0BD
:10DEE00045E031CF21E045E061E39ECE2CA13DA18C
:10DEF0002230310579F44F85588941505109588BAA
:10DF00004F87141615060CF4B0CFE1E0F0E0F88B63
:10DF1000EF87ABCF2CA13DA12330310509F0B9C368
:10DF200020911802222309F45BC0109218022CA140
:10DF30003DA12730310509F05DC020911402222354
:10DF400009F4A0C010921402ECA1FDA13C9709F0C5
:10DF50005EC029813A81215031093A8329832F3FBC
:10DF60003F4F21F42BE330E03A832983ECA1FDA15C
:10DF7000719709F05EC021E04B895C89452B09F05F
:10DF800020E0E22FF0E0FC8BEB8B2CA13DA12631B1
:10DF9000310509F061C031E0C31AD10810F4D12C69
:10DFA000C12C85392BE0920720E9A2072EE0B207A9
:10DFB00009F0B9C14CA15DA14130510509F09DC0E6
:10DFC00020910802309109022F5F3F4F2530310523
:10DFD00014F024E030E030930902209308029FC03F
:10DFE000F0921802A4CF20911702222309F441C015
:10DFF000109217024CA15DA14830510509F048C0AC
:10E0000020911302222309F440C010921302ECA1C4
:10E01000FDA13D9709F047C02B813C81215031097A
:10E020003C832B832F3F3F4F21F447E150E05C833B
:10E030004B832CA13DA12231310509F046C04F810F
:10E0400058854150510958874F834F3F5F4F21F406
:10E0500027E130E038872F83ECA1FDA1779709F005
:10E06000A0CFF5E0AF1AB108B7FE9BCFB12CA12C21
:10E0700098CFF0921702BECFF09216021CC3F09216
:10E080001502FFCEF09214025FCFF0921302BFCFC1
:10E09000ECA1FDA1399709F00EC3209112022223B1
:10E0A00049F110921202ECA1FDA13E9709F013C3B1
:10E0B0002D813E81215031093E832D832F3F3F4FDB
:10E0C00021F4EBE3F0E0FE83ED832CA13DA12331AD
:10E0D000310509F00BC349855A85415051095A87CA
:10E0E00049874F3F5F4F09F05CCF4BE350E05A87C1
:10E0F000498757CFF0921202D6CFECA1FDA13297FB
:10E1000009F04BC02F8538892F5F3F4F388B2F8701
:10E110002530310524F044E050E0588B4F874CA166
:10E120005DA14630510509F043C02091150222231C
:10E1300009F4C4C0109215022CA13DA12B30310569
:10E1400009F042C03FEF231A330A48E12416310494
:10E150000CF023C34CA15DA14031510509F043C02F
:10E1600055E0650E711CEDE36E1671041CF0FCE3C6
:10E170006F2E712C2CA13DA12531310509F042C033
:10E180004D855E854F5F5F4F5E874D874C335105F0
:10E190000CF4C9C01E861D86C6C0ECA1FDA1339734
:10E1A00009F0B9C2209118022223E9F11092180255
:10E1B000ECA1FDA1379709F03FC020911402222362
:10E1C00009F47FC010921402ECA1FDA13C9709F064
:10E1D0003FC029813A812F5F3F4F3A8329832C33F7
:10E1E00031050CF0DDC22CA13DA121313105F1F545
:10E1F00021E04B895C89452B09F020E0E22FF0E01B
:10E20000FC8BEB8BECA1FDA1769709F03FC0FFEFF3
:10E21000CF1ADF0A25E6C216D1040CF484C0E4E666
:10E22000CE2ED12C80C0F0921802C2CF20911702BE
:10E230002223F1F1109217022CA13DA128303105C3
:10E2400009F045C0209113022223F1F1109213022C
:10E250004CA15DA14D30510509F046C0EB81FC8118
:10E260003196FC83EB8378970CF09DC22CA13DA1E5
:10E270002231310509F048C04F8158854F5F5F4F0B
:10E2800058874F83483151050CF093C24CA15DA1D2
:10E290004731510509F047C055E0A50EB11CEDE32B
:10E2A000AE16B1040CF43FC07CE3A72EB12C3BC0EA
:10E2B000F0921702C1CFF092160240C2F0921502FE
:10E2C0003BCFF092140280CFF0921302C1CF4CA149
:10E2D0005DA14930510509F031C22091120222237B
:10E2E00009F497C0109212022CA13DA12E303105E5
:10E2F00009F033C24D815E814F5F5F4F5E834D8376
:10E300004C3351050CF052C2ECA1FDA1739709F0FA
:10E3100033C229853A852F5F3F4F3A8729872C33AF
:10E3200031050CF049C2853DFBE49F07F0E9AF07DA
:10E33000FEE0BF0709F089C02CA13DA12F5F3F4F30
:10E340003DA32CA32B30310509F066C049895A89B9
:10E35000452B09F48FC08091850890918608A09183
:10E360008708B091880884379A46A041BE4021F4BE
:10E370001092140881E08D8B64E670E080E090E0FC
:10E380000E94F52D82E0809356091092220A60E0E7
:10E390008DE00E946E2B0E94994E8091EC06813098
:10E3A00011F08B3021F41092140891E09D8B809134
:10E3B000080290910902EE89FF898E179F0709F0E4
:10E3C000B2CB60E08DE00E946E2BFD89FF2309F443
:10E3D00058C9109212086CE271E080E090E0A596B6
:10E3E0000FB6F894DEBF0FBECDBFDF91CF911F9166
:10E3F0000F91FF90EF90DF90CF90BF90AF909F90E4
:10E400008F907F906F905F904F903F902F900C94E3
:10E41000F52DF092120268CF8CA19DA1429751F484
:10E42000EB89FC89EF2B09F096CF21E030E03DA38A
:10E430002CA391CF4CA15DA181E090E04831510522
:10E4400009F089CF9DA38CA386CF8535EBEC9E0781
:10E45000E0E9AE07EEE0BE07F9F42CA13DA12150A2
:10E4600031093DA32CA3232B41F44B895C89452B17
:10E4700009F0BCC081E190E0E5CFECA1FDA170976F
:10E4800009F069CF29893A894AE050E0232B09F045
:10E4900062CF5DA34CA35FCF84309A41A041BE40C0
:10E4A00009F059CF0E94B03A019709F09AC08091C3
:10E4B0000802909109029C0121503109E29EF0016D
:10E4C000E39EF00D1124E35EFD4F298920833B89F3
:10E4D00031834F8542832382598154832B81258345
:10E4E0003D8136834F814783598550872B8521870E
:10E4F0003D85328743866486C586A68620911802AC
:10E50000278720911702208B20911602218B2091C2
:10E510001502228B20911402238B20911302248B4D
:10E5200020911202258B019791F40DE112E06AE827
:10E53000862E912CF80161918F01C4010E94CA5B63
:10E54000FFEF8F1A9F0A20EA8216910499F78091B3
:10E55000080290910902029791F403E312E050EA55
:10E56000852E912CF80161918F01C4010E94CA5B34
:10E57000FFEF8F1A9F0A26EB8216910499F780917C
:10E58000080290910902039791F409E412E046EB26
:10E59000842E912CF80161918F01C4010E94CA5B05
:10E5A000FFEF8F1A9F0A2CEC8216910499F7809145
:10E5B000080290910902049791F40FE512E03CECF7
:10E5C000832E912CF80161918F01C4010E94CA5BD6
:10E5D000FFEF8F1A9F0A22EE8216910499F70E948C
:10E5E000A24C1092140831E03D8BB5CE47E150E0CB
:10E5F00050CFF092EF0A3BCAF092EF0A45CAF09270
:10E60000EF0AB6CAF092EF0ABFCAF092EF0AD0CA78
:10E61000F092EF0A28CBF092EF0A7CCBF092EF0A4F
:10E620004ACAF092EF0AD6CAF092EF0A2DCBF092C6
:10E63000EF0ABBCBF092EF0A7FCBF092EF0A4CCA05
:10E64000F092EF0AD8CAF092EF0A30CBF092EF0ABC
:10E65000BDCBF092EF0A87CBF092EF0A4ECAF09250
:10E66000EF0ADACAF092EF0A33CBF092EF0ABECB90
:10E67000F092EF0A8ACBF092EF0A50CAF092EF0ABA
:10E68000E2CAF092EF0A36CB3093090220930802D7
:10E69000ECCBECA1FDA1349709F4A5CC4CA15DA174
:10E6A0004530510509F0E1CB20911602222309F4EF
:10E6B000E3CC109216022CA13DA12A30310509F0BD
:10E6C000E0CB21E049895A89452B09F020E0E22F6F
:10E6D000F0E0FA8BE98BECA1FDA13F9709F0DECBCE
:10E6E000F1E04F1A510810F4512C412C2CA13DA1FE
:10E6F0002431310509F0DFCB4B855C854150510950
:10E700005C874B874F3F5F4F09F04BCCE7E1F0E070
:10E71000FC87EB8746CC4CA15DA14430510509F440
:10E7200085CD2CA13DA12530310509F0F8CC2091F3
:10E730001602222309F4BFCD10921602ECA1FDA10E
:10E740003A9709F0F9CC21E049895A89452B09F01B
:10E7500020E0E22FF0E0FA8BE98BECA1FDA13F97DE
:10E7600009F0F8CCFFEF4F1A5F0A25E64216510474
:10E770001CF014E6412E512C4CA15DA144315105F1
:10E7800009F0F8CCEB85FC853196FC87EB87789710
:10E790000CF4C9CD1C861B86C6CD312C212CDACCBD
:10E7A0001A82198220CD1C821B8260CD1E821D829E
:10E7B000ABCD18861F826ACD1A861986B4CD1F92FA
:10E7C0000F920FB60F9211240BB60F922F933F9317
:10E7D0004F935F936F937F938F939F93AF93BF9369
:10E7E000EF93FF938FE998E00E94E729FF91EF9163
:10E7F000BF91AF919F918F917F916F915F914F9159
:10E800003F912F910F900BBE0F900FBE0F901F9056
:10E8100018951F920F920FB60F9211240BB60F92FC
:10E820002F938F939F93EF93FF93E091AF08F09115
:10E83000B0088081E091B508F091B60882FD1DC056
:10E8400090818091B8088F5F8F732091B9088217EB
:10E8500041F0E091B808F0E0E156F74F958F8093D2
:10E86000B808FF91EF919F918F912F910F900BBE60
:10E870000F900FBE0F901F9018958081F2CF1F92BE
:10E880000F920FB60F9211242F933F938F939F9364
:10E89000AF93BF9380918F0890919008A0919108B9
:10E8A000B09192083091650723E0230F2D3758F57A
:10E8B0000196A11DB11D2093650780938F08909349
:10E8C0009008A0939108B093920880916607909168
:10E8D0006707A0916807B09169070196A11DB11D56
:10E8E0008093660790936707A0936807B0936907C2
:10E8F000BF91AF919F918F913F912F910F900FBE3C
:10E900000F901F90189526E8230F0296A11DB11DA8
:10E91000D2CF1F920F920FB60F9211240BB60F9207
:10E920002F933F934F935F936F937F938F939F9317
:10E93000AF93BF93EF93FF93809155090E94462BAD
:10E9400020915809309159092F5F3F4F3093590951
:10E95000209358099091220A943618F095E09093EC
:10E96000560990915609933009F44CC0E0F4923066
:10E9700011F190915709992319F081116BC02F9AC9
:10E98000FF91EF91BF91AF919F918F917F916F9187
:10E990005F914F913F912F910F900BBE0F900FBE43
:10E9A0000F901F901895943009F448C0953009F7DE
:10E9B0008111DFCF09C08111DCCF2091580930913E
:10E9C00059092436310528F4109259091092580932
:10E9D000D0CF1092220AE091220A91E09E0F9093EC
:10E9E000220AF0E02091580930915909EE0FFF1FDB
:10E9F000EB5AF64F36832583109259091092580925
:10EA000093E019C0813009F0B4CFE091220A91E07F
:10EA10009E0F9093220AF0E02091580930915909F5
:10EA2000EE0FFF1FEB5AF64F3683258310925909DC
:10EA30001092580994E0909356099BCF882359F27D
:10EA400020915809309159092536310508F491CFA4
:10EA500095E0F1CF2F9894CF1F920F920FB60F929F
:10EA600011240BB60F922F933F934F935F936F93A5
:10EA70007F938F939F93AF93BF93EF93FF93809177
:10EA8000B900887F803609F44DC008F040C0883254
:10EA900009F4A9C028F5803109F49DC0C8F4882381
:10EAA00009F4FBC0883009F496C0FF91EF91BF9143
:10EAB000AF919F918F917F916F915F914F913F9116
:10EAC0002F910F900BBE0F900FBE0F901F901895B7
:10EAD000883109F488C0803241F78093550814C00A
:10EAE000803409F49DC040F48033B9F38833E9F6EB
:10EAF0008093550885ECB0C0803509F485C0883511
:10EB000009F496C0883489F60E94925BCECF88398A
:10EB100009F48CC038F5883729F050F4883611F0A4
:10EB2000803719F683E08093570810923B0757C04F
:10EB3000883809F47BC0803919F0803809F0B5CFE6
:10EB400080913B07803208F071C0E0913B0781E083
:10EB50008E0F80933B078091BB00F0E0E55EF84F9D
:10EB600080833DC0803B39F0E0F4803A09F479C0FD
:10EB7000883A09F09ACF84E08093570810921A07D8
:10EB800010921907E0916D07F0916E071995809129
:10EB9000190781110FC081E0809319071092F906BF
:10EBA00009C0803C09F4A6CF883C09F4A3CF883B78
:10EBB00009F07BCFE0911A0781E08E0F80931A074E
:10EBC000F0E0E750F94F80818093BB0090911A07E5
:10EBD0008091190729C0809132088093BB0085EC91
:10EBE0008093BC0062CF909154088091530898178D
:10EBF00058F5E091540881E08E0F80935408F0E0BE
:10EC0000ED5CF74F8081E9CFE091540881E08E0FF1
:10EC1000809354088091BB00F0E0ED5CF74F808357
:10EC200090915408809153089817C8F285E8D8CF7E
:10EC3000E091540881E08E0F809354088091BB00CE
:10EC4000F0E0ED5CF74F80838091560881115CCF36
:10EC500081E08093310884EA8093BC0010925708C9
:10EC600024CF85EC8093BC001092570880913B071D
:10EC7000803230F4E0913B07F0E0E55EF84F10821F
:10EC800060913B0770E0E0916B07F0916C078BE1BE
:10EC900097E0199510923B0708CF1092550834CF92
:10ECA0001092A2081092A10888EE93E0A0E0B0E0D4
:10ECB0008093A3089093A408A093A508B093A608F6
:10ECC00021E833E03093A00820939F0825EC30E042
:10ECD0003093AC082093AB0824EC30E03093AE08BE
:10ECE0002093AD0820EC30E03093B0082093AF08BB
:10ECF00021EC30E03093B2082093B10822EC30E0F0
:10ED00003093B4082093B30826EC30E03093B60873
:10ED10002093B5081092B8081092B9081092BA085A
:10ED20001092BB082FEF20933C0910923E091092DD
:10ED30003D0910924809109247094FEF5FEFBA0161
:10ED400040934309509344096093450970934609E1
:10ED500010924C0910924B0980934D0990934E09E3
:10ED6000A0934F09B093500983E993E090934A0927
:10ED7000809349091092CE0A1092CD0A85EA93E059
:10ED80009093CC0A8093CB0A1092060B1092070B3B
:10ED90001092080B1092D40A1092D30A1092D60A3D
:10EDA0001092D50A1092D80A81E08093D70A82E2A5
:10EDB0008093D90A1092DE0A1092DD0AE2EFFAE09F
:10EDC00020E03BE08FEF81932E173F07E1F791E0C2
:10EDD0009093EF0A2DE632E23093E50A2093E40A9D
:10EDE0009093E60A1092E70A1092E80A90E4909352
:10EDF000E90A1092EA0A2CE632E23093010B2093E2
:10EE0000000B28E433E03093D20A2093D10A9FE22A
:10EE10009093F60A90E39093F70A91E39093F40AA3
:10EE20008093F30A8093F20A0E94942F85EA93E07C
:10EE30009093CC0A8093CB0A87E38093B30A109215
:10EE4000B40A1092B50A1092B60A1092B70A10923C
:10EE5000B80A1092B90A1092BA0A1092BB0A10921C
:10EE6000BC0A1092BD0A1092BE0A1092BF0A1092FC
:10EE7000C00A1092C10A1092C20A42E350E05093B5
:10EE8000C40A4093C30A1092C60A1092C50A20ED24
:10EE900037E03093C80A2093C70A88EC90E090933B
:10EEA000CA0A8093C90A68E360939B0A10929C0A7D
:10EEB00010929D0A10929E0A10929F0A1092A00A28
:10EEC0001092A10A1092A20A1092A30A1092A40A08
:10EED0001092A50A1092A60A1092A70A1092A80AE8
:10EEE0001092A90A1092AA0A5093AC0A4093AB0A56
:10EEF0001092AE0A1092AD0A3093B00A2093AF0A76
:10EF00009093B20A8093B10A69E36093830A1092E6
:10EF1000840A1092850A1092860A1092870A10922B
:10EF2000880A1092890A10928A0A10928B0A10920B
:10EF30008C0A10928D0A10928E0A10928F0A1092EB
:10EF4000900A1092910A1092920A5093940A409358
:10EF5000930A1092960A1092950A3093980A209379
:10EF6000970A90939A0A8093990A6AE360936B0ACE
:10EF700010926C0A10926D0A10926E0A10926F0A2B
:10EF80001092700A1092710A1092720A1092730A0B
:10EF90001092740A1092750A1092760A1092770AEB
:10EFA0001092780A1092790A10927A0A50937C0A89
:10EFB00040937B0A10927E0A10927D0A3093800A59
:10EFC00020937F0A9093820A8093810A6BE3609377
:10EFD000530A1092540A1092550A1092560A10922F
:10EFE000570A1092580A1092590A10925A0A10920F
:10EFF0005B0A10925C0A10925D0A10925E0A1092EF
:10F000005F0A1092600A1092610A1092620A50938D
:10F01000640A4093630A1092660A1092650A30935C
:10F02000680A2093670A90936A0A8093690A6CE3DE
:10F0300060933B0A10923C0A10923D0A10923E0ADD
:10F0400010923F0A1092400A1092410A1092420A0E
:10F050001092430A1092440A1092450A1092460AEE
:10F060001092470A1092480A1092490A10924A0ACE
:10F0700050934C0A40934B0A10924E0A10924D0A3C
:10F080003093500A20934F0A9093520A8093510A6A
:10F090006DE36093230A1092240A1092250A1092BD
:10F0A000260A1092270A1092280A1092290A109212
:10F0B0002A0A10922B0A10922C0A10922D0A1092F2
:10F0C0002E0A10922F0A1092300A1092310A1092D2
:10F0D000320A5093340A4093330A1092360A10923F
:10F0E000350A3093380A2093370A90933A0A80936E
:10F0F000390A86E380935509109257090895CF93F2
:10F10000DF93CDB7DEB76C970FB6F894DEBF0FBEB6
:10F11000CDBF789484B5826084BD84B5816084BDA0
:10F1200085B5826085BD85B5816085BD80916E00A5
:10F13000816080936E0010928100809181008260D6
:10F140008093810080918100816080938100809113
:10F1500080008160809380008091B1008460809302
:10F16000B1008091B00081608093B00080919100E7
:10F1700082608093910080919100816080939100E2
:10F18000809190008160809390008091A1008260C6
:10F190008093A1008091A10081608093A100809163
:10F1A000A00081608093A000809121018260809303
:10F1B00021018091210181608093210180912001B2
:10F1C00081608093200180917A00846080937A002E
:10F1D00080917A00826080937A0080917A008160C9
:10F1E00080937A0080917A00806880937A001092F0
:10F1F000C10060E08AE20E949B2B61E08AE20E94EB
:10F200006E2B61E08DE20E949B2B61E08DE20E94FB
:10F210006E2B61E08DE00E949B2B61E082E00E94FA
:10F220009B2B61E083E00E949B2B61E084E00E94C5
:10F230009B2B61E085E00E949B2B61E086E00E94B1
:10F240009B2B61E087E00E949B2B61E088E00E949D
:10F250009B2B61E08CE00E949B2B1FB7F894809160
:10F260006A07811127C0E6E7FAE18491E0E3FAE159
:10F270009491E82FF0E0EE0FFF1FEF51F64EA591AD
:10F28000B491EC91E92321F461E085E30E946E2BB7
:10F2900061E085E30E949B2B8CB580618CBD8CB5B1
:10F2A00080648CBD61E084E30E949B2B61E083E37A
:10F2B0000E949B2B80916A078F5F80936A071FBF14
:10F2C00061E08CE20E949B2B61E08CE20E946E2B3D
:10F2D00061E08EE20E949B2B61E08EE20E946E2B29
:10F2E00085E0EEE4F3E0DE01119601900D928A953F
:10F2F000E1F764E670E080E090E00E94F52D60E7C1
:10F3000087E00E94C53E60E082E00E94C53E60E06A
:10F3100081E00E94C53E82E00E94E63E682F616067
:10F3200082E00E94C53E81E00E94E63E682F6E7F2B
:10F3300081E00E94C53E80E00E94E63E682F6C603E
:10F3400080E00E94C53E63E083E00E94C53E83E00A
:10F350000E94E63E12E0180F90E080E00E94623BBF
:10F360008AE20E94C43E9E012F5F3F4F79011150F7
:10F3700008F02BC481E090E00E94623B80E00E9494
:10F38000E63E682F616080E00E94C53E60E181E159
:10F390000E94C53E64E685E00E94C53E80E00E9472
:10F3A000E63E682F626080E00E94C53E62E070E049
:10F3B00080E090E00E94F52D1092700710926F0788
:10F3C00010925E08109280080E94BA3480EB9AE294
:10F3D00090936E0780936D0781EB9AE290936C0790
:10F3E00080936B0783EB9AE00E94F32E8BE99AE0FF
:10F3F0000E94F32E83E89AE00E94F32E8BE69AE0B7
:10F400000E94F32E83E59AE00E94F32E8BE39AE0AC
:10F410000E94F32E83E29AE00E94F32EF89482E099
:10F420008093B0008093B10094E69093B300109263
:10F43000B200809370007894809356091092220A4B
:10F440008091550960E00E949B2B10E000E078015C
:10F45000F7E1EF0EF11CC8010E94138DF801EB5883
:10F46000FD4F80830F5F1F4F0E151F05A1F70A3850
:10F47000110569F7F12CE12C98012D563E4F6901D9
:10F48000C701800F911F0E94138DF601EE0DFF1D25
:10F4900080833FEFE31AF30A46E1E416F10481F7B3
:10F4A0000A5E1F4F023E110529F78091280290E065
:10F4B000909376078093750780913E0290E0909339
:10F4C0007407809373078091540290E090937207C1
:10F4D0008093710785E0E82E83E0F82EC8010E9432
:10F4E000138DF70181937F010F5F1F4F0E3E1105B2
:10F4F000A9F70E945D400E94A24C0E94F13B8091BE
:10F500008A07811145C010927C0710927B078FEF0C
:10F5100080937F0780938007809381078093820781
:10F52000809383078093840781E0809385071092FE
:10F5300087071092860710927E0710927D078091B0
:10F54000990890919A08892B31F489E797E0909374
:10F550009A0880939908E0917707F091780730979F
:10F5600021F089E797E09583848389E797E090937A
:10F5700078078093770710928907109288078FE6A3
:10F5800093E090937A078093790781E080938A07CC
:10F59000809104018260809304018CE997E090934C
:10F5A0007C0780937B078EE190E0909387078093A0
:10F5B000860780913F0990914009A0914109B0913F
:10F5C0004209843CF9E09F07A105B10520F484ECD1
:10F5D00099E0A0E0B0E080933F0990934009A093A8
:10F5E0004109B093420980EF80933C090CE917E090
:10F5F000F8011382148215820E94D12C0D5F1F4FD7
:10F60000F7E0033F1F07A1F7772473941AE0E12E78
:10F61000F12CCC24C394DD24D3946EE571E080E01A
:10F6200090E00E94F52D0E94994E0E942423892B80
:10F6300011F00E941142CE010F960E94FA3E8A8973
:10F6400090E09093300880932F088B8990E09093FE
:10F650002E0880932D080C8910E010932C0800933D
:10F660002B08888990E090932A088093290889893B
:10F6700090E090932808809327088F8590E080532E
:10F68000984F9093260880932508CE010F960E94EC
:10F69000F72E90E09093240880932308809121080E
:10F6A0009091220801969093220880932108029756
:10F6B0004CF0809120088725809320081092220822
:10F6C0001092210880911E0890911F0880179107C1
:10F6D00024F00115110509F05DC010931F08009377
:10F6E0001E08012B09F456C080917B00886080932E
:10F6F0007B0080E480937C0080917A00806480931A
:10F700007A0080917A0086FDFCCF8091780020916C
:10F710007900322F282F80E094E0821B930B909386
:10F720001D0880931C08B0901B08B394B0921B086E
:10F730008AE20E94462B892BC9F460E08FEF0E9479
:10F74000C53E86FFFACF60E487E00E94C53E60E0D8
:10F750008FEF0E94C53E90E0959587958770873022
:10F7600009F039C281E090E00E94623B25E0B212CC
:10F7700007C010921B0880911A08872580931A08E9
:10F780008091190881110E94F13B80911808811124
:10F790000E94F13B0E94F52F7EE1672EEBE09E2E4A
:10F7A000F2E0BF2EA9E0AA2E8091160890911708CA
:10F7B000892B11F40E94CD5880911608909117085A
:10F7C000029709F42CC280911608909117080597AA
:10F7D00009F02DC1512C412C312C212C812C6EE5AE
:10F7E00071E080E090E00E94F52DCE0101960E942C
:10F7F000FA3E8C8190E09093300880932F088D81A1
:10F8000090E090932E0880932D088E8190E0909345
:10F810002C0880932B088A8190E090932A0880938B
:10F8200029080E94F52FECE8FAE0E419F509CF0168
:10F830006CE370E00E946F8F8B0144EC46039001F3
:10F84000479F300D11242E0F3F1FCF0168E572E056
:10F850000E946F8F7E8B6D8BC801B7010E946F8FE6
:10F86000988F8F8BC901B7010E946F8F7A8F698F34
:10F870009C8F8B8FD092EF0A07E81EE120E440E8CE
:10F8800060E080E00E94E9331092EF0A8FE395E296
:10F890000E94FA286092060B9092070B80912F0825
:10F8A00090913008B7010E946F8FCB010E94564E95
:10F8B00080912F0890913008B7010E946F8F0E94AD
:10F8C000564E89EB94E00E94364F80912D0890911E
:10F8D0002E08B7010E946F8FCB010E94564E809177
:10F8E0002D0890912E08B7010E946F8F0E94564EEE
:10F8F00089EB94E00E94364F80912B0890912C0860
:10F90000B7010E946F8FCB010E94564E80912B0849
:10F9100090912C08B7010E946F8F0E94564ED09292
:10F92000EF0A8EEE9AE30E94FA289092060BA092BC
:10F93000070B89EB94E00E94364F1092060BA092C1
:10F94000070B8D899E890E94564E8F89988D0E9443
:10F95000564E60E16093060BA092070B898D9A8D3D
:10F960000E94564E8B8D9C8D0E94564E0E942530D3
:10F97000811180CF0E942423892B39F1B09256093E
:10F980001092220A61E08DE00E946E2B8091850822
:10F9900090918608A0918708B091880884379A468C
:10F9A000A041BE4021F43DE8432E3AE0532E64E6E8
:10F9B00070E080E090E00E94F52DB0925609109220
:10F9C000220A60E08DE00E946E2B81100EC061E083
:10F9D00086E00E946E2B6AEF70E088E00E94D72BD1
:10F9E0006AEF70E08CE00E94D72B80912B089091F9
:10F9F0002C088215930519F0FFEF4F1A5F0A2DE8C6
:10FA000042162AE052060CF4CCC21092170810924B
:10FA1000160870E060E088E00E94D72B70E060E09C
:10FA20008CE00E94D72B60E086E00E946E2B8091D4
:10FA3000150881110E9468528091140881110E945A
:10FA4000DE5B8091130881110E943A4F8091120869
:10FA500081110E94706A8091110881110E946F6566
:10FA6000D092EF0A8EEE9AE30E94FA28B092060B2B
:10FA7000A092070B80910F0890911008039780F4D3
:10FA8000809100080E94B93E809101080E94B93E11
:10FA9000809102080E94B93E809103080E94B93EFD
:10FAA00080910F0890911008069731F48091FD071E
:10FAB0009091FE070E94564E80910F089091100879
:10FAC000079731F48091FB079091FC070E94564EF6
:10FAD00081ED94E00E94364F84E68093060BA0925D
:10FAE000070B8091F9079091FA070E94564E80917A
:10FAF00019080E94824E809118080E94824E8091BF
:10FB0000F80790E00E94564E0E94253081114CCE9D
:10FB100080912B0890912C08892B51F48091F90742
:10FB20009091FA07892B21F40E945D400E94A24C1B
:10FB300080912B0890912C084E9751F48091F907F1
:10FB40009091FA07892B21F40E945D400E94A24CFB
:10FB50008091270890912808892B21F41092F707AB
:10FB60001092F60780912D0890912E08009709F0C9
:10FB700022C220912B0830912C082530310511F03C
:10FB80000C94F68C20914703222309F414C240916F
:10FB90002F0850913008FA01EE0FFF1FE95EFC4F6D
:10FBA00020911C0830911D0831832083E7E1F3E0A8
:10FBB00030E020E0421753070CF4F7C161917191D6
:10FBC000860F971F2F5F3F4FF5CFF70181917F0180
:10FBD0000E94C43ECCCB90E080E00E94623B80E675
:10FBE0000E94C43E80E00E94BD3EA82E81E090E0CD
:10FBF0000E94623B90E080E00E94623B81E60E94AE
:10FC0000C43E0FEF17E0AA94FFEFAF1609F4AACD98
:10FC100080E00E94BD3EF80181938F01F4CF8824DB
:10FC20008394512CCE0101960E94FA3E8C8190E083
:10FC30009093300880932F088D8190E090932E0848
:10FC400080932D088E8190E090932C0880932B0850
:10FC500064E670E080E090E00E94F52D539433E07C
:10FC6000531206C080912008872580932008512CCC
:10FC70000E94F52FD092EF0A07E81AE120E440E84D
:10FC800060E080E00E94E9331092EF0A8FE395E292
:10FC90000E94FA286092060B9092070B80912F0821
:10FCA00090913008B7010E946F8FCB010E94564E91
:10FCB00080912F0890913008B7010E946F8F0E94A9
:10FCC000564E89EB94E00E94364F80912D0890911A
:10FCD0002E08B7010E946F8FCB010E94564E809173
:10FCE0002D0890912E08B7010E946F8F0E94564EEA
:10FCF00089EB94E00E94364F80912B0890912C085C
:10FD0000B7010E946F8FCB010E94564E80912B0845
:10FD100090912C08B7010E946F8F0E94564E41E0CF
:10FD2000841243C08091200881110C94D68C1092CB
:10FD3000EF0A21E041E364E185E20E94C7330E94BB
:10FD40002530811197CF0E942423892B09F46ACF93
:10FD5000B09256091092220A61E08DE00E946E2B4B
:10FD60008091850890918608A0918708B0918808B5
:10FD700085314BE8940740E9A4074EE0B40709F049
:10FD800086C062E0861609F479C0E1E08E1609F4B7
:10FD900078C0F3E08F1609F477C02CEF280D2230DD
:10FDA00008F091C058E0852E8EC062E086120CC02B
:10FDB0008091200881110C94DA8C1092EF0A21E0D6
:10FDC0004BE063E286E0B9CF83E088120CC08091FB
:10FDD000200881110C94DE8C1092EF0A21E04DE096
:10FDE00063E288E2AACF94E089120CC080912008D7
:10FDF00081110C94E28C1092EF0A21E04BE063E257
:10FE00008AE49BCFE5E08E120CC08091200881111E
:10FE10000C94E68C1092EF0A21E04DE063E28CE650
:10FE20008CCFF6E08F120CC08091200881110C94C9
:10FE3000EA8C1092EF0A21E047E065E389E17DCF8B
:10FE400027E082120CC08091200881110C94EE8C66
:10FE50001092EF0A21E047E065E38DE36ECF38E0D2
:10FE600083126DCF8091200881110C94F28C109236
:10FE7000EF0A21E04CE065E38BE55FCF66E0862E7C
:10FE80008CCF52E0852E89CF47E0842E86CF8539EE
:10FE90002BE0920720E9A2072EE0B207F1F432E04E
:10FEA000831611F40C94FF8C46E0841611F40C9424
:10FEB000038D68E0861611F40C94078DE7E08E162A
:10FEC00011F40C940B8D84379A46A041BE4099F4EE
:10FED00010921708109216082FC0853DFBE49F076B
:10FEE000F0E9AF07FEE0BF0741F4839429E08216F2
:10FEF00011F40C940F8D10E020C085353BEC930776
:10FF000030E9A3073EE0B30731F48A948110F3CFC0
:10FF100088E0882EF0CF84304AE1940740E1A407BE
:10FF20004EE0B40781F661E0861219C010921708FE
:10FF3000109216088092150811E064E670E080E0E7
:10FF400090E00E94F52DB09256091092220A60E0CE
:10FF50008DE00E946E2B112309F464CE34CC82E034
:10FF6000881207C01092170810921608D092140831
:10FF7000E3CF93E0891207C0109217081092160879
:10FF8000D0921108D9CFE6E08E1207C01092170860
:10FF900010921608D0921208CFCFF8E08F1661F3B6
:10FFA000AACF882483941C011ACC9093F7078093DE
:10FFB000F607109247038091160890911708892B35
:10FFC00009F06AC200912B0810912C08013011052C
:10FFD00079F00B30110561F00531110549F00F3151
:10FFE000110531F00932110519F00333110581F5BE
:10FFF00066E1CE0101960E944B37CE0101960E9428
:020000021000EC
:1000000013376CECCE0101960E9443296EE4CE01B9
:1000100001960E9443296DE7CE0101960E94432973
:100020006CEFCE0101960E9443296FE7CE01019645
:100030000E944329CE0101960E9413376CECCE0139
:1000400001960E94432964E4CE0101960E9443294F
:100050000230110581F00C30110569F006311105EF
:1000600051F00032110539F00A32110521F0043344
:10007000110509F06CC068E1CE0101960E944B3772
:10008000CE0101960E9413376CECCE0101960E94BE
:10009000432964E4CE0101960E94432968EC70E094
:1000A00080E090E00E94F52D66E1CE0101960E946D
:1000B0004B37CE0101960E9413376CECCE010196AE
:1000C0000E9443296EEBCE0101960E944329CE0186
:1000D00001960E94CF36B82ECE0101960E94CF36EF
:1000E00087FF07C0982F8B2D919581959109B82E88
:1000F000892F9B2D9F70492F440F990F990F990FAE
:10010000490F50E0B4E055954795BA95E1F7282F8F
:1001100030E0322F22272B0D311D94E035952795A5
:100120009A95E1F7222309F45BC1209302038091A1
:100130000203FA012AE0829FE00DF11D1124CF0194
:10014000B7010E946F8F6093020380930103033015
:10015000110581F00D30110569F00731110551F0DD
:100160000132110539F00B32110521F0053311056B
:1001700009F065C06AE1CE0101960E944B37CE01BD
:1001800001960E9413376CECCE0101960E94432920
:1001900064E4CE0101960E94432968EC70E080E09F
:1001A00090E00E94F52D68E1CE0101960E944B3748
:1001B000CE0101960E9413376CECCE0101960E948D
:1001C00043296EEBCE0101960E944329CE01019690
:1001D0000E94CF36B82ECE0101960E94CF3687FFFF
:1001E00007C0982F8B2D919581959109B82E892F55
:1001F0003B2D3F70232F220F330F330F330F90E02F
:10020000982F8827AC014B0D511DF4E0559547956B
:10021000FA95E1F7822F830F90E0A4E095958795FA
:10022000AA95E1F73AE0439F800D911D11240397B1
:10023000B7010E946F8F609300038093FF02043028
:10024000110581F00E30110569F00831110551F0EA
:100250000232110539F00C32110521F00633110577
:1002600009F01AC168EC70E080E090E00E94F52D82
:100270006AE1CE0101960E944B37CE0101960E94A1
:1002800013376CECCE0101960E9443296EEBCE0130
:1002900001960E944329CE0101960E94CF36182F65
:1002A000CE0101960E94CF3687FF07C0982F812F7D
:1002B000919581959109182F892F312F3F70232F08
:1002C000220F330F330F330F90E0982F8827AC01A4
:1002D000410F511D64E0559547956A95E1F7822FCE
:1002E000830F90E074E0959587957A95E1F76AE041
:1002F000469F800D911D1124B7010E946F8FB62E6D
:1003000060930403982E8093030380910C03813043
:1003100009F0C2C000910D03A09002030A1164C04D
:1003200090910E0380910103981780F480919307B8
:10033000811104C061E086E00E946E2B61E089E0DB
:100340000E946E2BC0929207C092930710910F03E8
:10035000A1125EC09091100380910103891770F47F
:1003600080919307811104C060E086E00E946E2BAB
:1003700060E089E00E946E2B10929207A09000032B
:100380000A114AC090910E038091FF02981780F4E1
:1003900080919307811104C061E086E00E946E2B7A
:1003A00061E08AE00E946E2BC0929207C092930790
:1003B0001A1145C0909110038091FF02891708F02F
:1003C00041C080919307811104C060E086E00E94E3
:1003D0006E2B60E08AE00E946E2B1092920732C072
:1003E00088E180930203A3CE0A1508F0AFCF809175
:1003F0009307811104C061E086E00E946E2BC092D9
:10040000930761E089E00E946E2BC09292079ECF15
:10041000A11608F4A5CFB2CF0A1550F68091930724
:10042000811104C061E086E00E946E2BC0929307A8
:1004300061E08AE00E946E2BC0929207B9CFA116AC
:1004400008F4BFCFB012D7C080910E03891580F495
:1004500080919307811104C061E086E00E946E2BB9
:1004600061E08BE00E946E2BC0929207C0929307CE
:10047000B112D5C080911003981670F48091930743
:10048000811104C060E086E00E946E2B60E08BE08A
:100490000E946E2B1092920780910F089091100885
:1004A0000197C1F48091150390911603019791F47F
:1004B0000CE917E0F8011382148215820E94D12CF6
:1004C0000A5F1F4FF7E0063F1F07A1F710921603C0
:1004D0001092150380910F08909110080297F1F483
:1004E00080911503909116030197C1F40CE917E070
:1004F000F8011682178210861382148215821186E3
:10050000128613860E94D12C045F1F4FF7E00C3F28
:100510001F0771F7109216031092150380910F08B0
:1005200090911008069709F0D9C08091FD0790912D
:10053000FE0701969093FE078093FD0780911503B7
:1005400090911603019709F082C080912108909143
:100550002208892B49F480919A0790919B07019674
:1005600090939B0780939A0780919A0790919B079D
:100570000B970CF46CC080911303909114035C01F1
:1005800022E0A21AB108B0921403A09213031092B1
:100590009B0710929A078C01000F111F080F191F5B
:1005A0000A56184FAEE18A2E912CB4E63B2E8CE30E
:1005B000482E9AE5592E22E0622E809113039091E5
:1005C00014039401281B390BA216B30664F5F80135
:1005D00030824182528222E030E030931203209335
:1005E000110360923C090E94D12C32E0A30EB11C91
:1005F0000A5F1F4FE2CF0B1508F03ACF80919307A7
:10060000811104C061E086E00E946E2BC0929307C6
:1006100061E08BE00E946E2BC092920729CFB11649
:1006200008F42CCF39CF1092990710929807892B94
:1006300071F4109216031092150310929B071092FA
:100640009A0780E190E090931403809313038091C4
:10065000210890912208892B49F480919807909164
:10066000990701969093990780939807809198072E
:1006700090919907CD9794F188E290E09093990733
:1006800080939807809111039091120324E130E048
:100690008035910594F42AE030E0883291056CF4BD
:1006A0008A30910514F40C94E28B2EE130E0309303
:1006B00099072093980725E030E0820F931F813F30
:1006C000910514F00C94EA8B90931203809311031C
:1006D0008091110380933C090E94D12C80910F08D6
:1006E00090911008079711F00C94DE8B8091150300
:1006F00090911603019721F410921603109215039E
:100700008091FB079091FC0701969093FC078093E2
:10071000FB078091210890912208892B49F4809150
:100720009A0790919B07019690939B0780939A0755
:1007300080919A0790919B07CD9714F40C94DE8BCF
:1007400080919407909195070196909395078093D7
:10075000940710929B0710929A07019701F5A6EF54
:10076000AA2EA7E0BA2E0CE917E0BEE66B2E8FE0AA
:10077000882E9FE5992EF8016082818292826382A1
:10078000848295820E94D12C0A5F1F4FA016B10669
:1007900091F788E290E090939B0780939A0780916D
:1007A000940790919507029721F546EFA42E47E014
:1007B000B42E0CE917E053E7452E64E1562E7AE596
:1007C000972EEAE06E2EF0E58F2EF80140825182DE
:1007D00092829382648285820E94D12C0A5F1F4F8D
:1007E000A016B10691F788E290E090939B07809362
:1007F0009A078091940790919507039711F516EF4A
:10080000A12E17E0B12E0CE917E088E7582E99E1E8
:10081000692E20E5922E3CE3832EF80150826182FE
:1008200092829382148285820E94D12C0A5F1F4F8C
:10083000A016B10691F782E390E090939B07809316
:100840009A078091940790919507049721F566EF98
:10085000A62E67E0B62E0CE917E07DE7472EEEE105
:100860005E2EFBE46F2EACE38A2EB8E29B2EF801DD
:100870004082518262828382148295820E94D12CAE
:100880000A5F1F4FA016B10691F782E390E09093A4
:100890009B0780939A0780919407909195070597FD
:1008A00009F50CE917E092E8692E23E2822E36E47E
:1008B000932E48E2A42E54E1B52EF8016082818285
:1008C0009282A3821482B5820E94D12C0A5F1F4FAC
:1008D000F7E0063F1F0789F782E390E090939B07BC
:1008E00080939A078091940790919507069721F538
:1008F00076EFA72E77E0B72E0CE917E0E7E84E2E4B
:10090000F8E25F2EA1E46A2EB4E18B2E8AE0982EE5
:10091000F8014082518262828382148295820E9411
:10092000D12C0A5F1F4FA016B10691F782E390E029
:1009300090939B0780939A078091940790919507D5
:10094000079721F596EFA92E97E0B92E0CE917E04D
:100950002CE8422E3DE2532E4CE3642E5AE0852EC5
:1009600065E0962EF8014082518262828382148271
:1009700095820E94D12C0A5F1F4FA016B10691F7F5
:1009800082E390E090939B0780939A07809194076D
:10099000909195070897E9F40CE917E0A1E99A2EE0
:1009A000B7E3AB2E82E3B82EF8019082A182B28227
:1009B0001382148215820E94D12C0A5F1F4FF7E028
:1009C000063F1F0789F782E390E090939B0780938F
:1009D0009A0780919407909195070997D1F40CE9B3
:1009E00017E076E9972EE6E4AE2EF8E2BF2EF80186
:1009F0009082A182B2820E94D12C0A5F1F4FF7E041
:100A0000063F1F07A1F782E390E090939B07809336
:100A10009A0780919407909195070A97E9F436EF29
:100A2000A32E37E0B32E0CE917E046E9642E50E51B
:100A3000852E6EE1962EF8016082818292820E945C
:100A4000D12C0A5F1F4FA016B106A9F782E390E0F0
:100A500090939B0780939A078091940790919507B4
:100A60000B97E9F4B6EFAB2EB7E0BB2E0CE917E01D
:100A700086E9682E9AE5892E24E1922EF80160829B
:100A8000818292820E94D12C0A5F1F4FA016B1066C
:100A9000A9F782E390E090939B0780939A07809157
:100AA0009407909195070C97B9F476EFA72E77E00D
:100AB000B72E0CE917E0E6E96E2EFAE58F2EAAE0D4
:100AC0009A2EF8016082818292820E94D12C0A5F64
:100AD0001F4FA016B106A9F7809194079091950732
:100AE0000D97B9F436EFA32E37E0B32E0CE917E0DB
:100AF00040EA642E5AE5852E6AE0962EF80160825F
:100B0000818292820E94D12C0A5F1F4FA016B106EB
:100B1000A9F780919407909195070E97B9F4B6EFD5
:100B2000AB2EB7E0BB2E0CE917E08AEA682E9AE5F7
:100B3000892E2AE0922EF8016082818292820E94A0
:100B4000D12C0A5F1F4FA016B106A9F78091940718
:100B5000909195070F97B9F476EFA72E77E0B72E0F
:100B60000CE917E0E4EB6E2EFAE58F2EAAE09A2E40
:100B7000F8016082818292820E94D12C0A5F1F4F0D
:100B8000A016B106A9F78091940790919507469712
:100B9000E9F436EFA32E37E0B32E0CE917E045EA6F
:100BA000642E55E5852E6BE0962EF80160828182D9
:100BB00092820E94D12C0A5F1F4FA016B106A9F79E
:100BC0008EE190E090939B0780939A078091940721
:100BD000909195074797E9F416EFA12E17E0B12EF3
:100BE0000CE917E080EA682E90E5892E2CE0922E21
:100BF000F8016082818292820E94D12C0A5F1F4F8D
:100C0000A016B106A9F78EE190E090939B07809320
:100C10009A0780919407909195074897D1F40CE931
:100C200017E0FBE99F2EABE4AA2EBDE0BB2EF80136
:100C30009082A182B2820E94D12C0A5F1F4FF7E0FE
:100C4000063F1F07A1F78EE190E090939B078093EA
:100C50009A0780919407909195074997E9F456EF88
:100C6000A52E57E0B52E0CE917E06CE8662E76E469
:100C7000872EEEE09E2EF8016082818292820E9491
:100C8000D12C0A5F1F4FA016B106A9F78EE190E0A4
:100C900090939B0780939A07809194079091950772
:100CA0004A97E9F496EFA92E97E0B92E0CE917E0E0
:100CB00027E8622E31E4832E4FE0942EF801608203
:100CC000818292820E94D12C0A5F1F4FA016B1062A
:100CD000A9F78EE190E090939B0780939A0780910B
:100CE0009407909195074B97E9F4F6EFAF2EF7E054
:100CF000BF2E0CE917E0A2E86A2EBCE38B2E80E140
:100D0000982EF8016082818292820E94D12C0A5F23
:100D10001F4FA016B106A9F78EE190E090939B07B4
:100D200080939A0780919407909195074C97E9F4E6
:100D300056EFA52E57E0B52E0CE917E068E7662EB2
:100D400077E3872EE1E19E2EF80160828182928214
:100D50000E94D12C0A5F1F4FA016B106A9F78EE1A1
:100D600090E090939B0780939A07809194079091CD
:100D700095074D97D1F40CE917E02EE6922E32E359
:100D8000A32E42E1B42EF8019082A182B2820E9489
:100D9000D12C0A5F1F4FF7E0063F1F07A1F78EE136
:100DA00090E090939B0780939A078091940790918D
:100DB00095074E97D1F40CE917E0B4E69B2E8DE22F
:100DC000A82E93E1B92EF8019082A182B2820E94EE
:100DD000D12C0A5F1F4FF7E0063F1F07A1F78EE1F6
:100DE00090E090939B0780939A078091940790914D
:100DF00095074F97D1F40CE917E0EFE59E2EF8E246
:100E0000AF2EA4E1BA2EF8019082A182B2820E9494
:100E1000D12C0A5F1F4FF7E0063F1F07A1F78EE1B5
:100E200090E090939B0780939A078091940790910C
:100E300095078097D1F40CE917E05AE5952E63E207
:100E4000A62E73E1B72EF8019082A182B2820E9491
:100E5000D12C0A5F1F4FF7E0063F1F07A1F78EE175
:100E600090E090939B0780939A07809194079091CC
:100E700095078197E9F496EFA92E97E0B92E0CE932
:100E800017E025E5622E3EE1832E42E1942EF80123
:100E90006082818292820E94D12C0A5F1F4FA0162D
:100EA000B106A9F78EE190E090939B0780939A0793
:100EB00080919407909195078297E9F4F6EFAF2E11
:100EC000F7E0BF2E0CE917E0A0E56A2EB9E18B2E02
:100ED00081E1982EF8016082818292820E94D12C59
:100EE0000A5F1F4FA016B106A9F78EE190E090931C
:100EF0009B0780939A078091940790919507839719
:100F0000E9F456EFA52E57E0B52E0CE917E06BE497
:100F1000662E74E1872EE0E19E2EF80160828182C8
:100F200092820E94D12C0A5F1F4FA016B106A9F72A
:100F30008EE190E090939B0780939A0780919407AD
:100F4000909195078497E9F496EFA92E97E0B92E32
:100F50000CE917E026E4622E32E1832E4FE0942E56
:100F6000F8016082818292820E94D12C0A5F1F4F19
:100F7000A016B106A9F78EE190E090939B078093AD
:100F80009A0780919407909195078597E9F4F6EF79
:100F9000AF2EF7E0BF2E0CE917E0A1E46A2EBFE008
:100FA0008B2E8EE0982EF8016082818292820E94C0
:100FB000D12C0A5F1F4FA016B106A9F78EE190E071
:100FC00090939B0780939A0780919407909195073F
:100FD0008697E9F456EFA52E57E0B52E0CE917E0F9
:100FE00067E3662E7EE0872EEDE09E2EF80160829C
:100FF000818292820E94D12C0A5F1F4FA016B106F7
:10100000A9F78EE190E090939B0780939A078091D7
:101010009407909195078797D9F426EFA22E27E0A1
:10102000B22E0CE917E032E3832E4DE0942EF80146
:101030008082918292820E94D12C0A5F1F4FA0165B
:10104000B106A9F78EE190E090939B0780939A07F1
:1010500080919407909195078897E9F4A6EFAA2EBE
:10106000A7E0BA2E0CE917E0BDE26B2E8CE0882ECB
:101070009DE0992EF8016082818292820E94D12C9B
:101080000A5F1F4FA016B106A9F78EE190E090937A
:101090009B0780939A078091940790919507899771
:1010A000E9F466EFA62E67E0B62E0CE917E078E2C9
:1010B000672EEAE08E2EFDE09F2EF801608281828D
:1010C00092820E94D12C0A5F1F4FA016B106A9F789
:1010D0008EE190E090939B0780939A07809194070C
:1010E000909195078A97E9F426EFA22E27E0B22E79
:1010F0000CE917E033E2632E48E0842E5CE0952E85
:10110000F8016082818292820E94D12C0A5F1F4F77
:10111000A016B106A9F78EE190E090939B0780930B
:101120009A0780919407909195078B97E9F4A6EF21
:10113000AA2EA7E0BA2E0CE917E0BEE16B2E88E0DC
:10114000882E9BE0992EF8016082818292820E9413
:10115000D12C0A5F1F4FA016B106A9F78EE190E0CF
:1011600090939B0780939A0780919407909195079D
:101170008C97E9F466EFA62E67E0B62E0CE917E02F
:1011800079E1672EE7E08E2EFAE09F2EF80160826B
:10119000818292820E94D12C0A5F1F4FA016B10655
:1011A000A9F78EE190E090939B0780939A07809136
:1011B0009407909195078D97E9F426EFA22E27E0EA
:1011C000B22E0CE917E036E1632E47E0842E5AE098
:1011D000952EF8016082818292820E94D12C0A5F52
:1011E0001F4FA016B106A9F78EE190E090939B07E0
:1011F00080939A0780919407909195078E97E9F4D0
:10120000A6EFAA2EA7E0BA2E0CE917E0B4E16B2EE8
:1012100086E0882E99E0992EF80160828182928280
:101220000E94D12C0A5F1F4FA016B106A9F78EE1CC
:1012300090E090939B0780939A07809194079091F8
:1012400095078F97E9F466EFA62E67E0B62E0CE9B6
:1012500017E072E1672EE6E08E2EF9E09F2EF8018E
:101260006082818292820E94D12C0A5F1F4FA01659
:10127000B106A9F78EE190E090939B0780939A07BF
:101280008091940790919507C097E9F426EFA22EDC
:1012900027E0B22E0CE917E03FE0632E46E0842EF3
:1012A00059E0952EF8016082818292820E94D12CB1
:1012B0000A5F1F4FA016B106A9F78EE190E0909348
:1012C0009B0780939A078091940790919507C19707
:1012D000E9F4A6EFAA2EA7E0BA2E0CE917E0BEE0CB
:1012E0006B2E86E0882E99E0992EF801608281822B
:1012F00092820E94D12C0A5F1F4FA016B106A9F757
:101300008EE190E090939B0780939A0780919407D9
:1013100090919507C297E9F466EFA62E67E0B62E86
:101320000CE917E07DE0672EE5E08E2EF9E09F2EB8
:10133000F8016082818292820E94D12C0A5F1F4F45
:10134000A016B106A9F78EE190E090939B078093D9
:101350009A078091940790919507C397E9F426EF37
:10136000A22E27E0B22E0CE917E03BE0632E45E009
:10137000842E5AE0952EF8016082818292820E942A
:10138000D12C0A5F1F4FA016B106A9F78EE190E09D
:1013900090939B0780939A0780919407909195076B
:1013A000C497D9F4B6EFAB2EB7E0BB2E0CE917E02B
:1013B00089E0982E95E0892EF801908281829282B0
:1013C0000E94D12C0A5F1F4FA016B106A9F78EE12B
:1013D00090E090939B0780939A0780919407909157
:1013E0009507C597D9F4E6EFAE2EE7E0BE2E0CE9DF
:1013F00017E0F8E09F2EA5E08A2EF8019082818206
:1014000092820E94D12C0A5F1F4FA016B106A9F745
:101410008EE190E090939B0780939A0780919407C8
:1014200090919507C697E9F446EFA42E47E0B42EB5
:101430000CE917E056E0652E65E0862E78E0972EE1
:10144000F8016082818292820E94D12C0A5F1F4F34
:10145000A016B106A9F78EE190E090939B078093C8
:101460009A078091940790919507C797D9F496EFC2
:10147000A92E97E0B92E0CE917E025E0922E38E06E
:10148000832EF8019082918282820E94D12C0A5F81
:101490001F4FA016B106A9F78EE190E090939B072D
:1014A00080939A078091940790919507C897D1F4FB
:1014B0000CE917E0A4E09A2EB5E0AB2E88E0B82E38
:1014C000F8019082A182B2820E94D12C0A5F1F4F44
:1014D000F7E0063F1F07A1F78EE190E090939B078E
:1014E00080939A078091940790919507C997E9F4A2
:1014F00066EFA62E67E0B62E0CE917E073E0672EC4
:10150000E4E08E2EF7E09F2EF801608281829282C5
:101510000E94D12C0A5F1F4FA016B106A9F78EE1D9
:1015200090E090939B0780939A0780919407909105
:101530009507CA97D1F40CE917E032E0932E44E006
:10154000A42E56E0B52EF8019082A182B2820E94AC
:10155000D12C0A5F1F4FF7E0063F1F07A1F78EE16E
:1015600090E090939B0780939A07809194079091C5
:101570009507CB97C1F40CE917E094E0A92E25E07C
:10158000B22EF8017082A182B2820E94D12C0A5F31
:101590001F4FF7E0063F1F07A1F78EE190E0909301
:1015A0009B0780939A078091940790919507CC9719
:1015B000D9F4A6EFAA2EA7E0BA2E0CE917E0B2E004
:1015C0008B2E84E0982EF8011082818292820E94F4
:1015D000D12C0A5F1F4FA016B106A9F78EE190E04B
:1015E00090939B0780939A07809194079091950719
:1015F000CD97D9F476EFA72E77E0B72E0CE917E058
:10160000E2E08E2EF3E09F2EF8011082818292821A
:101610000E94D12C0A5F1F4FA016B106A9F78EE1D8
:1016200090E090939B0780939A0780919407909104
:101630009507CE97D1F410929C0710929D071092B7
:101640009E071092CC071092CD071092CE071092F1
:10165000F6071092F7071092F8070E94D12C8EE13E
:1016600090E090939B0780939A07809194079091C4
:101670009507CF9701F51092A2071092A307109239
:10168000A4071092D2071092D3071092D407109299
:10169000C6071092C7071092C8071092F007109261
:1016A000F1071092F2070E94D12C8EE190E0909306
:1016B0009B0780939A0780919407909195078034B7
:1016C000910501F51092A8071092A9071092AA0798
:1016D0001092D8071092D9071092DA071092C0071B
:1016E0001092C1071092C2071092EA071092EB07FE
:1016F0001092EC070E94D12C8EE190E090939B0712
:1017000080939A0780919407909195078134910571
:10171000D1F41092AE071092AF071092B00710925A
:10172000DE071092DF071092E0071092BA071092BE
:10173000BB071092BC070E94D12C8EE190E09093E1
:101740009B0780939A078091940790919507823424
:10175000910571F41092E4071092E5071092E607E4
:101760000E94D12C8EE190E090939B0780939A0782
:10177000809194079091950783349105F9F466EF71
:10178000A62E67E0B62E0CE917E0F8011082118250
:1017900012820E94D12C0A5F1F4FA016B106A9F732
:1017A00010929507109294071092FC071092FB0775
:1017B00081E090E09093100880930F080E947D2AAA
:1017C0000C940D7B109299071092980721E030E05D
:1017D0000C945D8380EF90E090931203809311034B
:1017E00086E090E09093100880930F08109299077C
:1017F0001092980780919607909197070196909381
:101800009707809396070597D1F40CE917E064E6F3
:10181000962E72E3A72EEFE5BE2EF8019082A182EC
:10182000B2820E94D12C0A5F1F4FF7E0063F1F07CC
:10183000A1F78EE190E090939907809398078091AB
:101840009607909197070697D1F40CE917E03EE6CA
:10185000932E48E2A42E59E6B52EF8019082A1827B
:10186000B2820E94D12C0A5F1F4FF7E0063F1F078C
:10187000A1F78EE190E0909399078093980780916B
:101880009607909197070797C1F40CE917E098E73E
:10189000B92E2EE1A22EF801B082A182B2820E945E
:1018A000D12C0A5F1F4FF7E0063F1F07A1F78EE11B
:1018B00090E0909399078093980780919607909174
:1018C00097070897D9F4A6EFAA2EA7E0BA2E0CE93D
:1018D00017E0B2E89B2E8EE1882EF801908281827B
:1018E00092820E94D12C0A5F1F4FA016B106A9F761
:1018F0008EE190E0909399078093980780919607E6
:10190000909197070997E9F466EFA62E67E0B62E47
:101910000CE917E078EC672EE2E38E2EF0EF9F2EB5
:10192000F8016082818292820E94D12C0A5F1F4F4F
:10193000A016B106A9F788E290E0909399078093EA
:10194000980780919607909197070A9711F00C9449
:10195000688326EFA22E27E0B22E0CE917E03CEDBB
:10196000632E46E4842E50EF952EF801608281822A
:1019700092820E94D12C0D5F1F4FA016B106A9F7CD
:10198000109297071092960781E090E090931008CC
:1019900080930F081092FE071092FD0780E190E0FF
:1019A00090931403809313030C9468838092EF0A3E
:1019B0000C94997ED092EF0A0C94DF7ED092EF0ABD
:1019C0000C94EE7ED092EF0A0C94FD7ED092EF0A3A
:1019D0000C940C7FD092EF0A0C941B7FD092EF0AEC
:1019E0000C942A7FD092EF0A0C94397F263031056F
:1019F00011F00C94DB7FC09247030C94DB7F8824AA
:101A000083940C94637F42E0842E0C94637F34E0D3
:101A1000832E0C94637F23E0822E0C94637F8824B2
:101A200083940C947B7FF999FECF92BD81BDF89A87
:101A3000992780B50895262FF999FECF1FBA92BD38
:101A400081BD20BD0FB6F894FA9AF99A0FBE01969F
:101A500008955058BB27AA270ED075C166D130F023
:101A60006BD120F031F49F3F11F41EF45BC10EF4F2
:101A7000E095E7FB51C1E92F77D180F3BA176207F0
:101A800073078407950718F071F49EF58FC10EF463
:101A9000E0950B2EBA2FA02D0B01B90190010C017E
:101AA000CA01A0011124FF27591B99F0593F50F496
:101AB000503E68F11A16F040A22F232F342F4427EE
:101AC000585FF3CF469537952795A795F0405395E6
:101AD000C9F77EF41F16BA0B620B730B840BBAF0B6
:101AE0009150A1F0FF0FBB1F661F771F881FC2F721
:101AF0000EC0BA0F621F731F841F48F48795779535
:101B00006795B795F7959E3F08F0B3CF9395880FEB
:101B100008F09927EE0F979587950895D9D008F486
:101B200081E008950CD00FC107D140F0FED030F015
:101B300021F45F3F19F0F0C0511139C1F3C014D145
:101B400098F39923C9F35523B1F3951B550BBB2784
:101B5000AA2762177307840738F09F5F5F4F220F31
:101B6000331F441FAA1FA9F333D00E2E3AF0E0E82A
:101B700030D091505040E695001CCAF729D0FE2F76
:101B800027D0660F771F881FBB1F26173707480708
:101B9000AB07B0E809F0BB0B802DBF01FF279358BE
:101BA0005F4F2AF09E3F510568F0B6C000C15F3F0D
:101BB000ECF3983EDCF3869577956795B795F795A6
:101BC0009F5FC9F7880F911D9695879597F908959E
:101BD000E1E0660F771F881FBB1F6217730784073A
:101BE000BA0720F0621B730B840BBA0BEE1F88F749
:101BF000E095089504D06894B111D9C00895BCD07F
:101C000088F09F5790F0B92F9927B751A0F0D1F0E5
